:100000000C946F1B0C94A11B0C94A11B0C94A11BB2
:100010000C94A11B0C94A11B0C94A11B0C94A11B70
:100020000C94A11B0C94A11B0C94A11B0C94A11B60
:100030000C94A11B0C9471360C94A11B0C94A11B65
:100040000C94A11B0C94A11B0C94A11B0C94A11B40
:100050000C94A11B0C94A11B0C94A11B0C94A11B30
:100060000C94A11B0C94FC1B0C94C01C0C94A11BA5
:100070000C94A11B0C94A11B0C94A11B0C94A11B10
:100080000C94A11B0C94A11B0C94A11B0C94A11B00
:100090000C94F41C0C945A1D0C94A11B0C94A11BE1
:1000A0000C94A11B0C94A11B0C94A11B0C94A11BE0
:1000B0000C94A11B0C94A11B0C94A11B0C94A11BD0
:1000C0000C94A11B0C94A11B0C94A11B0C948E1DD1
:1000D0000C94F41D0C94A11B0C94281E0C948E1EE1
:1000E0000C94A11B777AE57A1C7A6579E57A2478F5
:1000F000E57AE57A9A79E57AE57AE879E57AE57A52
:100100002078F178E57A2878E57AE57AE57AE57A73
:10011000E57AE578B4793379E57AE57AE57AE57ACE
:10012000E57AE57A777AE57A1C7A6579E57A247852
:10013000E57AE57A9A79E57AE57AE879E57AE57A11
:100140002078F178E57A2878E57AE57AE57AE57A33
:10015000E57AE578B4793379FA978B97559875965F
:1001600055985598C09755985598559855985598BD
:10017000719617975598799655985598559855981A
:1001800055980B97DA9759975598559855985598CB
:100190005598559855985598FA978B975598759600
:1001A00055985598C097559855985598559855987D
:1001B00071961797559879965598559855985598DA
:1001C00055980B97DA9759978BBE69BD2BBE69BDC1
:1001D00069BDA3BD69BD69BDA9BF69BD69BD69BD73
:1001E0009EBE69BD82BD69BD69BD69BDCFBD6BBD28
:1001F00069BD69BD01BFFABD69BD69BD69BD69BDA4
:1002000069BD69BD69BD69BD8BBE69BD2BBE69BDD8
:1002100069BDA3BD69BD69BDA9BF69BD69BD69BD32
:100220009EBE69BD82BD69BD69BD69BDCFBD6BBDE7
:1002300069BD69BD01BFFABD202C3A0D0A09002035
:100240002C3A3D0D0A00706D310000000000706D09
:10025000320000000000706D330000000000636693
:10026000670000000000626F6172644944007365BA
:1002700074446C79000069640000000000003132B1
:100280003363626469313233434244490050494226
:100290000053656E64696E67204E414B2066726F35
:1002A0006D2030782530345820746F203078253018
:1002B00034580053656E64696E672041434B206675
:1002C000726F6D2030782530345820746F2030786C
:1002D0002530345800504942207665722E2025641E
:1002E0002E25642E25642E20426F617264204944BD
:1002F000203D203078253032582E20506F7765729F
:1003000020446F776E2044656C6179203D20256420
:10031000207365632E004F4B202D2D20506F776585
:100320007220646F776E2064656C617920736574E8
:1003300020746F202564207365636F6E6473004FB3
:100340004B202D2D20426F61726420494420776933
:100350006C6C2062652025303258206166746572AD
:10036000207061796C6F6164207265626F6F7400D8
:1003700063666720726573756C743A203C25733E22
:1003800000506F77657220446F776E2044656C6112
:1003900079203D202564207365636F6E647300507F
:1003A0004D25643D25732000534D4300434F4D4D73
:1003B00000504D25642C2044657669636520616C8E
:1003C00072656164792068657265004661696C696F
:1003D0006E672E2E2E006E756D6265722E2E2E00AB
:1003E000534D4300434F4D4D00436F6D6D616E643F
:1003F00020706172616D733A203C25733E00436F3B
:100400006D6D616E642069733A203C25633E004245
:10041000616420636F6D6D616E642E20526573752B
:100420006C7420636F64653A203C25643E0050493B
:10043000420050726F63657373696E6720636F6EFD
:10044000736F6C6520696E7075743A203C25733E3D
:100450000053656E74204E414B2E2E2E0053656E58
:1004600064696E67204E414B0053656E64696E6728
:100470002041434B20746F2030782530347820663B
:10048000726F6D2030782530347800546F6F206D96
:10049000616E7920636F6D6D616E647300556E6B74
:1004A0006E6F776E2064657374696E6174696F6EC8
:1004B000004C656E67746820746F6F206C617267A2
:1004C000650050726F63657373696E6720436F6E6A
:1004D000736F6C6520496E7075742E2E2E2E004140
:1004E000646472657373206F7574206F6620726127
:1004F0006E67652E00416464726573733D3D3030F4
:1005000030302E00466F7277617264696E67206DBD
:1005100065737361676520746F2030782530347897
:100520000D0A00526563656976656420756E6B6EB1
:100530006F776E206D657373616765207479706580
:100540003A203078257800526563656976656420C5
:1005500073657269616C20706F727420706173735F
:10056000207468726F756768207265717565737441
:1005700000526563656976656420666F72776172A3
:100580006420636F6D6D616E6400526563656976AA
:10059000656420706F776572206E6F746966696339
:1005A0006174696F6E005265636569766564207277
:1005B0006571756573742077616974696E67207001
:1005C00061636B657400526563656976656420508C
:1005D0004942207374617475732072657175657317
:1005E000740052656365697665642069642072658C
:1005F000717565737400524543563A095372633AF4
:1006000030782530345809446573743A3078253091
:10061000345809547970653A307825303458000DD3
:100620000A426F6172642049443D253032642C20B7
:100630005461736B2049443D253032642C20546151
:10064000736B206973206E6F7420757365642F75EA
:100650006E6B6E6B6F776E0D0A0D0A000D0A426F9E
:100660006172642049443D253032642C205461730A
:100670006B2049443D253032642C205461736B203B
:1006800052756E6E696E67206973204D4241524902
:1006900020434F322053656E736F720D0A0D0A00AE
:1006A0000D0A426F6172642049443D253032642C4A
:1006B000205461736B2049443D253032642C205412
:1006C00061736B2052756E6E696E6720697320547A
:1006D000656C6564796E652041544D0D0A0D0A0004
:1006E0000D0A426F6172642049443D253032642C0A
:1006F000205461736B2049443D253032642C2054D2
:1007000061736B2052756E6E696E6720697320612C
:1007100020506F776572204F6E2F4F6666205365AD
:100720006E736F720D0A0D0A000D0A426F617264DA
:100730002049443D253032642C205461736B20499C
:10074000443D253032642C205461736B2052756E09
:100750006E696E6720697320616E20456D707479D3
:1007600020504D2053656E736F720D0A0D0A000DF7
:100770000A426F6172642049443D253032642C2066
:100780005461736B2049443D253032642C20546100
:10079000736B2052756E6E696E6720697320746882
:1007A00065205475726E657220433320466C6F75F8
:1007B000726F6D657465720D0A0D0A000D0A426F45
:1007C0006172642049443D253032642C20546173A9
:1007D0006B2049443D253032642C205461736B20DA
:1007E00052756E6E696E6720697320746865205358
:1007F0006561626972642047504354440D0A0D0AD2
:10080000000D0A426F6172642049443D2530326414
:100810002C205461736B2049443D253032642C20D8
:100820005461736B2052756E6E696E672069732018
:100830007468652053656162697264203337534977
:10084000204354440D0A0D0A000D0A426F61726480
:100850002049443D253032642C205461736B20497B
:10086000443D253032642C205461736B2052756EE8
:100870006E696E672069732074686520534D43204C
:10088000436F6D6D20537570706F72740D0A0D0A91
:10089000000D0A426F6172642049443D2530326484
:1008A0002C205461736B2049443D253032642C2048
:1008B0005461736B2052756E6E696E672069732088
:1008C000746865205061796C6F616420436F6D6D51
:1008D00020537570706F72740D0A0D0A00693D2502
:1008E000642C2074736B3D2564006F6E0000000063
:1008F000000000006F6666000000000000006175E7
:10090000746F72756E00000072756E00000000005A
:10091000000073746F700000000000007374617455
:100920007573000000006964000000000000000012
:10093000636D6400000000000000434F32006F66EA
:100940006172787369634F46415258534943004F6F
:100950004B004175746F52756E20697320257300CA
:100960004D4241524920434F322053656E736F729E
:1009700000506F7765722069732025732E205361B4
:100980006D706C696E672069732025732E20417528
:10099000746F72756E20697320257300506F7765D0
:1009A0007220646F776E0D004D4241524920434FD3
:1009B0003220666F7220504D2564000D0A0064736A
:1009C000006463006765746864006765746364004D
:1009D00072657365746C6F6767696E6700646174D4
:1009E0006574696D653D253032642530326425308B
:1009F000346425303264253032642530326400623C
:100A0000617564726174653D256C64006F75747006
:100A1000757465786563757465643D2563006175FB
:100A2000746F72756E3D2563006F757470757466B2
:100A30006F726D61743D2564006D696E636F6E64E5
:100A4000667265713D256400696E74657276616CCD
:100A50003D256400637573746F6D70756D706D6F97
:100A600064653D25630074787265616C74696D65B9
:100A70003D2563007273323332666F7263656F6E49
:100A80003D25630073746172740073746F7000703D
:100A9000756D706661737400533E000D0A0020206E
:100AA0000020093D2C3A0D0A003C53424534333EA8
:100AB0007965733C2F53424534333E000D0A616320
:100AC000717569726520534245203433004F6E00C2
:100AD0004F666600535543434553533A00464149D8
:100AE0004C45443A00205077723D002020536D70F1
:100AF0006C3D002020496E7472766C3D2530346464
:100B0000207365632053697A653D25303264207314
:100B10006D706C2F706B74204F66662D546D3D2583
:100B20006420466C7573682D546D3D256420536CAC
:100B3000703D257320446573743D307825303458FA
:100B4000002020496E7472766C3D25303464207329
:100B500065632053697A653D2530326420736D707A
:100B60006C2F706B74204F66662D546D3D2564208C
:100B7000466C7573682D546D3D256420536C703D33
:100B8000257320446573743D53484F52450020201F
:100B90004F787967656E3D0020204175746F7275DE
:100BA0006E3D00596573004E6F006F6E00000000CF
:100BB00000006F666600000000006175746F72755A
:100BC0006E0072756E000000000073746F7000009C
:100BD0000000706572696F64000073697A650000D7
:100BE0000000646573740000000073746174000099
:100BF00000006964000000000000636D64000000F4
:100C000000006379636C65000000666C75736800B2
:100C10000000435444006F66617278707A647369AF
:100C200063796C4F46415258505A44534943594C8A
:100C300000726573657465630072657365746C6FCB
:100C40006767696E6700676574006175746F7275B8
:100C50006E007374617274006F757470757465786A
:100C600065637574656474616700626175640043EF
:100C700054442056657273696F6E20616E64205310
:100C8000657269616C204E756D62657220697320B2
:100C90006E6F7420617661696C61626C652E0043D1
:100CA0006F6D6D616E64204661696C656400556EA0
:100CB0007265636F676E697A656420436F6D6D61FD
:100CC0006E6400436F6D6D616E642072656365696B
:100CD00076656420776173206E6F7420666F722072
:100CE00074686520475043544400526563656976D3
:100CF000656420616E20456D70747920436F6D6D61
:100D0000616E640020004E6F207374617274206104
:100D100064647265737320666F7220454550524F4C
:100D20004D00456E64696E67207461736B2E2E2EC4
:100D30002E0072756E0000000073746F700000006A
:100D4000636D6400000000696400000000007374BB
:100D50006174757300333753490072786369735255
:100D60005843495300556E7265636F676E697A65C3
:100D70006420436F6D6D616E6400596F75206D75F1
:100D800073742073746F702073616D706C696E671B
:100D9000206669727374004F4B00435444333753D9
:100DA000492E2053616D706C696E67206973202530
:100DB000730053544154555320434F4D4D414E44BD
:100DC00000435444333753492E204572726F7220CA
:100DD00072656164696E672073657269616C206E0B
:100DE000756D6265722E00435444333753492E208B
:100DF00053657269616C204E756D6265723D257335
:100E000000494420434F4D4D414E4400596F7520D9
:100E10006D7573742073746F702073616D706C697D
:100E20006E6720666972737400434D4420746F20AE
:100E300074686520435444004F4B0053544F502076
:100E4000434F4D4D414E44004F4B0052554E2043B1
:100E50004F4D4D414E440050617273696E6720439F
:100E60006F6D6D616E64203C25633E203C25733EB2
:100E700000636D64203D203C25733E3C25733E009D
:100E8000626164202E2E20636F64653D25640067D7
:100E90006F6F64206D657373616765005061727375
:100EA000696E6720636F6E736F6C653A203C2573C3
:100EB0003E004E6F207374617274206164647265C9
:100EC000737320666F7220454550524F4D00456E3A
:100ED00064696E67207461736B2E2E2E2E00506F26
:100EE00077657220646F776E2E2E2E004354443344
:100EF000375349204C6F6F7020666F7220504D251C
:100F000064000D0A006473006463006765746864BC
:100F10000072657365746C6F6767696E6700646102
:100F2000746574696D653D25303264253032642501
:100F30003034642530326425303264253032640028
:100F400062617564726174653D256C64006F7574CF
:100F500070757465786563757465643D25630061BB
:100F600075746F72756E3D2563006F75747075745E
:100F7000666F726D61743D2564006D696E636F6E9E
:100F800064667265713D25640073616D706C65699E
:100F90006E74657276616C3D256400637573746F61
:100FA0006D70756D706D6F64653D2563007478724A
:100FB00065616C74696D653D25630072733233320F
:100FC000666F7263656F6E3D256300737461727442
:100FD0000073746F7000533E000D0A002020002043
:100FE000093D2C3A0D0A004F6E004F6666005355BE
:100FF00043434553533A004641494C45443A002047
:101000005077723D002020536D706C3D00202049C8
:101010006E7472766C3D25303464207365632053A2
:10102000697A653D2530326420736D706C2F706B6A
:1010300074204F66662D543D256420536C703D2509
:101040007320446573742E3D307825303458002069
:1010500020496E7472766C3D25303464207365636C
:101060002053697A653D2530326420736D706C2F92
:10107000706B74204F66662D543D256420536C7050
:101080003D257320446573742E3D53484F524500EF
:101090006F6E0000000000006F6666000000000038
:1010A00072756E000000000073746F700000000025
:1010B000706572696F64000073697A6500000000F2
:1010C00064657374000000007374617400000000B4
:1010D0006964000000000000636D6400000000000F
:1010E0006379636C6500000033375349006F6672A3
:1010F00078707A64736963794F465258505A4453F2
:101100004943590072657365746563007265736560
:10111000746C6F6767696E670067657400617574EA
:101120006F72756E007374617274006F7574707590
:101130007465786563757465647461670062617570
:1011400064004354442056657273696F6E20616E6B
:10115000642053657269616C204E756D6265722002
:101160006973206E6F7420617661696C61626C6571
:101170002E0070756D7020696E7374616C6C65649F
:10118000203D2079657300506F77657220646F771A
:101190006E2E2E2E003337534920666F7220504D2D
:1011A00025640072756E0000000073746F7000009B
:1011B000006F6E00000000006F66660000000063B4
:1011C0006D64000000006964000000000073746139
:1011D0007475730041544D0072786F666369735281
:1011E000584F46434953004D6F64656D2069732025
:1011F0004F6666202D2D20506C65617365207475D7
:10120000726E206974206F6E2066697273742E008E
:10121000556E7265636F676E697A656420436F6DA2
:101220006D616E6400596F75206D757374207374F1
:101230006F702073616D706C696E67206669727380
:1012400074004F4B004D6F64656D206973204F66CD
:1012500066202D2D20506C65617365207475726E4B
:10126000206974206F6E2066697273742E004F4B74
:1012700000596F75206D7573742073746F702073CF
:10128000616D706C696E6720666972737400434D9E
:101290004420746F2073656E640054656C656479D6
:1012A0006E652041544D2D3838582E2053616D7095
:1012B0006C696E672069732025732E20506F7765E7
:1012C000722069732025732E0054656C6564796EF5
:1012D000652041544D2D3838580052554E20434F0B
:1012E0004D4D414E440050617273696E6720436FEB
:1012F0006D6D616E64203C25633E203C25733E008D
:10130000636D64203D203C25733E3C25733E0062A6
:101310006164202E2E20636F64653D256400676F35
:101320006F64206D657373616765005061727369E6
:101330006E6720636F6E736F6C653A203C25733E59
:10134000004E6F20737461727420616464726573FF
:101350007320666F7220454550524F4D00456E64B4
:10136000696E67207461736B2E2E2E2E00506F777E
:10137000657220646F776E2E2E2E00476F74207377
:101380006F6D657468696E670054656C6564796E2D
:10139000652041544D204C6F6F7020666F72205055
:1013A0004D25640073746174650000006F6E000069
:1013B000000000006F666600000000007374617238
:1013C0007400000073746F700000000063666700B3
:1013D0000000000063616C000000000074696D0093
:1013E00000000000776970000000000069640000E0
:1013F00000000000433300746F66737863616D779B
:1014000069544F46535843414D57490020090D0A2E
:10141000004E4E4E4E4E4E4E4E4F66664F6E205311
:101420004E3A30303030303030302066773A253028
:1014300032642E2530326420436F6D6D3A25303290
:10144000642E253032642043313A2E2E2E2E2E2E3D
:101450002E2E2E2E2E2E2E2E2E2043323A2E2E2E95
:101460002E2E2E2E2E2E2E2E2E2E2E2E2043333A84
:101470002E2E2E2E2E2E2E2E2E2E2E2E2E2E2E209A
:10148000503A256320543A256320573A25630025B6
:101490003032642F253032642F25303464202025EB
:1014A0003032643A253032643A2530326400534E8B
:1014B0003A25632563256325632563256325632515
:1014C000632066773A25642E25642C2043313A2523
:1014D000632043323A25632043333A256320433463
:1014E0003A25632043353A25632043363A25632065
:1014F000503A256320543A2563204C6F673A2563A0
:101500002C2053697A653A256420467265653A2530
:101510006420436F6D6D3A25642E2564004E6F2064
:10152000466C756F726F6D65746572200053616DE6
:10153000706C65733A256420506572696F643A2552
:1015400064204F6E2044656C61793A2564204331F4
:101550003A25632043323A25632043333A256320FA
:1015600043343A25632043353A25632043363A25F0
:101570006320503A256320543A25632047313A25A9
:10158000642047323A25642047333A2564204734A3
:101590003A25642047353A25642047363A256420A9
:1015A00047373A25642047383A2564204176672337
:1015B0003A2564205077723A2563256325632057C6
:1015C000697065733A256400556E7265636F676E66
:1015D000697A656420436F6D6D616E640054686163
:1015E0007420636F6D6D616E642069732063757222
:1015F00072656E746C79206E6F7420737570706F85
:10160000727465640053797374656D206973206921
:101610006E20616E20756E6B6E6F776E20737461D5
:10162000746500506F776572206973204F46462CB1
:101630002053616D706C696E67206973204F464658
:1016400000506F776572206973204F46462C2053F7
:10165000616D706C696E67206973204F4E00506F2A
:10166000776572206973204F4E2C2053616D706C2A
:10167000696E67206973204F464600506F77657228
:10168000206973204F4E2C2053616D706C696E671A
:10169000206973204F4E004333204461746120530E
:1016A000616D706C696E67206973204F4E202D2D1F
:1016B00020756E61626C6520746F2070726F636557
:1016C0007373206F7468657220636F6D6D616E64F3
:1016D0007300433320446174612053616D706C6901
:1016E0006E6720697320616C7265616479204F6652
:1016F0006600433320506F77657220697320616CF8
:101700007265616479204F4E00433320506F7765D6
:1017100072206973204F6666202D2D20506C656104
:101720007365207475726E206974206669727374B3
:1017300000496E76616C696420506172616D6574F8
:101740006572204C697374004F4B00474554005339
:1017500045540049440057495000474554005345FB
:10176000540054494D0043414C00474554005345F3
:1017700054004346470053544F5000535441525471
:10178000004F4646004F4E00535441544500434DD0
:101790004400556E7265636F676E697A65642043B5
:1017A0006F6D6D616E64005468617420636F6D6D60
:1017B000616E642069732063757272656E746C79F2
:1017C000206E6F7420737570706F7274656400534F
:1017D000797374656D20697320696E20616E207560
:1017E0006E6B6E6F776E20737461746500506F77E7
:1017F0006572206973204F46462C2053616D706CD2
:10180000696E67206973204F464600506F77657296
:10181000206973204F46462C2053616D706C696EB1
:1018200067206973204F4E00506F7765722069738F
:10183000204F4E2C2053616D706C696E6720697368
:10184000204F464600506F776572206973204F4ED7
:101850002C2053616D706C696E67206973204F4E48
:1018600000433320446174612053616D706C696E74
:1018700067206973204F4E202D2D20756E61626C9C
:101880006520746F2070726F63657373206F746866
:10189000657220636F6D6D616E6473004333204425
:1018A0006174612053616D706C696E67206973208B
:1018B000616C7265616479204F6666004333205025
:1018C0006F77657220697320616C7265616479203D
:1018D0004F4E00433320506F776572206973204F5D
:1018E0006666202D2D20506C6561736520747572BD
:1018F0006E20697420666972737400496E76616C3B
:10190000696420506172616D65746572204C697301
:1019100074004F4B0072657476616C203D20256425
:10192000004745540053455400494400574950006E
:10193000474554005345540054494D0043414C0021
:1019400047455400534554004346470053544F50B5
:10195000005354415254004F4646004F4E005354DA
:1019600041544520434F4D4D414E440050617273E8
:10197000696E6720436F6D6D616E64203C25633E28
:10198000203C25733E00636D64203D203C25733E62
:101990003C25733E00626164202E2E20636F6465D7
:1019A0003D256400676F6F64206D657373616765C3
:1019B0000050617273696E6720636F6E736F6C6540
:1019C0003A203C25733E004E6F2073746172742080
:1019D0006164647265737320666F7220454550526E
:1019E0004F4D00456E64696E67207461736B2E2ED7
:1019F0002E2E00476F7420736F6D657468696E6773
:101A0000004333204C6F6F7020666F7220504D255D
:101A1000640025202E3A2F090D0A0020090D0A0026
:101A20006F6E0000000000006F666600000000009E
:101A30006175746F72756E0072756E000000000043
:101A400073746F7000000000696400000000000003
:101A500073746174757300004333006F666172784C
:101A600069734F46415258495300556E7265636F12
:101A7000676E697A656420436F6D6D616E64004FB7
:101A80004B005475726E65722043333A20205361C7
:101A90006D706C696E672069732025733A20204150
:101AA00075746F72756E20697320257300636D64A1
:101AB000203D203C25733E3C25733E00626164203E
:101AC0002E2E20636F64653D256400676F6F642070
:101AD0006D6573736167650050617273696E67202D
:101AE000636F6E736F6C653A203C25733E004E6FDA
:101AF000207374617274206164647265737320660C
:101B00006F7220454550524F4D00456E64696E67B7
:101B1000207461736B2E2E2E2E00506F776572200D
:101B2000646F776E2E2E2E004333204F726967202C
:101B30004C6F6F7020666F7220504D256400696491
:101B400000454D50545900694900456D7074792025
:101B5000504D2073656E736F722E006F6E00000023
:101B600000000000006F66660000000000000061D9
:101B700075746F72756E00000072756E0000000063
:101B800000000073746F70000000000000696400C2
:101B900000000000000000737461747573000000A1
:101BA00000504F574552006F6661727869734F4617
:101BB0004152584953004175746F52756E206973D4
:101BC00020257300506F7765722069732025733A62
:101BD00020004175746F52756E2069732025730063
:101BE000506F77657220697320257300506F776599
:101BF00072206973202573002444454641554C5496
:101C000000244E455750524F47008F929F92AF92FB
:101C1000BF92CF92DF92EF92FF920F931F93DF93C9
:101C2000CF93CDB7DEB727970FB6F894DEBF0FBEC0
:101C3000CDBFFC0180818A8381818B8384819581E2
:101C40009F838E838E010E5F1F4FC8010E947567B0
:101C50008F3F09F000C153EF852E58E1952E48EAD9
:101C6000A42E49E0B42EC801F02E092F39E0C32E6E
:101C700031E0D32E80E060E040E024EF31E00E94CC
:101C80002A2E00D000D0EDB7FEB73196ADB7BEB763
:101C900012969C928E921197B382A2828B8184833A
:101CA00015820E9451F1EE81FF81EF5FFA4F2DB74F
:101CB0003EB72A5F3F4F0FB6F8943EBF0FBE2DBF11
:101CC00080818F3F21F48F2D902F0E946A63EB81DA
:101CD000F0E0EB56FE4580818F3F49F48F2D902F29
:101CE0000E94A663EB81F0E0EB56FE451082EE8188
:101CF000FF81EE5FFA4F80818F3F99F40E94233479
:101D0000EE81FF81ED5FFA4F208131814281538165
:101D1000261737074807590720F48F2D902F0E9468
:101D20002D618B81A82FB0E0FD01E756FE451081A3
:101D30001F3FB9F410939DA16FEF40E00E94A238BD
:101D400080E060E040E024EF31E00E942A2E109312
:101D50009EA181E060E040E020E030E00E942A2E79
:101D6000F8CFA357BE458C918F3F69F5EE81FF8177
:101D70008A8190E0E25EF94F8C9DD0018D9DB00D7F
:101D80009C9DB00D1124A759B2468D919C9111973D
:101D9000819391931082329613968C91139781932D
:101DA00015968D919D910D90BC91A02D808391836E
:101DB000A283B3838F2D902F0E947E66EB81F0E08B
:101DC000E357FE4510828B81E82FF0E0EF56FE4589
:101DD00090819F3F09F04ECF9983813029F400E034
:101DE00013E080E093E019C0823029F400E015E0B0
:101DF00080E095E012C0833011F010823BCF00E00C
:101E000017E080E097E009C0C801B60141E050E06A
:101E10000E94F7370F5F1F4F09C0E12C22E0F22E1E
:101E2000E80EF91E6E010894C11CD11C0E151F0589
:101E300058F3EE81FF8187E297E0DF019C011D925C
:101E400021503040E1F781E060E040E020E030E008
:101E50000E942A2EF8CF27960FB6F894DEBF0FBE49
:101E6000CDBFCF91DF911F910F91FF90EF90DF9049
:101E7000CF90BF90AF909F908F9008952F923F92F8
:101E80004F925F926F927F928F929F92AF92BF928A
:101E9000CF92DF92EF92FF920F931F93DF93CF9336
:101EA000CDB7DEB728970FB6F894DEBF0FBECDBF13
:101EB0006C0119828E010D5F1F4F86E0D8011D92C3
:101EC0008A95E9F7F60180818B8381818C838481F7
:101ED000958198878F83C8010E94F97C8F3F09F014
:101EE00065C2198280E060E042E020E030E00E94BC
:101EF0002A2E20E031E0EF81F885DF01A9011D9253
:101F000041505040E1F78F81988580509F4FDC0110
:101F1000A9011D9241505040E1F7580120E7422E9F
:101F2000512C612C712C99E0892E91E0992E83EF30
:101F3000282E88E1382E80E060E040E024EF31E098
:101F40000E942A2E8C81E82FF0E0E756FE45108192
:101F50001F3FB9F410939DA16FEF40E00E94A2389B
:101F600080E060E040E024EF31E00E942A2E1093F0
:101F70009EA181E060E040E020E030E00E942A2E57
:101F8000F8CF0E9423347B018C01EF81F885E75E56
:101F9000F64F80819181E951F940892B59F1E05E3A
:101FA000F64F20813181E052F9402115310511F1C0
:101FB000EE5DF64F8081E252F9408823D9F4E15E6C
:101FC000F64F8081EF51F9408F3FA1F4E55EF64F67
:101FD00080819181A281B3818E199F09A00BB10BE1
:101FE00040E050E0281739074A075B0718F0C501A1
:101FF0000E94B974EF81F885E15EF64F8081EF5160
:10200000F9408F3F09F042C0E55EF64F8081918133
:10201000A281B381E816F9060A071B07B8F10097F9
:10202000A105B10599F1C5010E943A76EF81F885C5
:10203000BF01655E764FDF01AF5FBA4FED5FFA4FCC
:102040002D913C9180819181DC012A9FC0012B9FC1
:10205000900D3A9F900D1124EA5EFB4F2081318153
:10206000820F931F7C0100E010E0DB012D913D9178
:102070004D915C911397E20EF31E041F151FED9214
:10208000FD920D931C93139736961082EF81F8857D
:10209000E95AFA4F10811F3F09F08BC08C81BE01B5
:1020A0006F5F7F4F0E94A131EF81F885E75AFA4FA9
:1020B00080819981813081F1913108F46DC0C50131
:1020C0000E941D6FEF81F885EE59FA4F808190E0F4
:1020D000EF55F04020813181E350F540821793079E
:1020E00008F459C0E55AFA4F4192519261927192A7
:1020F0008091E60381938B81819388E48083C5017D
:102100000E94C56B8F819885855A9A4FDC0128EF14
:102110001D922A95E9F72FC09131F0F1C5010E9477
:10212000236DEF81F885E65AF94F808190E0E755FD
:10213000F14020813181E350F5408217930758F137
:10214000ED5AF94F41925192619271928091E6035A
:1021500081938B81819389E48083C5010E94476BC1
:102160008F8198858D5A994FDC0120E231E01D92D4
:1021700021503040E1F7EF81F885E75EF64F80812E
:102180009181892B41F0C5010E940B75EF81F88583
:10219000E15EF64F10831982EF81F885E65AFA4F17
:1021A00080818F3F31F48981882319F0C5010E9415
:1021B000B270D60111968C91A82FB0E0FD01EF59B5
:1021C000F24680818F3F61F5EF81F885E05FF64F41
:1021D000AA0FBB1FAA0FBB1FAD57B84F8D919D9182
:1021E0000D90BC91A02D80839183A283B383C50100
:1021F00062E00E94FC7AD6011196EC911197F0E012
:10220000EE0FFF1FEE0FFF1FED57F84F10821182E8
:10221000128213821196EC91F0E0EF59F24610828F
:10222000EC81F0E0E357FE4580818F3F09F044C028
:102230002F8138852D58384F8B8190E0889DF00193
:10224000899DF00D989DF00D1124E759F24680818B
:102250009181F901819391939F0110822E5F3F4FED
:102260008B8190E0889DF001899DF00D989DF00D87
:102270001124E759F2468381D9018D939D018B8109
:1022800090E0889DF001899DF00D989DF00D11243E
:10229000E759F24685819681A781B085F90180834F
:1022A0009183A283B383C50161E00E94FC7AEC8133
:1022B000F0E0E357FE451082EC81F0E0EF56FE457A
:1022C00010811F3F09F037CE00D00F92ADB7BEB7D7
:1022D00012963C922E921197E2E2FDE01496FC9346
:1022E000EE9313970E9451F11A838C810F900F90F7
:1022F0000F900F90813029F400E013E080E093E02C
:1023000031C0823029F400E015E080E095E02AC079
:102310008330D1F000D00F92ADB7BEB712963C9289
:102320002E921197E6E0FDE01496FC93EE9313973E
:102330000E9451F1EC81F0E0EF56FE4510820F90C3
:102340000F900F900F90F7CD00E017E080E097E03E
:1023500009C0C801B60141E050E00E94F7370F5FA5
:102360001F4F0AC0E12CF2E0FF2EE80EF91EE2E05A
:10237000CE2ED12CCC0EDD1E0E151F0550F38C81F8
:1023800060E040E00E94A238EF81F88580EA9FE09B
:10239000DF019C011D9221503040E1F781E060E0B7
:1023A00040E020E030E00E942A2EF8CF28960FB6B9
:1023B000F894DEBF0FBECDBFCF91DF911F910F917B
:1023C000FF90EF90DF90CF90BF90AF909F908F9055
:1023D0007F906F905F904F903F902F9008952F9235
:1023E0003F924F925F926F927F928F929F92AF92A5
:1023F000BF92CF92DF92EF92FF920F931F93DF93E2
:10240000CF93CDB7DEB727970FB6F894DEBF0FBED8
:10241000CDBF6C01DC018C918A8311968C91119750
:102420008B8314968D919C9115979F838E838E013B
:102430000E5F1F4FC8010E94D58A8F3F09F06BC104
:1024400083EFA82E88E1B82E4801B9E02B2EB1E029
:102450003B2EAEEC4A2EAEE05A2EF2EB6F2EFEE093
:102460007F2E80E060E040E024EF31E00E942A2EE1
:1024700000D000D0EDB7FEB73196ADB7BEB712961B
:10248000BC92AE9211972CEE3EE0338322838B8177
:10249000848315820E9451F1EE81FF81EC5EFA4F38
:1024A0008DB79EB706960FB6F8949EBF0FBE8DBF30
:1024B00080818F3F29F50E9423347B018C01EE81BE
:1024C000FF81EB5EFA4F80819181A281B381E81692
:1024D000F9060A071B07A0F0C4010E944189EE819A
:1024E000FF81E050FB4F80819181A281B3818E0DED
:1024F0009F1DA01FB11F759680839183A283B38314
:10250000EB81F0E0EB56FE4580818F3FA1F400D0D7
:102510000F92ADB7BEB71296BC92AE921197EEED88
:10252000FEE01496FC93EE9313970E9451F10F90E6
:102530000F900F900F908B81E82FF0E0E756FE454B
:1025400010811F3FB9F410939DA16FEF40E00E94EE
:10255000A23880E060E040E024EF31E00E942A2EC3
:1025600010939EA181E060E040E020E030E00E9416
:102570002A2EF8CFD60111968C91A82FB0E0FD013C
:10258000EF59F24680818F3F11F5AA0FBB1FAA0FAA
:10259000BB1FAD57B84F4D915D916D917C91C401BA
:1025A0000E94C182D6011196EC911197F0E0EE0FD6
:1025B000FF1FEE0FFF1FED57F84F1082118212829E
:1025C00013821196EC91F0E0EF59F2461082EB8104
:1025D000F0E0E357FE4580818F3F61F5EE81FF819A
:1025E0008A8190E0E156FA4F829DD001839DB00D23
:1025F000929DB00D1124A759B2468D919C911197CF
:10260000819391931082329613968C9113978193B4
:1026100015968D919D910D90BC91A02D80839183F5
:10262000A283B383C4010E94D487EB81F0E0E35717
:10263000FE451082EB81F0E0EF56FE4510811F3F12
:1026400009F00FCF00D00F92EDB7FEB7B282A18292
:10265000548243820E9451F119838B810F900F9015
:102660000F900F90813029F400E013E080E093E0B8
:102670002FC0823029F400E015E080E095E028C00A
:102680008330C1F000D00F92ADB7BEB71296BC92A6
:10269000AE92119714967C926E9213970E9451F10C
:1026A000EB81F0E0EF56FE4510820F900F900F90F7
:1026B0000F90D7CE00E017E080E097E009C0C80196
:1026C000B60141E050E00E94F7370F5F1F4F09C08D
:1026D000E12C62E0F62EE80EF91E6E010894C11C92
:1026E000D11C0E151F0558F38B8160E040E00E945D
:1026F000A238EE81FF818CEB96E0DF019C011D92F8
:1027000021503040E1F781E060E040E020E030E03F
:102710000E942A2EF8CF27960FB6F894DEBF0FBE80
:10272000CDBFCF91DF911F910F91FF90EF90DF9080
:10273000CF90BF90AF909F908F907F906F905F9061
:102740004F903F902F9008952F923F924F925F921B
:102750006F927F928F929F92AF92BF92CF92DF92B1
:10276000EF92FF920F931F93DF93CF93CDB7DEB716
:1027700028970FB6F894DEBF0FBECDBFFC011982BB
:102780008E010D5F1F4F86E0D8011D928A95E9F7F3
:1027900080818B8381818C838481958198878F83CD
:1027A000C8010E9461998F3F09F0B1C1198280E090
:1027B00060E042E020E030E00E942A2E20E031E09C
:1027C000EF81F885DF01C9011D920197E9F78F813B
:1027D000988580509F4FDC01C9011D920197E9F750
:1027E00083EF682E88E1782E68011E010894211C71
:1027F000311C11E2812E912CA12CB12CB9E04B2E71
:10280000B1E05B2E80E060E040E024EF31E00E9428
:102810002A2E00D000D0EDB7FEB73196ADB7BEB7C7
:1028200012967C926E92119725E931E133832283CF
:102830008C81848315820E9451F1EC81F0E0EB568B
:10284000FE458DB79EB706960FB6F8949EBF0FBE95
:102850008DBF80818F3FA1F400D00F92ADB7BEB77E
:1028600012967C926E921197E7E8F1E11496FC9330
:10287000EE9313970E9451F10F900F900F900F90CD
:102880008C81E82FF0E0E756FE4510811F3FB9F438
:1028900010939DA16FEF40E00E94A23880E060E0BD
:1028A00040E024EF31E00E942A2E10939EA181E0A7
:1028B00060E040E020E030E00E942A2EF8CFEF8177
:1028C000F885E650F84F8081EA5FF7408823C9F029
:1028D000EA50F84FE080F180028113810E94233496
:1028E000E616F7060807190760F4C6010E9423944C
:1028F000EF81F885EA50F84F1192119211921192DE
:102900001082EF81F885EA5AFA4F10811F3F09F0D3
:102910007DC08C81B1010E94A131EF81F885E65A1A
:10292000FA4F2081EA55F54030E0285F3F4F89811A
:1029300090E0281739070CF051C0E85AFA4F80810F
:10294000882309F04BC0C6010E945F8EEF81F88595
:10295000ED59FA4F808190E0E156F04020813181BD
:10296000E250F54082179307C0F1E45AFA4F819282
:102970009192A192B1928091E60381938B81819390
:1029800088E48083C6010E94C18D8F819885845A16
:102990009A4FDC0128EF1D922A95E9F7EF81F8851F
:1029A000EC50F84F80819181892BB9F0C6010E94CB
:1029B00086930E942334EF81F885EC50F84F2191E3
:1029C000319140E050E0260F371F481F591F2083E8
:1029D000318342835383349610831982EF81F885C3
:1029E000E85AFA4F8081E855F5408F3F79F4298104
:1029F00030E0E65AFA4F808190E00996880F991FDF
:102A0000281739071CF0C6010E94B58FEC81F0E051
:102A1000E357FE4580818F3F61F5EF81F8858B811B
:102A200090E0EC5AF94F849DD001859DB00D949DA6
:102A3000B00D1124A759B2468D919C9111978193A5
:102A400091931082329613968C91139781931596D9
:102A50008D919D910D90BC91A02D80839183A28337
:102A6000B383C6010E946A98EC81F0E0E357FE450B
:102A700010828C81E82FF0E0EF56FE4590819F3F59
:102A800009F0C0CE9A83813029F400E013E080E0A1
:102A900093E019C0823029F400E015E080E095E071
:102AA00012C0833011F01082ADCE00E017E080E05C
:102AB00097E009C0C801B60141E050E00E94F73735
:102AC0000F5F1F4F0AC0E12CF2E0FF2EE80EF91E47
:102AD000E2E0CE2ED12CCC0EDD1E0E151F0550F3DC
:102AE0008C8160E040E00E94A238EF81F88580EAA6
:102AF0009FE0DF019C011D9221503040E1F781E011
:102B000060E040E020E030E00E942A2EF8CF2896D6
:102B10000FB6F894DEBF0FBECDBFCF91DF911F91EE
:102B20000F91FF90EF90DF90CF90BF90AF909F906C
:102B30008F907F906F905F904F903F902F9008956F
:102B40002F923F924F925F926F927F928F929F92BD
:102B5000AF92BF92CF92DF92EF92FF920F931F93AB
:102B6000DF93CF93CDB7DEB727970FB6F894DEBFCC
:102B70000FBECDBF6C01DC018C918A8311968C91C4
:102B800011978B8314968D919C9115979F838E83BB
:102B90008E010E5F1F4FC8010E9401A78F3F09F0F1
:102BA0007AC1A3EFAA2EA8E1BA2E4801FDE62F2E86
:102BB000F3E13F2EEDE54E2EE3E15E2E71E4672E4C
:102BC00073E1772E80E060E040E024EF31E00E9486
:102BD0002A2E00D000D0EDB7FEB73196ADB7BEB704
:102BE0001296BC92AE92119729E833E13383228387
:102BF0008B81848315820E9451F1EE81FF81EC5E0E
:102C0000FA4F8DB79EB706960FB6F8949EBF0FBECB
:102C10008DBF80818F3F29F50E9423347B018C0179
:102C2000EE81FF81EB5EFA4F80819181A281B381B9
:102C3000E816F9060A071B07A0F0C4010E94B8A510
:102C4000EE81FF81E050FB4F80819181A281B381B1
:102C50008E0D9F1DA01FB11F759680839183A28347
:102C6000B383D60111968C91A82FB0E0FD01EF59E6
:102C7000F24680818F3F11F5AA0FBB1FAA0FBB1F21
:102C8000AD57B84F4D915D916D917C91C4010E94FB
:102C9000B79FD6011196EC911197F0E0EE0FFF1F50
:102CA000EE0FFF1FED57F84F108211821282138230
:102CB0001196EC91F0E0EF59F2461082EB81F0E0D2
:102CC000E357FE4580818F3FF1F500D00F92EDB7BD
:102CD000FEB7B282A1822BE733E1348323830E94C3
:102CE00051F1EE81FF818A8190E0EE51FA4F29E0A7
:102CF00031E0829FD001839FB00D929FB00D1124CF
:102D0000A759B2468D919C9111978193919310820E
:102D1000329613968C911397819315968D919D9170
:102D20000D90BC91A02D80839183A283B3830F90DB
:102D30000F900F900F90C4010E944BA4EB81F0E024
:102D4000E357FE451082EB81F0E0EB56FE458081B3
:102D50008F3F91F400D00F92ADB7BEB71296BC92E0
:102D6000AE92119714963C922E9213970E9451F1B5
:102D70000F900F900F900F908B81A82FB0E0FD0166
:102D8000E756FE4510811F3FB9F410939DA16FEFE8
:102D900040E00E94A23880E060E040E024EF31E0B3
:102DA0000E942A2E10939EA181E060E040E020E086
:102DB00030E00E942A2EF8CFAF56BE451C911F3F2F
:102DC00009F000CF00D00F92EDB7FEB7B282A1821A
:102DD000548243820E9451F119838B810F900F908E
:102DE0000F900F90813029F400E013E080E093E031
:102DF0002FC0823029F400E015E080E095E028C083
:102E00008330C1F000D00F92ADB7BEB71296BC921E
:102E1000AE92119714967C926E9213970E9451F184
:102E2000EB81F0E0EF56FE4510820F900F900F906F
:102E30000F90C8CE00E017E080E097E009C0C8011D
:102E4000B60141E050E00E94F7370F5F1F4F09C005
:102E5000E12C42E0F42EE80EF91E6E010894C11C2C
:102E6000D11C0E151F0558F38B8160E040E00E94D5
:102E7000A238EE81FF818BEE96E0DF019C011D926E
:102E800021503040E1F781E060E040E020E030E0B8
:102E90000E942A2EF8CF27960FB6F894DEBF0FBEF9
:102EA000CDBFCF91DF911F910F91FF90EF90DF90F9
:102EB000CF90BF90AF909F908F907F906F905F90DA
:102EC0004F903F902F9008952F923F924F925F9294
:102ED0006F927F928F929F92AF92BF92CF92DF922A
:102EE000EF92FF920F931F93DF93CF93CDB7DEB78F
:102EF00027970FB6F894DEBF0FBECDBF7C01DC0173
:102F00008C918A8311968C9111978B8314968D9155
:102F10009C9115979F838E838E010E5F1F4FC80172
:102F20000E94C0C3CC24F3EFAF2EF8E1BF2ED02E09
:102F3000012FE3EF2E2EE9E13E2E79E0472E71E0DE
:102F4000572E63EE662E69E1762E57EC852E59E1F9
:102F5000952E80E060E040E024EF31E00E942A2ED0
:102F600000D000D0EDB7FEB73196ADB7BEB7129620
:102F7000BC92AE92119721E03AE1338322838B8198
:102F8000848315820E9451F1EE81FF81EC5FFA4F3C
:102F90008DB79EB706960FB6F8949EBF0FBE8DBF35
:102FA0008081E450F5408F3F29F48D2D902F0E94B1
:102FB00013B10EC0EB5FFA4F80818F3F49F4C39489
:102FC00093E09C1528F48D2D902F0E9404C3CC24EF
:102FD000D70111968C91A82FB0E0FD01EF59F24670
:102FE00080818F3F19F5AA0FBB1FAA0FBB1FAD57DA
:102FF000B84F4D915D916D917C918D2D902F0E94D8
:1030000080B9D7011196EC911197F0E0EE0FFF1FF8
:10301000EE0FFF1FED57F84F1082118212821382BC
:103020001196EC91F0E0EF59F2461082EB81F0E05E
:10303000E357FE4580818F3FD9F500D00F92EDB761
:10304000FEB7B282A182348223820E9451F1EE81C6
:10305000FF818A8190E0E35AF84F849DD001859DDD
:10306000B00D949DB00D1124A759B2468D919C913D
:103070001197819391931082329613968C911397A6
:10308000819315968D919D910D90BC91A02D80837B
:103090009183A283B3830F900F900F900F908D2D8B
:1030A000902F0E9497C1EB81F0E0E357FE4510821C
:1030B000EB81F0E0EF56FE4510811F3F09F049CF4C
:1030C00000D00F92ADB7BEB71296BC92AE921197D8
:1030D00014967C926E9213970E9451F119838B8102
:1030E0000F900F900F900F90813029F400E013E0C3
:1030F00080E093E02BC0823029F400E015E080E00E
:1031000095E024C08330A1F000D00F92EDB7FEB758
:10311000B282A182948283820E9451F1EB81F0E01D
:10312000EF56FE4510820F900F900F900F9011CF29
:1031300000E017E080E097E009C0C801B60141E077
:1031400050E00E94F7370F5F1F4F09C0E12C22E0CB
:10315000F22EE80EF91E6E010894C11CD11C0E154A
:103160001F0558F3EE81FF8180EA9FE0DF019C019B
:103170001D9221503040E1F781E060E040E020E026
:1031800030E00E942A2EF8CF2F923F924F925F920A
:103190006F927F928F929F92BF92CF92DF92EF9227
:1031A000FF920F931F93DF93CF93CDB7DEB727978F
:1031B0000FB6F894DEBF0FBECDBF8C01DC018C9141
:1031C0008A8311968C9111978B8314968D919C9183
:1031D00015979F838E8372E0E72EF12CEC0EFD1E77
:1031E000C7010E943DD08F3F09F088C163EFC62E12
:1031F00068E1D62EC701BE2CE92E5AE1252E5BE1EF
:10320000352E49E0442E41E0542E3AE0632E3BE156
:10321000732E2EEE822E2AE1922E80E060E040E0B6
:1032200024EF31E00E942A2E00D000D0EDB7FEB787
:103230003196ADB7BEB71296DC92CE92119728E2C6
:103240003BE1338322838B81848315820E9451F179
:10325000EE81FF81EC5FFA4F8DB79EB706960FB6F1
:10326000F8949EBF0FBE8DBF80818F3F21F48B2DC0
:103270009E2D0E94AFCCEB81F0E0EF59F2468081A9
:103280008F3F11F5D8011196EC91F0E0EE0FFF1F82
:10329000EE0FFF1FED57F84F40815181628173811E
:1032A0008B2D9E2D0E94D4C7AB81B0E0FD01EE0FA7
:1032B000FF1FEE0FFF1FED57F84F10821182128291
:1032C0001382AF59B2461C92EB81F0E0EB56FE45FB
:1032D00080818F3F71F400D00F92EDB7FEB7D2829C
:1032E000C182348223820E9451F10F900F900F907F
:1032F0000F908B81A82FB0E0FD01E756FE45E081DD
:10330000EF3F09F05CC0E0939DA140E051EE60E02A
:1033100070E026E000E0EE240E94EE2F80E060E006
:103320004FE020E030E00E942A2E9B81923079F01D
:103330009330C1F09130C1F4809107018460809393
:103340000701809108018460809308010DC080917D
:103350000101806480930101809102018064809367
:10336000020102C0829A8A9A892F6FEF40E00E9480
:10337000A23880E060E040E024EF31E00E942A2E95
:103380008B81823051F0833071F0813069F480910B
:1033900008018B7F8093080107C0809102018F7B19
:1033A0008093020101C08A988FEF80939EA181E0F3
:1033B00060E040E020E030E00E942A2EF8CFA357E2
:1033C000BE458C918F3F69F5EE81FF818A8190E047
:1033D000E45FF84F849DD001859DB00D949DB00DA4
:1033E0001124A759B2468D919C9111978193919385
:1033F0001082329613968C911397819315968D9126
:103400009D910D90BC91A02D80839183A283B38365
:103410008B2D9E2D0E9442CBEB81F0E0E357FE45C1
:103420001082EB81F0E0EF56FE45F080FFEFFF16D3
:1034300009F0F3CE00D00F92ADB7BEB71296DC9272
:10344000CE92119714967C926E9213970E9451F12E
:10345000F9828B810F900F900F900F90813029F49B
:1034600000E013E080E093E02BC0823029F400E01C
:1034700015E080E095E024C08330A1F000D00F92E9
:10348000EDB7FEB7D282C182948283820E9451F14D
:10349000EB81F0E0EF56FE4510820F900F900F90F9
:1034A0000F90BBCE00E017E080E097E009C0C801B4
:1034B000B60141E050E00E94F7370F5F1F4F09C08F
:1034C000E12CF2E0FF2EE80EF91E6E010894C11CFB
:1034D000D11C0E151F0558F3EE81FF8180EA9FE095
:1034E000DF019C011D9221503040E1F781E060E056
:1034F00040E020E030E00E942A2EF8CF27960FB659
:10350000F894DEBF0FBECDBFCF91DF911F910F9119
:10351000FF90EF90DF90CF90BF909F908F907F9023
:103520006F905F904F903F902F900895CF92DF92D1
:10353000EF92FF920F931F93DF93CF93CDB7DEB738
:1035400027970FB6F894DEBF0FBECDBFFC01808178
:103550008A8381818B83848195819F838E838E0171
:103560000E5F1F4FC8010E9415D38F3F09F0A8C0FE
:1035700039E0C32E31E0D32EC801F02E092F80E0B0
:1035800060E045E020E030E00E942A2E8B81A82FE9
:10359000B0E0FD01E756FE4510811F3FB9F41093DE
:1035A0009DA16FEF40E00E94A23880E060E040E023
:1035B00024EF31E00E942A2E10939EA181E060E06A
:1035C00040E020E030E00E942A2EF8CFA357BE450D
:1035D0008C918F3F69F5EE81FF818A8190E0EC5EEE
:1035E000FE4F8C9DD0018D9DB00D9C9DB00D112482
:1035F000A759B2468D919C91119781939193108216
:10360000329613968C911397819315968D919D9177
:103610000D90BC91A02D80839183A283B3838F2DC5
:10362000902F0E9425D2EB81F0E0E357FE451082F7
:103630008B81E82FF0E0EF56FE4590819F3F09F027
:103640009ECF9983813029F400E013E080E093E07D
:1036500019C0823029F400E015E080E095E012C046
:10366000833011F010828BCF00E017E080E097E00C
:1036700009C0C801B60141E050E00E94F7370F5F72
:103680001F4F09C0E12C22E0F22EE80EF91E6E0158
:103690000894C11CD11C0E151F0558F3EE81FF8143
:1036A00082E291E0DF019C011D9221503040E1F760
:1036B00081E060E040E020E030E00E942A2EF8CF78
:1036C00027960FB6F894DEBF0FBECDBFCF91DF9126
:1036D0001F910F91FF90EF90DF90CF9008951124EC
:1036E0001FBECFEFD1E2DEBFCDBF00E00CBF112483
:1036F00080EC8093010180E8809374001092750043
:1037000088E10FB6F89480936000109260000FBEBD
:1037100015E0A0E0B2E0E2E7F9EE01E00BBF02C085
:1037200007900D92AC37B107D9F719E1ACE7B5E0D6
:1037300001C01D92A535B107E1F70E94AF1B0C94A3
:10374000B7F40C9400000E94745DFC01009719F01E
:1037500080E090E019958FEF0E94A42A08958F923F
:103760009F92AF92BF92CF92DF92EF92FF920F9310
:103770001F93DF93CF930F92CDB7DEB70E94E8601F
:103780000E945B240F920F9281E090E0EDB7FEB7AC
:103790009283818383EA9BE160E070E04BE756E02F
:1037A00020E008EE13E0ECE7EE2EE5E0FE2EA12C83
:1037B00031E0B32EC12CD12C882499240E94972C5F
:1037C0000F900F9080E060E072E0AE014F5F5F4FBE
:1037D0000E941F2C0E94CB2380E090E00F90CF919D
:1037E000DF911F910F91FF90EF90DF90CF90BF90EE
:1037F000AF909F908F9008950F920F93CF93DF9388
:103800000FB700680F9300917D180C7F00937D180F
:103810000091C00004FB56F4C0916D18D0916E1851
:10382000219621F0C0936D18D0936E1803FB56F4C7
:10383000C0916F18D0917018219621F0C0936F1825
:10384000D0937018C0917318D0E80091C600099306
:10385000C0937318009174180C1771F403950093BA
:103860007418C0917118D0917218219621F0C093EC
:103870007118D09372180AC0C0917718D091781837
:10388000219621F0C0937718D0937818C0917B18B7
:10389000D0917C180D81002359F40981002341F057
:1038A0000F910F770FBFDF91CF910F910F90189568
:1038B00000917818002321F400917718003184F3E7
:1038C0001F922F923F924F925F926F927F928F92B0
:1038D0009F92AF92BF92CF92DF92EF92FF921F938F
:1038E0002F933F934F935F936F937F938F939F9308
:1038F000AF93BF93EF93FF930BB70F930CB70F9357
:1039000011240091DD11002341F4E091DE11F091CA
:10391000DF111DB711931EB7119303950093DD11AD
:103920007894CE0161E077270E94DB250E94F8237E
:103930000F910CBF0F910BBFFF91EF91BF91AF9112
:103940009F918F917F916F915F914F913F912F91B7
:103950001F91FF90EF90DF90CF90BF90AF909F901E
:103960008F907F906F905F904F903F902F901F901F
:103970000F910F770FBFDF91CF910F910F90189597
:103980000F920F93CF93DF930FB700680F93C091FF
:103990008018C15010F1C0938018C0917618D4E8F7
:1039A00009910093C600C0937618C0917E18D091FB
:1039B0007F180D81002359F40981002341F00F91F4
:1039C0000F770FBFDF91CF910F910F901895009156
:1039D0008018003FA0F70C94601C0091C1000F7D7F
:1039E0000093C1000C94D51C0F920F93CF93DF93DB
:1039F0000FB700680F93009191180C7F00939118F6
:103A00000091C80004FB56F4C0918118D09182182F
:103A1000219621F0C0938118D093821803FB56F4AD
:103A2000C0918318D0918418219621F0C0938318F7
:103A3000D0938418C0918718D1E80091CE000993E3
:103A4000C0938718009188180C1771F403950093A0
:103A50008818C0918518D0918618219621F0C093BE
:103A60008518D09386180AC0C0918B18D0918C18F5
:103A7000219621F0C0938B18D0938C18C0918F1889
:103A8000D09190180D81002359F40981002341F051
:103A90000F910F770FBFDF91CF910F910F90189576
:103AA00000918C18002321F400918B18003184F3CD
:103AB0000C94601C0F920F93CF93DF930FB70068A5
:103AC0000F93C0919418C15010F1C0939418C091F5
:103AD0008A18D5E809910093CE00C0938A18C09146
:103AE0009218D09193180D81002359F40981002375
:103AF00041F00F910F770FBFDF91CF910F910F9092
:103B0000189500919418003FA0F70C94601C009148
:103B1000C9000F7D0093C9000C946F1D0F920F9385
:103B2000CF93DF930FB700680F930091A5180C7F18
:103B30000093A5180091D00004FB56F4C09195188D
:103B4000D0919618219621F0C0939518D09396188D
:103B500003FB56F4C0919718D0919818219621F044
:103B6000C0939718D0939818C0919B18D2E80091F1
:103B7000D6000993C0939B1800919C180C1771F400
:103B8000039500939C18C0919918D0919A1821968A
:103B900021F0C0939918D0939A180AC0C0919F1829
:103BA000D091A018219621F0C0939F18D093A0180F
:103BB000C091A318D091A4180D81002359F4098154
:103BC000002341F00F910F770FBFDF91CF910F913D
:103BD0000F9018950091A018002321F400919F18D0
:103BE000003184F30C94601C0F920F93CF93DF93FA
:103BF0000FB700680F93C091A818C15010F1C0937F
:103C0000A818C0919E18D6E809910093D600C093D9
:103C10009E18C091A618D091A7180D81002359F4C1
:103C20000981002341F00F910F770FBFDF91CF91F2
:103C30000F910F9018950091A818003FA0F70C94D1
:103C4000601C0091D1000F7D0093D1000C94091EDF
:103C50000F920F93CF93DF930FB700680F930091EC
:103C6000B9180C7F0093B9180091300104FB56F489
:103C7000C091A918D091AA18219621F0C093A91833
:103C8000D093AA1803FB56F4C091AB18D091AC188E
:103C9000219621F0C093AB18D093AC18C091AF1807
:103CA000D3E8009136010993C093AF180091B01882
:103CB0000C1771F403950093B018C091AD18D09112
:103CC000AE18219621F0C093AD18D093AE180AC05B
:103CD000C091B318D091B418219621F0C093B318B5
:103CE000D093B418C091B718D091B8180D810023A3
:103CF00059F40981002341F00F910F770FBFDF9135
:103D0000CF910F910F9018950091B418002321F4D2
:103D10000091B318003184F30C94601C0F920F9340
:103D2000CF93DF930FB700680F93C091BC18C150B9
:103D300010F1C093BC18C091B218D7E80991009354
:103D40003601C093B218C091BA18D091BB180D813A
:103D5000002359F40981002341F00F910F770FBF21
:103D6000DF91CF910F910F9018950091BC18003FF3
:103D7000A0F70C94601C009131010F7D009331017C
:103D80000C94A31ECF93DF93FC01DB01EA01809129
:103D9000DD11882311F081E105C0808181508430DC
:103DA00020F081E0888330E010C04FB7F894CF0155
:103DB0000E96FC0102C02D9331963E2F381B2081B8
:103DC0002223C9F71C924FBF1882832FDF91CF9116
:103DD0000895CF93DF939C01DB01EA018091DD110F
:103DE000882311F082E115C0F9018081815084306F
:103DF00010F081E00EC04FB7F894FB0101C031967E
:103E00009E2F9A1B80818823D1F7903120F04FBFDD
:103E10008BE088830BC0F9013E9602C08193119616
:103E20008C918823D9F710824FBF1882DF91CF91F0
:103E300008958091BA10813039F48091DD118F3F5F
:103E400019F08F5F8093DD1108958091BA10813051
:103E500071F49FB7F8948091DD11882339F4809133
:103E6000B9108F3F19F08F5F8093B9109FBF0895ED
:103E70008EE191E008950F931F93CF93DF938C0110
:103E8000DC011596EC91F0E0EE5DFD4F8081C82FCE
:103E9000D0E0F801EC0FFD1FE681F0E0EE5DFD4F94
:103EA000582F550F550F550F8081580FE52FF0E013
:103EB000EE0FFF1FE751F84EA081B18159961C9279
:103EC0001E92589757967C936E93569740955A96A4
:103ED0008C915A9784235A968C935A975B962C937D
:103EE0005B9783FD11C08091D21190969C91909721
:103EF000892B8093D211FE01ED52FE4E80815F9698
:103F00009C915F97892B80835E968C915E97F801D8
:103F1000E80FF11D5F968C915F97809596818923BC
:103F20008683882341F490969C9190979095F80110
:103F300085818923858354962D913C915597211530
:103F4000310539F15E968C915E9790964C919097E1
:103F50005F969C915F97F901C081D181682F70E0D5
:103F60009095409510C0FE01E60FF71F86818923CA
:103F70008683882319F48D8184238D832E5F3F4FA0
:103F8000F901C081D181209771F753961C930E934C
:103F90005297852FDF91CF911F910F910895CF9365
:103FA000DF93AC01A091DE11B091DF1153969C9389
:103FB0008E9352975E96EC915E97F0E05F969C919F
:103FC0005F979A012E0F3F1FE9018E81892B8E8307
:103FD00090962C91DA0115968C911597822B159657
:103FE0008C93ED52FE4E9095808198239083992377
:103FF00031F420958091D21182238093D211DF91E8
:10400000CF910895CF93DF93FC01C091DE11D09141
:10401000DF111B8A1A8A9D8B8C8BA081B1819C0138
:1040200013C0AD014E0F511DFA018681892B868385
:1040300015968C91159798A1892B15968C932E5FC8
:104040003F4FF901A081B181EE8D9F8D109749F707
:10405000F0E0ED52FE4E892F809590818923808378
:10406000882339F498A190958091D2118923809367
:10407000D211DF91CF910895CF93DF93DC01EB0153
:104080005E968C915E97FB01E80FF11D5F968C9117
:104090005F978095968189238683882331F4909653
:1040A0009C9190958D8189238D83DF91CF91089587
:1040B000CF93DF93FC01DB01868D20A1978DCD91FD
:1040C000DC911197482F50E0909520950FC0FE018C
:1040D000E40FF51F868189238683882319F48D8157
:1040E00082238D831296CD91DC911197209779F7D9
:1040F000DF91CF910895FC011582369680E01192F0
:104100008F5F8830E1F70895FC0103C01192615080
:10411000704061157105D1F70895DC01FB0104C001
:1041200081918D934150504041155105C9F7089533
:10413000582FDB01282F392FF90102C091931196D6
:104140008E2F851B9C919923C9F710820895582FB3
:10415000282F392FF90101C031969E2F951B8081A0
:104160008823D1F7892F08959F92AF92BF92CF9263
:10417000DF92EF92FF920F931F93CF93DF93982ECE
:10418000EFB7F894C091CC11D091CD11209709F4DC
:1041900082C08E859F859093CD118093CC11EFBF07
:1041A000798368839C8E1A8E1B8E198E188EDB8203
:1041B000CA82EE82FF82088719875D834C83BB86A3
:1041C000AA863D872C87292D2695269526952E8F04
:1041D000492D47704D8F81E090E0BC0102C0660F11
:1041E000771F2A95E2F768A302C0880F991F4A95A6
:1041F000E2F78F8F1B8A1A8A1D8A1C8A1F8A1E8AE1
:1042000019A21AA21BA21CA219A61AA61BA61CA6BA
:104210001DA21EA21FA218A61EA61DA61FA618AA92
:1042200019AA1AAA8FE38BAB1CAACE010E94F32E07
:10423000CE010E94022F2FB7F894E92DF0E0EE0F87
:10424000FF1FE751F84ED183C083E091C110F09178
:10425000C210FF87EE87198A188A309711F0D18B28
:10426000C08BD093C210C093C1108091D21198A17D
:10427000892B8093D211EE8DF0E0ED52FE4E8081BD
:104280009F8D892B80838091CF118F5F8093CF1179
:104290002FBF80E002C0EFBF82E4DF91CF911F917A
:1042A0000F91FF90EF90DF90CF90BF90AF909F90D5
:1042B0000895CF92DF92FF920F931F93DF93CF93D6
:1042C000CDB7DEB728970FB6F894DEBF0FBECDBFCF
:1042D00009EE17E1FF246E010894C11CD11C8F2D3B
:1042E000B6010E94362A8823C1F4D801ED91FC91D1
:1042F000309799F0E130F10581F084819581268134
:104300003781820F931F96A785A78D819E81AF81EC
:10431000B88587A790ABA1ABB2ABF3940E5F1F4FEC
:10432000B0E4FB16E1F628960FB6F894DEBF0FBE98
:10433000CDBFCF91DF911F910F91FF90DF90CF9074
:1043400008952FB7F8948091BB109091BC10A09164
:10435000BD10B091BE100196A11DB11D8093BB1080
:104360009093BC10A093BD10B093BE102FBF0E94BD
:10437000FC2EE7CF1F931FB7F8948091DD1188239F
:1043800009F04CC08091B910882309F047C0E09132
:10439000D211F0E0EE5DFD4F8081E82FF0E0ED52AC
:1043A000FE4EE081F0E0EE5DFD4F982F990F990FE2
:1043B000990F8081980F9093BF108091C01098172B
:1043C00069F1E92FF0E0EE0FFF1FE751F84E019081
:1043D000F081E02DF093D111E093D01181A192A151
:1043E000A3A1B4A10196A11DB11D81A392A3A3A372
:1043F000B4A38091C4119091C511A091C611B09140
:10440000C7110196A11DB11D8093C4119093C511D0
:10441000A093C611B093C7110E943B2F1FBF1F91DD
:1044200008958091BA108130C1F49FB7F8948091BB
:10443000B910882389F081508093B910882351F4F2
:104440008091DD11882321F49FBF0E94BA21089535
:104450009FBF08959FBF08959FBF08954F925F9299
:104460007F928F929F92AF92BF92CF92DF92EF9204
:10447000FF920F931F93CF93DF937C016B012A016F
:104480004801DB011D921C92FC0100811181DC01BD
:10449000F80109C08081813011F081E015C01296C9
:1044A000ED91FC9111973097A9F78091DD11882348
:1044B00031F082E0F4018083AA24BB24E5C080911E
:1044C000B910882321F08DE0D4018C93F5CF7FB60D
:1044D000F894F70150E0AA24BB2440E024C0D8019E
:1044E0008C918130D9F4D80111968D919C911297BD
:1044F000009791F0D2018D939D932D01D8011296D2
:104500001C921E921197D6010D931D936D01089474
:10451000A11CB11C51E004C0426002C07FBE95C026
:1045200032960081118101151105C9F6513039F417
:10453000F601118210827FBED4011C92A5C0E091C9
:10454000DE11F091DF11828D8068842B828F138EB3
:10455000318F208FC7010E9402207FBE0E94BA21A6
:104560003FB7F894C091DE11D091DF118B8D882375
:1045700011F08230A1F50A891B890115110551F04E
:10458000F601019311936F01118210820894A11C0E
:10459000B11C47C081E08B8F8E8D28A19F8DF701C4
:1045A000A081B181482F50E09095209515C0FD0164
:1045B000E40FF51F868189238683882331F41596BD
:1045C0008C911597822315968C9362E070E0E60E2D
:1045D000F71EF701A081B181109749F722C08E8D97
:1045E00028A19F8DF701A081B181482F50E09095BF
:1045F000209515C0FD01E40FF51F86818923868370
:10460000882331F415968C911597822315968C93F7
:1046100062E070E0E60EF71EF701A081B18110970D
:1046200049F78B8D882319F08230D9F415C0D80151
:104630008C918150823040F48E899F89F201918360
:104640008083D4011C9213C03FBFF60111821082F7
:1046500081E0D4018C9318C0F201118210828EE0A7
:1046600004C0F201118210828AE0D4018C93E0919F
:10467000DE11F091DF11128E138E138A128A158AC1
:10468000148A178A168A3FBFC501DF91CF911F9107
:104690000F91FF90EF90DF90CF90BF90AF909F90E1
:1046A0008F907F905F904F9008950E94F02E2FB7CB
:1046B000F8948091E0119091E111A091E211B091F4
:1046C000E3110196A11DB11D8093E0119093E111BA
:1046D000A093E211B093E3112FBF9091BA109130E3
:1046E00009F058C08091C310813009F453C0813063
:1046F00038F0823019F49093C31002C01092C310A6
:10470000A091C110B091C21031E03EC02FB7F89413
:1047100058968D919C915997009789F101975996D8
:104720009C938E935897892B51F55A969C915A9742
:10473000892F877341F0987C5A969C935A975B9681
:104740003C935B9703C05B961C925B975A968C9147
:104750005A9783FD14C08091D21190969C919097A6
:10476000892B8093D2115E96EC915E97F0E0ED522A
:10477000FE4E80815F969C915F97892B80831E9669
:104780000D90BC91A02D2FBF5C968C915C978F33C0
:1047900009F0BCCF08958091BA10882341F5E091CB
:1047A000D211F0E0EE5DFD4FA081EA2FF0E0ED5276
:1047B000FE4EE081F0E0EE5DFD4FAA0FAA0FAA0FBA
:1047C0008081A80FA093BF10A093C010B0E0AA0FE3
:1047D000BB1FA751B84E8D919C919093D11180939E
:1047E000D0119093DF118093DE110E94052F089560
:1047F0001F938091BA10813009F05BC01FB7F89405
:104800008091DD11882319F081508093DD11809112
:10481000DD11882309F04CC08091B910882309F07C
:1048200047C0E091D211F0E0EE5DFD4F8081E82FAE
:10483000F0E0ED52FE4EE081F0E0EE5DFD4F982F8E
:10484000990F990F990F8081980F9093BF108091C5
:10485000C010981769F1E92FF0E0EE0FFF1FE75144
:10486000F84E0190F081E02DF093D111E093D0113A
:1048700081A192A1A3A1B4A10196A11DB11D81A303
:1048800092A3A3A3B4A38091C4119091C511A09148
:10489000C611B091C7110196A11DB11D8093C4111D
:1048A0009093C511A093C611B093C7110E94AC2F6D
:1048B0001FBF1F9108954F925F926F927F928F92C8
:1048C0009F92AF92BF92CF92DF92EF92FF920F939F
:1048D0001F93DF93CF930F92CDB7DEB70E94A72E21
:1048E0001092E0111092E1111092E2111092E31176
:1048F0001092DD111092B9101092CF111092BA10CF
:104900001092C4111092C5111092C6111092C711C5
:104910001092BB101092BC101092BD101092BE10DD
:104920001092691810926A1810926B1810926C18F5
:104930001092C8111092C9111092CA111092CB1185
:104940001092E8171092D211E3EDF1E1119281E19A
:10495000EB3DF807D9F71092C0101092BF101092DB
:10496000D1111092D0111092DF111092DE11E4ECEF
:10497000F4E1119297E1E83EF907D9F7E9EEF7E1A2
:10498000119288E1E936F807D9F7A7EFB4E18FE390
:10499000FD01B5975096B183A08350978C931196E3
:1049A0001C921197AD5BBF4F97E1A83DB90781F706
:1049B0001092B4171092B3178C9311961C92109208
:1049C000C2101092C11084EC94E19093CD118093A9
:1049D000CC11E4EEF2E1119284E1E43CF807D9F75E
:1049E000E4EEF2E18FE3DF015E961082B283A183F1
:1049F0008687178694E1A63AB90711F0FD01F3CF37
:104A00001C9210A2178E84A715A684EE92E19093B3
:104A1000DC118093DB110F920F92B3E04B2E512CDF
:104A2000EDB7FEB75282418281EA91E260E070E028
:104A300043EE52E12FE30FEF1FEFA4EEEA2EA1E1C8
:104A4000FA2EA12CF1E0BF2EC12CD12C8824992460
:104A50000E94972C0F900F908FE366E072E03E016A
:104A60000894611C711CA3010E941F2C0F920F92CD
:104A7000EDB7FEB75282418283EC99E360E070E0CB
:104A800043EC51E12EE30EEF1FEFE4ECEE2EE0E1FC
:104A9000FE2E0E94972C0F900F908EE364E172E03F
:104AA000A3010E941F2C0E94A82E0F90CF91DF918E
:104AB0001F910F91FF90EF90DF90CF90BF90AF903C
:104AC0009F908F907F906F905F904F900895FC0122
:104AD0008081813019F020E030E007C08FB7F89472
:104AE00021813281128211828FBFC9010895CF9333
:104AF000DF93FC01DB018081813011F081E01BC07C
:104B00004FB7F89485811A968C931A979F012A5F64
:104B10003F4F6E5F7F4F90E0E90189919E01EB016D
:104B20008993BE019F5F9830B9F7818192818D93FF
:104B30009C934FBF80E0DF91CF910895EF92FF9259
:104B40000F931F93CF93DF93EC018B01E42E8881A9
:104B5000813011F081E028C0FFB6F8948D81882360
:104B6000C1F040FD07C00AC0CE01B80142E020E01C
:104B70000E943B1F8D818823B9F705C0CE0142E01A
:104B800020E00E943B1FFFBEE2FC0DC00E94BA2144
:104B90000AC089819A81892B19F0FFBE84E104C083
:104BA0007A836983FFBE80E0DF91CF911F910F91DF
:104BB000FF90EF9008951F93FC018081813011F0E8
:104BC00081E019C01FB7F8948581882349F0CF018F
:104BD00042E020E00E943B1F1FBF0E94BA210AC092
:104BE00081819281892B19F01FBF84E104C07283F7
:104BF00061831FBF80E01F910895EF92FF920F9392
:104C00001F93CF93DF93EC017A018881813021F0EB
:104C100081E0FA01808327C00FB7F8948D81882343
:104C2000F9F0613071F410E008C0CE0160E070E08E
:104C300042E022E00E943B1F1F5F8D818823A9F77D
:104C400008C0CE0160E070E042E022E00E943B1F1D
:104C500011E00FBF0E94BA218EE0F701808304C0EB
:104C60000FBFFA01108210E0812FDF91CF911F91C9
:104C70000F91FF90EF900895DF92EF92FF920F93C4
:104C80001F93CF93DF937C01EA01FC018081813087
:104C900011F081E005C08091DD11882329F082E0C8
:104CA000888300E010E048C08091B910882311F09B
:104CB0008DE0F6CFDFB6F894F7010181128101157E
:104CC000110529F012821182DFBE188235C0E091F1
:104CD000DE11F091DF11828D8260828F138E718FD1
:104CE000608FC7010E94CF1FDFBE0E94BA21DFB6CE
:104CF000F894E091DE11F091DF11838D882319F093
:104D0000823039F404C006891789188208C08EE001
:104D100005C0CF01B7010E943C208AE08883E09162
:104D2000DE11F091DF11128E138E138A128A158A0A
:104D3000148A178A168ADFBEC801DF91CF911F91AE
:104D40000F91FF90EF90DF900895CF93DF93AC0128
:104D50008091DD11882319F0C0E0D0E01DC02FB78D
:104D6000F894C091DB11D091DC11209731F089814A
:104D70009A819093DC118093DB112FBF209761F013
:104D800081E088831C821B825A8349838FE38E874C
:104D90001F86CE010E947B20CE01DF91CF91089526
:104DA000CF93DF93DC01EB018C91843011F081E033
:104DB00005C08091DD11882319F082E0888327C027
:104DC0005FB7F89413966D917C9114976F3FE9F457
:104DD000E091DE11F091DF11448D842F90E09B0172
:104DE0002070822B932B14969C938E93139712967C
:104DF000FC93EE931197741720F05FBF88E78883C8
:104E000002C05FBF188281E003C05FBF188280E0EC
:104E1000DF91CF910895DC01FB018091DD118823A2
:104E200011F086E008958C91843011F081E00895AE
:104E30002FB7F89413969C91139714968C9114970E
:104E4000838792879F3F19F481E0818701C0118693
:104E500015968C9115978087169690E08D91819389
:104E60009F5F9830D9F72FBF80E008950F931F936D
:104E7000CF93DF93EC018091DD11882311F085E061
:104E8000A5C08881843011F081E0A0C01FB7F894DC
:104E90003B810C81A091DE11B091DF1189819A8153
:104EA000A817B90719F01FBF84E690C05C968C91D3
:104EB0005C97801709F051C05E96EC915E97F0E028
:104EC000ED52FE4E5F968C915F978095908189237D
:104ED0008083882349F490969C9190979095809137
:104EE000D21189238093D2115C963C935C97832FD7
:104EF00086958695869587705E968C935E97232F10
:104F000027705D962C935D9741E050E0BA0102C096
:104F1000660F771F8A95E2F790966C93909702C080
:104F2000440F551F2A95E2F75F964C935F972091A7
:104F3000D211262B2093D2115E96EC915E97F0E071
:104F4000ED52FE4E8081842B8083E32FF0E0EE0F44
:104F5000FF1FE751F84EB183A083E02FF0E0EE0F82
:104F6000FF1FE751F84E81E090E0918380838D81AF
:104F7000882319F1CE0160E070E040E120E00E945A
:104F80003B1FE82FF0E02B813C8120702E2B3F2B24
:104F90003C832B83EE0FFF1FE751F84E20813181B8
:104FA0003A832983081728F01FBF0E94BA2188E797
:104FB0000DC01FBF0E94BA2108C08B819C818F6FDA
:104FC0009C838B831A8219821FBF80E0DF91CF916F
:104FD0001F910F910895EF92FF920F931F93CF931C
:104FE000DF93EC018A018881843011F081E0C0C038
:104FF0008091DD11882311F08FE0BAC0EFB6F894EC
:10500000FD80FF2011F0FF24F394662321F061302E
:1050100009F0ACC01FC0FF20D1F48FE38E871F863C
:10502000EC81F0E0EE0FFF1FE751F84E1182108285
:1050300018828091DB119091DC119A8389831C8204
:105040001B82D093DC11C093DB11EFBE8AC0EFBE90
:1050500089E48EC03B819C81A981BA81109709F4B3
:105060005FC05C968C915C97891709F059C05E9679
:10507000EC915E97F0E0ED52FE4E5F968C915F975B
:105080008095908189238083882349F490969C9110
:10509000909790958091D21189238093D2115C963C
:1050A0003C935C97832F86958695869587705E9650
:1050B0008C935E97232F27705D962C935D9741E02C
:1050C00050E0BA0102C0660F771F8A95E2F790960A
:1050D0006C93909702C0440F551F2A95E2F75F9694
:1050E0004C935F972091D211262B2093D2115E967C
:1050F000EC915E97F0E0ED52FE4E8081842B808330
:10510000E32FF0E0EE0FFF1FE751F84EB183A083CD
:1051100007C0CE0160E070E040E120E00E943B1F4C
:105120008D818823B1F78FE38E871F86EC81F0E0B5
:10513000EE0FFF1FE751F84E118210821882809106
:10514000DB119091DC119A8389831C821B82D0939E
:10515000DC11C093DB11EFBE71E0F71611F40E9471
:10516000BA21F8011082C0E0D0E004C0EFBE87E0B1
:10517000F8018083CE01DF91CF911F910F91FF90B5
:10518000EF900895AF92BF92DF92EF92FF920F934C
:105190001F93CF93DF938C015B017A01DC018C912B
:1051A000843011F081E033C08091DD11882321F03B
:1051B00082E0DA018C9302C18091B910882311F04A
:1051C0008DE025C0DFB6F894D80113962D913C915F
:1051D0001497432F632F2F3F09F5207014963C93AB
:1051E0002E931397E091DE11F091DF11848D90E002
:1051F000822B932B14969C938E9313971296FC9369
:10520000EE931197848D481728F0DFBE88E7F701E9
:105210008083D4C0DFBED7011C92D0C0F801A18129
:10522000B2815C968C915C97381708F092C0E0913F
:10523000DE11F091DF11848D821708F08AC05E962E
:105240008C915E97282F30E0F901ED52FE4E40819F
:105250005F969C915F97842F892389F0892F809591
:1052600084238083882349F490969C91909790950D
:105270008091D21189238093D211E1E018C0529617
:10528000CD91DC915397209789F0FE01E20FF31F37
:10529000892F8095968189238683882339F4909677
:1052A0009C91909790958D8189238D83E0E05C9609
:1052B0006C935C97862F8695869586955E968C93E3
:1052C0005E97962F97705D969C935D9721E030E0F6
:1052D000A90102C0440F551F8A95E2F790964C939E
:1052E000909702C0220F331F9A95E2F75F962C9396
:1052F0005F97E13091F48091D211842B8093D21189
:105300005E96EC915E97F0E0ED52FE4E80815F96E6
:105310009C915F97892B808314C05296ED91FC91EC
:105320005397309771F08581842B85835E968C919D
:105330005E97E80FF11D86815F969C915F97892BA0
:105340008683E62FF0E0EE0FFF1FE751F84EB183A2
:10535000A083E091DE11F091DF11828D8061828F58
:10536000138EB18EA08EC8010E94CF1FDFBE0E9497
:10537000BA21DFB6F894E091DE11F091DF11838D50
:10538000882319F0823041F403C0D7011C920BC06E
:105390008EE0F701808307C0CF01B8010E943C2056
:1053A0008AE0D7018C93E091DE11F091DF11128E2B
:1053B000138E138A128A158A148ADFBEDF91CF9169
:1053C0001F910F91FF90EF90DF90BF90AF900895E5
:1053D0000F931F93CF93DF93382F8B018091DD11B3
:1053E000882311F080E10EC02FB7F894E32FF0E08E
:1053F000EE0FFF1FE751F84E80819181892B39F024
:105400002FBF88E2F8018083C0E0D0E029C081E0AE
:1054100090E091838083C091DB11D091DC112097C3
:1054200039F4118210822FBF84E0FB01808318C001
:1054300089819A819093DC118093DB112FBF84E0E6
:105440008883932F80E08F6F9C838B831A821982CD
:105450008FE38E871F86CE010E947B20F801108289
:10546000CE01DF91CF911F910F910895EF92FF929E
:105470000F931F93DB011D921D921D921C92139797
:1054800014961D921D921D921C9217979FB7F89427
:105490008F3F29F4E091DE11F091DF11848DE82F28
:1054A000F0E0EE0FFF1FE751F84E0190F081E02D84
:1054B000309711F49FBF04C0E130F10519F49FBF8C
:1054C00083E42CC0828580FD03C09FBF85E426C095
:1054D000E680F78000851185648175819FBF20E09B
:1054E00030E040E050E004C02F5F3F4F4F4F5F4F30
:1054F000FB01E20FF31F80818823B1F32D933D93CD
:105500004D935C931397E21AF30A040B150B149650
:10551000ED92FD920D931C93179780E01F910F91D0
:10552000FF90EF900895FC0120FF0DC021FD06C003
:10553000089541505040604070401192411551050E
:1055400061057105B1F70895E82F3FB7F894A09170
:10555000DE11B091DF118F3F19F45C96EC9106C01B
:105560005C968C91E81711F020E001C021E0F0E09A
:10557000EE0FFF1FE751F84EA081B181109719F48B
:105580003FBF88E40895A130B10519F43FBF83E41B
:1055900008955E96EC915E97F0E0ED52FE4E5F96B8
:1055A0008C915F978095908189238083882349F42B
:1055B00090969C91909790958091D2118923809399
:1055C000D2115A968C915A9788605A968C933FBF05
:1055D000213011F080E008950E94BA2180E0089502
:1055E000E82F2FB7F894F0E0EE0FFF1FE751F84EC9
:1055F000A081B181109719F42FBF86E40895A130DE
:10560000B10519F42FBF83E408955A968C915A97E7
:1056100083FF2CC0877F5A968C935A97882319F55D
:1056200058968D919C915997892BD9F48091D211DC
:1056300090969C919097892B8093D2115E96EC91D5
:105640005E97F0E0ED52FE4E80815F969C91892B33
:1056500080832FBF8091BA10813031F40E94BA212B
:1056600003C02FBF01C02FBF80E008952FBF84E487
:105670000895AF92BF92CF92DF92EF92FF920F9375
:105680001F93CF93DF93282FD62ECFB6F894A62F53
:10569000B0E0FD01EE0FFF1FE751F84E80819181D0
:1056A000892B19F0CFBE88E2BFC02F3F29F4E091CB
:1056B000DE11F091DF11248DE22FF0E0EE0FFF1FDD
:1056C000E751F84EC081D181209719F4CFBE89E20D
:1056D000ABC0C130D10519F4CFBE83E4A5C0AD2C59
:1056E000A694A694A69457E0B52EBD206A2D70E02E
:1056F00021E030E0C9010A2C02C0880F991F0A94EA
:10570000E2F7E82EF22E0B2C01C0FF0C0A94EAF708
:1057100011821082AA0FBB1FA751B84ECD93DC9304
:1057200008A11F8D8E8D282F30E0F901ED52FE4E1D
:105730009081892F8123C1F0812F809589238083D7
:10574000882339F4902F90958091D21189238093EA
:10575000D2118091D2118E298093D211FB01ED528A
:10576000FE4E80818F298083AA89BB89109701F121
:10577000FD01E20FF31F812F809596818923868397
:10578000882349F4902F909515968C91159789232D
:1057900015968C93159715968C9115978E291596BD
:1057A0008C931597FD01E60FF71F86818F2986835D
:1057B0004C895D894115510551F1FA01A081B181F2
:1057C0001095902F909521C0FD01E20FF31F868167
:1057D00081238683882339F415968C911597892324
:1057E00015968C93159715968C9115978E2915966D
:1057F0008C931597FD01E60FF71F86818F2986830D
:105800004E5F5F4FFA01A081B1811097E9F6DC8EFF
:10581000AE8EBD8EE8A2FF8ECFBE8091BA108130D1
:1058200011F40E94BA2180E0DF91CF911F910F9176
:10583000FF90EF90DF90CF90BF90AF900895CF9200
:10584000DF92FF920F931F93CF93DF93E82F6B01AB
:105850008A018091DD11882311F082E121C0FFB619
:10586000F894EF3F29F4E091DE11F091DF11E48D1F
:10587000F0E0EE0FFF1FE751F84EC081D181209775
:1058800011F4FFBE04C0C130D10519F4FFBE83E49A
:1058900007C0C6010E94A720803128F0FFBE81E426
:1058A000F801808308C0CE01C396B6010E949820FB
:1058B000FFBEF8011082DF91CF911F910F91FF90F1
:1058C000DF90CF9008951F93CF93DF93E82F9B0134
:1058D000EA018091DD11882311F081E115C01FB725
:1058E000F894EF3F29F4E091DE11F091DF11E48D9F
:1058F000F0E0EE0FFF1FE751F84E608171816115F6
:10590000710529F41FBF83E4888380E00CC06130F7
:10591000710511F41FBFF7CF6D5C7F4FC9010E9465
:1059200098201FBF1882DF91CF911F9108952F9269
:105930003F924F925F926F927F928F929F92AF921F
:10594000BF92CF92DF92EF92FF920F931F93DF935C
:10595000CF9300D00F920F92CDB7DEB73C012B0151
:105960001A012983AA82CB82DC826401AB8C2C8D44
:105970002D832FB7F8948091DD11882319F02FBF64
:105980001CE355C03981832E9924F401EE0FFF1FCB
:10599000E751F84E80819181892B09F046C081E062
:1059A00090E0918380832FBFA0FE16C0A1FE14C09B
:1059B0002A813B2D4B815C81C901DA01AC01BD011B
:1059C000F70105C0415050406040704011924115B0
:1059D000510561057105B1F7C301B201A1012A2D7D
:1059E0003D810E94A92EBC018981A7019801EA800E
:1059F000FB2C0B811C81BD800E94B420182F8823B2
:105A000039F48091BA10813091F40E94BA210FC00C
:105A10008FB7F894880C991CE9EEF7E18E0E9F1E63
:105A2000F401118210828FBF02C02FBF18E2812FB4
:105A30000F900F900F900F900F90CF91DF911F91CB
:105A40000F91FF90EF90DF90CF90BF90AF909F901D
:105A50008F907F906F905F904F903F902F90089520
:105A6000AF92BF92CF92DF92EF92FF920F931F936C
:105A7000CF93DF93DC01122F2FB7F8948091DD11C3
:105A8000882319F02FBF1CE33AC0C12FD0E0FE01DC
:105A9000EE0FFF1FE751F84E80819181892B69F548
:105AA00081E090E0918380832FBFCD0120E030E042
:105AB0000E94A92EBC01812F40E050E020E030E0A0
:105AC000EE24FF248701CC24DD24AA24BB240E94D9
:105AD000B420182F882339F48091BA10813079F4DA
:105AE0000E94BA210CC08FB7F894CC0FDD1FC751AC
:105AF000D84E198218828FBF02C02FBF18E2812FA3
:105B0000DF91CF911F910F91FF90EF90DF90CF9099
:105B1000BF90AF9008958FB7F8942091E011309125
:105B2000E1114091E2115091E3118FBFB901CA0117
:105B300008952FB7F8946093E0117093E11180936A
:105B4000E2119093E3112FBF08958F3310F08AE292
:105B500008952FB7F894E82FF0E0EE0FFF1FE751FC
:105B6000F84EA081B181109711F42FBF04C0A1306D
:105B7000B10519F42FBF83E4089558968D919C9137
:105B80005997892B19F42FBF80E5089559961C92D7
:105B90001E9258975A969C915A97892F877349F06D
:105BA000987C5A969C935A9781E05B968C935B976E
:105BB00003C05B961C925B975A968C915A9783FD13
:105BC00018C08091D21190969C919097892B8093C8
:105BD000D2115E96EC915E97F0E0ED52FE4E808120
:105BE0005F969C91892B80832FBF0E94BA2180E011
:105BF00008952FBF80E008959C018091DD118823D6
:105C000041F52115310529F14FB7F894A091DE1126
:105C1000B091DF115E96EC915E97F0E0ED52FE4E92
:105C20005F968C915F9780959081892380838823EC
:105C300049F490969C91909790958091D2118923E8
:105C40008093D21159963C932E9358974FBF0E9440
:105C5000BA2108958F929F92AF92BF92CF92DF9216
:105C6000EF92FF920F931F93CF93DF93882EE62E30
:105C7000942E8091DD11882311F085E55BC0B90178
:105C800080E090E06D5F7F4F8F4F9F4F37E0660F52
:105C9000771F881F991F3A95D1F728EE33E040E02F
:105CA00050E00E9424F459016A016E2D70E080E0FA
:105CB00090E02CE330E040E050E00E94F2F37B0102
:105CC0008C01E90CF11C011D111D682D70E080E0B4
:105CD00090E020E13EE040E050E00E94F2F3E60E6A
:105CE000F71E081F191F27E0EE0CFF1C001F111FD5
:105CF0002A95D1F7AE0CBF1CC01ED11EC601AA2723
:105D0000BB27EC018FEF9FEFA0E0B0E0A822B92203
:105D1000CA22DB22C5010E94FC2D09C080E090E868
:105D20000E94FC2D80E090E80E94FC2D2197209796
:105D3000A9F780E0DF91CF911F910F91FF90EF9035
:105D4000DF90CF90BF90AF909F908F90089508956F
:105D50000895FA01808392931292129286E18293BF
:105D600088E2829389E2829380E88293129282E0B1
:105D7000829383E0829384E0829385E0829386E03D
:105D8000829387E0829388E0829389E0829380E126
:105D9000829381E1829382E1829383E1829384E121
:105DA000829385E1829387E1829388E1829389E1FE
:105DB000829380E2829381E2829382E2829383E201
:105DC00082936293729386E2829387E2829380E366
:105DD000829381E38293129212923197CF010895B8
:105DE0000E94B13308950E94B03308950E94C333D6
:105DF00008950E94AF3308950E94B23308950E941F
:105E0000AE3308950E94AD330895F0DF0091BA10CB
:105E100003950093BA10E091D011F091D111019146
:105E20000DBF01910EBF0F910CBF0F910BBFFF91E2
:105E3000EF91BF91AF919F918F917F916F915F9102
:105E40004F913F912F911F91FF90EF90DF90CF9056
:105E5000BF90AF909F908F907F906F905F904F908A
:105E60003F902F901F900F910F770FBFDF91CF9131
:105E70000F910F9018950F920F93CF93DF930FB759
:105E80000F931F922F923F924F925F926F927F9249
:105E90008F929F92AF92BF92CF92DF92EF92FF923A
:105EA0001F932F933F934F935F936F937F938F93A2
:105EB0009F93AF93BF93EF93FF930BB70F930CB7E1
:105EC0000F931124E091DE11F091DF110DB70193D2
:105ED0000EB701930E94F62E0091BF100093C010E0
:105EE000E091D011F091D111E093DE11F093DF1128
:105EF00001910DBF01910EBF0F910CBF0F910BBF10
:105F0000FF91EF91BF91AF919F918F917F916F9191
:105F10005F914F913F912F911F91FF90EF90DF90F4
:105F2000CF90BF90AF909F908F907F906F905F9039
:105F30004F903F902F901F900F9107FD06C00FBF0D
:105F4000DF91CF910F910F9008950F770FBFDF91E1
:105F5000CF910F910F9018950E94F62E0091BF10CF
:105F60000093C010E091D011F091D111E093DE11B7
:105F7000F093DF1101910DBF01910EBF0F910CBF86
:105F80000F910BBFFF91EF91BF91AF919F918F91B7
:105F90007F916F915F914F913F912F911F91FF9052
:105FA000EF90DF90CF90BF90AF909F908F907F90B9
:105FB0006F905F904F903F902F901F900F9107FD33
:105FC000C4CF0FBFDF91CF910F910F9008950F773E
:105FD0000FBFDF91CF910F910F901895AF92BF92A5
:105FE000CF92DF92EF920F931F93CF93DF935A01DB
:105FF0006B01122F843010F087E938C0282F30E071
:10600000F901EE0FFF1FE20FF31FEE0FFF1FEC5D14
:10601000FC4FC181D28184E190E0289FF001299F4B
:10602000F00D389FF00D1124E359F74E86859785C2
:10603000892B11F486E91AC00894A11CB11CC11C5B
:10604000D11C60E078E087E090E0A60195010E9415
:1060500024F49FB7F89419823D832C83188288E931
:106060008983012B0E290A839FBF80E0DF91CF91A6
:106070001F910F91EF90DF90CF90BF90AF90089558
:10608000FC01E081E13001F1E13030F0E230B9F1C2
:10609000E33009F064C04BC0662321F480916400B2
:1060A000826003C0809164008D7F809364008DB115
:1060B000847F8A608DB9662319F08EB1886002C032
:1060C0008EB1877F8EB90895662321F48091650093
:1060D000816003C0809165008E7F809365008AB1E6
:1060E000837F88608AB9809107018360809307016C
:1060F000809108018C7F8260809308010895662357
:1061000021F480916500826003C0809165008D7FDD
:1061100080936500809101018C7C826380930101F2
:10612000809102018F7C8062809302010895662332
:1061300021F480916500846003C0809165008B7FAD
:1061400080936500809104018C7F826080930401BC
:1061500080B3836080BB81B38C7F826081BB0895F4
:10616000FC0111821082138212821582148216821F
:106170001782108611861386128615861486178656
:10618000168680898160808B80898D7F808B128AC2
:10619000118A138A08950F931F93CF93DF930DE60F
:1061A00018E1C4E2D3E0E981FA811182CE0160E016
:1061B0000E944030C8010E94B03026960C5E1F4FEE
:1061C00083E0CC33D80779F7DF91CF911F910F91FE
:1061D00008950F931F93CF93DF93982FDB01EA016C
:1061E000A801843010F087E92CC084E1989FF00169
:1061F0001124E359F74E86859785892B11F486E99A
:1062000020C06FB7F894109721F0828593858D9305
:106210009C93209721F08081918199838883211517
:10622000310529F082819381D9018D939C93411589
:10623000510529F084819581FA01918380836FBF94
:1062400080E0DF91CF911F910F910895982FDB018E
:10625000843010F087E9089584E1989FF0011124BB
:10626000E359F74E86859785892B11F486E90895C1
:106270009FB7F8946115710521F083898C9311966D
:106280001C929FBF80E008950F931F93CF93DF93DD
:10629000982FDB01EA01A801843010F087E925C0BE
:1062A00084E1989FF0011124E359F74E8685978584
:1062B000892B11F486E919C09FB7F894611571050F
:1062C00011F086818C93209711F0878188832115A6
:1062D000310519F08085D9018C934115510519F0CC
:1062E0008185FA0180839FBF80E0DF91CF911F916C
:1062F0000F910895982F843010F087E9089584E174
:10630000989FF0011124E359F74E86859785892BD4
:1063100011F486E908959FB7F89460FF0AC01682C9
:1063200017821386128680898160808B80898D7F99
:10633000808B61FF03C010861186138A9FBF80E0A7
:106340000895982FDB01843010F087E9089584E1E7
:10635000989FF0011124E359F74E86859785892B84
:1063600011F486E908952FB7F894828593858C936C
:106370002FBF80E008950F931F93CF93DF93CDE657
:10638000D8E100E012E0EE85FF853097F9F08889CA
:1063900080FD10C0888981FF0AC08581882351F063
:1063A000B80160507140CF010E94DB2503C088898D
:1063B0008260888B8B89882349F4E989FA898581F1
:1063C000882321F0CF01B8010E94DB250F5F1F4F0A
:1063D00088E1C93AD80711F06496D5CFDF91CF9103
:1063E0001F910F9108956F927F929F92AF92BF92EB
:1063F000CF92DF92EF92FF920F931F93DF93CF9391
:106400000F92CDB7DEB7282F962E5A01843010F0A8
:1064100087E953C084E1289F800111240359174E56
:10642000F80186859785892B11F486E946C0198283
:10643000822F90E0FC01EE0FFF1FE80FF91FEE0F17
:10644000FF1FEC5DFC4FE180F280D82ECC243E0192
:106450000894611C711C9FB7F894F701818185FD38
:1064600005C0808185FF02C0968218C0F80183892B
:106470008F3F11F480E013C0F80183898F5F838B15
:106480008085F601E80FF11DE050FC4790828F5F98
:10649000F8018087F70181818062818381E09FBF5D
:1064A000882351F4F80181899289B501A3010E94E2
:1064B0003C268981882379F289810F90CF91DF91E1
:1064C0001F910F91FF90EF90DF90CF90BF90AF9012
:1064D0009F907F906F9008959F92AF92BF92CF92BE
:1064E000DF92EF92FF920F931F93CF93DF93982E3B
:1064F0005B017A016901EB0101C02196E114F1040D
:1065000011F480E00AC0892D6881A6010E94F33150
:106510000894E108F108882381F30115110511F0B1
:10652000F80180839E012A193B09C901DF91CF91AF
:106530001F910F91FF90EF90DF90CF90BF90AF90A1
:106540009F900895EF92FF920F931F937A01890114
:10655000DB010D900020E9F71197A61BB70BAD01E9
:1065600097010E946C321F910F91FF90EF90089558
:106570006F927F928F929F92AF92BF92CF92DF9253
:10658000EF92FF920F931F93DF93CF930F92CDB7AC
:10659000DEB7A82E4B016A0183E08A1530F441155D
:1065A000510509F453C087E910C084E1A89E800119
:1065B00011240359174EF80186859785892B41F4DC
:1065C0004115510509F442C086E9F60180833EC0B9
:1065D0001982BB243E010894611C711C2FB7F894EA
:1065E000F80182859385892B11F480E01BC0F801A6
:1065F0008285938501979387828782859385892BEE
:1066000019F480898160808BF8018781FA2CEE244F
:10661000F701E80FF11DE050F048B0808F5FF801FE
:10662000878381E02FBF882351F4F8018685978501
:10663000B401A3010E943C268981882379F2C11408
:10664000D10429F08981F601808301C0BB248B2D00
:106650000F90CF91DF911F910F91FF90EF90DF90FE
:10666000CF90BF90AF909F908F907F906F90089544
:106670005F926F927F928F929F92AF92BF92CF92D2
:10668000DF92EF92FF920F931F93CF93DF935A0104
:106690006B01522E702E6E2C843010F087E94DC0A5
:1066A00090E024E130E0829F7001839FF00C929F84
:1066B000F00C11242DE638E1E20EF31EEC01CC0FB4
:1066C000DD1FC80FD91FCC0FDD1FCC5DDC4F8980CB
:1066D0009A80F70186859785892B11F088E92DC06E
:1066E0000894A11CB11CC11CD11C60E078E087E0BB
:1066F00090E0A60195010E9424F4890180E090E0D9
:106700000E94A526F7019787868780E090E00E9487
:10671000A526F701928B818BFFB6F894CE0161E03C
:106720000E944030F40115830483108288E981833C
:10673000752876287282FFBE80E0DF91CF911F918D
:106740000F91FF90EF90DF90CF90BF90AF909F9010
:106750008F907F906F905F900895089508950895A9
:106760000895089561E070E080E090E00E94E83BC9
:1067700083B7817F83BF83B7816083BF889583B7E9
:106780008E7F83BF0895E091DE11F091DF11848D3B
:10679000882339F4E091D011F091D111848D8823B0
:1067A00031F062E070E080E090E00E94E83B809190
:1067B000DE119091DF110E9460390895E4E6F0E067
:1067C00080818860808380818064808308952FB772
:1067D000F89480916500877F8093650080916400C4
:1067E0008F7B809364001092900084E080939100EE
:1067F00010929200109295001092940080E2809383
:10680000B60082E08093B00081E08093B1001092E6
:10681000B2008FEF8093B3008091B60090E08F714B
:106820009070892BC9F787E087BB82E08093700066
:106830002FBF08959FB7F894E0E7F0E020818083B0
:106840009FBF822F08952FB7F894609180067091B2
:10685000810680918206909183062FBF08952FB7FD
:10686000F89460937C0670937D0680937E069093E7
:106870007F062FBF80E008952FB7F89460917C06C3
:1068800070917D0680917E0690917F062FBF0895BE
:106890002F923F924F925F926F927F928F929F9230
:1068A000AF92BF92CF92DF92EF92FF920F931F931E
:1068B000DF93CF93CDB7DEB762970FB6F894DEBF04
:1068C0000FBECDBF89829A82AB82BC82CD82DE822E
:1068D000EF82F8862B873C878B859C8569807A8040
:1068E0002F8138854D805E802B803C804FEF641671
:1068F0004FEF740629F420E030E040E050E097C00C
:10690000902E52E0501710F45C0106C0ACE09A0ED5
:106910005C010894A108B1086901EE24D7FCE09459
:10692000FE2C80E89CEBAAEDBFEFC80ED91EEA1E34
:10693000FB1EB501882777FD8095982F25EB35E064
:1069400040E050E00E94F2F3645A7D4D86499F4F2B
:1069500024E030E040E050E00E9446F4C20ED31E36
:10696000E41EF51EC5016CE97FEF0E9411F48B0156
:10697000C50160E971E00E9411F4060F171F0E5F58
:106980001F4F222717FD2095322FC00ED11EE21E69
:10699000F31E892D90E0019629E930E0DC01A29FE9
:1069A000C001A39F900DB29F900D112465E070E08F
:1069B0000E9411F4882777FD8095982FC60ED71E68
:1069C000E81EF91EC701B60128E130E040E050E0C2
:1069D0000E94F2F39B01AC01B201882777FD8095FC
:1069E000982F620F731F841F951F2CE330E040E047
:1069F00050E00E94F2F39B01AC01B101882777FDC2
:106A00008095982F620F731F841F951F2CE330E031
:106A100040E050E00E94F2F39B01AC01C301AA27C1
:106A200097FDA095BA2F280F391F4A1F5B1FB90188
:106A3000CA0162960FB6F894DEBF0FBECDBFCF91EC
:106A4000DF911F910F91FF90EF90DF90CF90BF905B
:106A5000AF909F908F907F906F905F904F903F90FE
:106A60002F900895AF92BF92CF92DF92EF92FF9254
:106A70000F931F93FC01E080F18002811381C80114
:106A8000B70120E831E541E050E00E9424F4D62E21
:106A9000C72EB82EA92EC801B70120E831E541E084
:106AA00050E00E9424F4C901DA017C018D016D2DB2
:106AB0007C2D8B2D9A2D2CE330E040E050E00E949D
:106AC00024F470938606609385066D2D7C2D8B2DA6
:106AD0009A2D20E13EE040E050E00E9424F42CE3B7
:106AE00030E040E050E00E9424F430938806209388
:106AF00087066D2D7C2D8B2D9A2D20E13EE040E008
:106B000050E00E9424F430938A0620938906C8013D
:106B1000B7016C5F7F4F8F4F9F4F27E030E040E021
:106B200050E00E9424F4709392066093910622EB49
:106B300037E01FC0AB2899F4C90164E670E00E94F9
:106B400011F4892B39F4C90160E971E00E9411F454
:106B5000892B29F48EE691E0A0E0B0E004C08DE638
:106B600091E0A0E0B0E0E81AF90A0A0B1B0B2F5FD6
:106B70003F4F83E0A82EB12CA222B322A114B1046E
:106B800099F4C90164E670E00E9411F4892B39F48C
:106B9000C90160E971E00E9411F4892B29F48EE6A5
:106BA00091E0A0E0B0E004C08DE691E0A0E0B0E0AC
:106BB000E816F9060A071B0708F0BCCF2C56374029
:106BC0003093900620938F062459384FC701E092E6
:106BD000930690939406C90164E670E00E9411F454
:106BE0006C01C90160E971E00E9411F49C0140E070
:106BF00050E02FC0A114B10419F080E090E00EC065
:106C0000C114D10419F081E090E008C0E0E0F0E0A8
:106C10002115310511F4E1E0F0E0CF01FC01EE0FA8
:106C2000FF1FE80FF91FEE0FFF1FEE0FFF1FE40F0E
:106C3000F51FEE0FFF1FE45CFC4F80819181AA27B6
:106C400097FDA095BA2FE81AF90A0A0B1B0B4F5FA4
:106C50005F4FA114B10419F080E090E00EC0C114A0
:106C6000D10419F081E090E008C0E0E0F0E02115E7
:106C7000310511F4E1E0F0E0CF01FC01EE0FFF1F60
:106C8000E80FF91FEE0FFF1FEE0FFF1FE40FF51FB8
:106C9000EE0FFF1FE45CFC4F80819181AA2797FDD6
:106CA000A095BA2FE816F9060A071B0708F0A2CF2D
:106CB00050938E0640938D06C701019690938C06E3
:106CC00080938B06109296061092950685E896E0C2
:106CD0001F910F91FF90EF90DF90CF90BF90AF90FA
:106CE00008950F920F93CF93DF930FB700680F9320
:106CF0001F922F923F924F925F926F927F928F924C
:106D00009F92AF92BF92CF92DF92EF92FF921F932A
:106D10002F933F934F935F936F937F938F939F93A3
:106D2000AF93BF93EF93FF930BB70F930CB70F93F2
:106D300011240091DD1103950093DD11013041F420
:106D4000E091DE11F091DF110DB701930EB70193C1
:106D5000809170008D7F8093700078940E945523FD
:106D60000E94BB31809184068F3721F08F5F809322
:106D700084062CC010928406809180069091810632
:106D8000A0918206B09183060196A11DB11D80934A
:106D9000800690938106A0938206B093830680912B
:106DA0007C0690917D06A0917E06B0917F060097AB
:106DB000A105B10559F00196A11DB11D80937C0676
:106DC00090937D06A0937E06B0937F06F894809101
:106DD00070008260809370000E94F8230F910CBFB6
:106DE0000F910BBFFF91EF91BF91AF919F918F9149
:106DF0007F916F915F914F913F912F911F91FF90E4
:106E0000EF90DF90CF90BF90AF909F908F907F904A
:106E10006F905F904F903F902F901F900F910F7742
:106E20000FBFDF91CF910F910F90189541E050E087
:106E300068E070E020910701CB01042E02C0880FAA
:106E4000991F0A94E2F7382F3095232320930701E6
:106E500020910A01822B80930A0180910B01382333
:106E600030930B014F5F5F4F4430510519F7089580
:106E7000FB019C0180E12030380718F080E090E0B1
:106E80000895F999FECFF999FECF32BD21BDF89A48
:106E900080B580838FEF90E00895FB012FE08F3F56
:106EA000920710F080E00895F999FECFF999FECF8E
:106EB00092BD81BDF89A20B5F999FECF019692BD99
:106EC00081BDF89A80B5208381838FEF0895FB01FF
:106ED0009C0180E120303807D0F480E090E1821BF3
:106EE000930B8417950798F0F999FECF0BC0F99989
:106EF000FECF32BD21BDF89A80B581932F5F3F4F01
:106F0000415050404115510591F78FEF089580E0B1
:106F100008959C0180E12030380710F080E008954A
:106F2000F999FECFF999FECF1FBA32BD21BD60BDE0
:106F30000FB6F894FA9AF99A0FBE8FEF08959C0154
:106F400080E12030380710F080E00895F999FECFF5
:106F5000F999FECF1FBA32BD21BD60BD0FB6F894BE
:106F6000FA9AF99A0FBE8FEF08952FE08F3F92079C
:106F700010F080E00895F999FECFF999FECF1FBA7D
:106F800092BD81BD60BD0FB6F894FA9AF99A0FBE12
:106F9000F999FECF1FBA019692BD81BD70BD0FB6A3
:106FA000F894FA9AF99A0FBE8FEF08952FE08F3F69
:106FB000920710F080E00895F999FECFF999FECF7D
:106FC0001FBA92BD81BD60BD0FB6F894FA9AF99AC6
:106FD0000FBEF999FECF1FBA019692BD81BD70BD5B
:106FE0000FB6F894FA9AF99A0FBE8FEF0895FB0145
:106FF0009C0180E12030380700F580E090E1821BA1
:10700000930B84179507C8F0F999FECF11C08081C2
:10701000F999FECF31961FBA32BD21BD80BD0FB6A2
:10702000F894FA9AF99A0FBE2F5F3F4F41505040A3
:107030004115510561F78FEF089580E008954F9253
:107040005F926F927F928F929F92AF92BF92CF92F8
:10705000DF92EF92FF920F931F93DF93CF930F92E4
:10706000CDB7DEB76C015B01442E522E4801198268
:10707000FC0100811181C8016CE673E042E050E040
:107080000E9459F0009779F50E5F1F4FF6011183AA
:10709000008380E090E0B701A6010E94A0F03C01CF
:1070A00000E010E0C52CDD24E42CFF2418C0C5014D
:1070B0000E94C6EFAC01C301B5010E94CFEF892B3E
:1070C00051F4080D191DCE010196B80141E050E0C0
:1070D0000E94ABEF24C0AE0CBF1C0F5F1F4F0C15FE
:1070E0001D052CF31CC0F80180818D32C1F4C8014C
:1070F0000196F60191838083F8011181198301962D
:10710000F60191838083C4010E94C6EFAC01C401E3
:10711000612F70E00E949EEF892B09F4198289810A
:107120000F90CF91DF911F910F91FF90EF90DF9023
:10713000CF90BF90AF909F908F907F906F905F9017
:107140004F900895FF920F931F93CF93DF93982F43
:10715000F62E8150833010F090E053C080910701EB
:10716000C8E0D0E002C0CC0FDD1F9A95E2F79C2F5B
:107170000C2F009580238093070180910A018C2BAE
:1071800080930A01662331F080910B01982B909334
:107190000B0105C080910B01802380930B014423D8
:1071A00079F180E060E040E024E630E00E942A2EA1
:1071B00010E0FF2009F411E08091060120E090E04A
:1071C0008C239D23892B09F021E01217C9F480E05C
:1071D00060E040E024E630E00E942A2E8091060123
:1071E00020E090E08C239D23892B09F021E0912F52
:1071F000922739F480910B01082300930B0101C001
:1072000091E0892FDF91CF911F910F91FF90089509
:107210004FB7F8948091940090919500109295004A
:10722000109294004FBF08955FB7F8948091F118C1
:107230009091F2189093F0188093EF181092F21832
:107240001092F118A091C110B091C2104091BD18D8
:107250003091BE186BE67CE427C0CD01845C94417C
:10726000869FF001879FF00D969FF00D1124EE0F81
:10727000FF1FEE0FFF1FE154F74E90812181928393
:1072800023831182108291961D921D921D921C9251
:1072900094975C968C915C978F3311F4492F322F21
:1072A0001E960D90BC91A02D1097B9F64093BD1875
:1072B0003093BE185FBF8091EF189091F018089539
:1072C000CF93DF93EC010E940839AC018091E8175D
:1072D000882321F12FB7F8948091F1189091F2183A
:1072E000840F951F9093F2188093F118C45CD441D9
:1072F0008BE69CE4C89FF001C99FF00DD89FF00D6C
:107300001124EE0FFF1FEE0FFF1FE154F74E808197
:107310009181840F951F918380832FBFDF91CF913F
:10732000089582E090E00E94FC2D9FB7F89410929F
:10733000BE181092BD181092F0181092EF1810920B
:10734000F2181092F118EFEBF8E11182108213821B
:107350001282349688E1EF3EF807B9F71092BB101D
:107360001092BC101092BD101092BE101092C81155
:107370001092C9111092CA111092CB1181E0809322
:10738000E8179FBF08950F931F93CF93DF9304C017
:1073900089E190E00E94FC2D8091E8178823C1F3D9
:1073A0001AE00FEF112311F0115020C00E94143980
:1073B000C091EF18D091F0182097A9F06091BD18F6
:1073C0007091BE1880E090E02CE93FEF4FEF5FEF47
:1073D0000E94F2F39E0140E050E00E9446F42C59D6
:1073E0002093CE1102C00093CE111AE00E94F92E14
:1073F0000E9459218CE090E00E94FC2DD3CFCF92C7
:10740000DF92EF92FF920F931F93DF93CF930F9230
:10741000CDB7DEB7082FF62EE72E142FD22EA62FCB
:10742000B72FFD0101900020E9F73197CE2EC61A43
:10743000222339F40BC0802F60E240E050E00E942C
:10744000F3311150812F8F5FC816A8F3802F6F2D55
:107450007E2D40E050E09E012F5F3F4F0E94A23200
:10746000DD2041F009C0802F60E240E050E00E9442
:10747000F3311150C116B8F30F90CF91DF911F91E6
:107480000F91FF90EF90DF90CF9008952F923F9251
:107490004F925F926F927F928F929F92AF92BF9224
:1074A000CF92DF92EF92FF920F931F93DF93CF93D0
:1074B000CDB7DEB72C970FB6F894DEBF0FBECDBFA9
:1074C000B82E6FB7F894F090CE112090EF1830904E
:1074D000F0182091C1103091C210E7E9CE2EE6E0FD
:1074E000DE2E4BE65CE44BC02D5C3F4FF601318352
:1074F000208323533040F901848DF6018283F90102
:1075000084859585F60194838383F90181A192A1F5
:10751000A3A1B4A1F60185839683A783B087F9015F
:1075200086819781A085B185F60181879287A3879F
:10753000B487F90187A590A9A1A9B2A9F601858709
:107540009687A787B08BC901845C9441849FF00122
:10755000859FF00D949FF00D1124EE0FFF1FEE0F8D
:10756000FF1FE154F74E82819381F601928B818B4C
:10757000F9012685378583E190E0C80ED91E2115D3
:10758000310509F0B1CF6FBF8B2D6FE673E040E09E
:1075900050E08E010F5F1F4F98010E94A2326F2DA5
:1075A00070E080E090E022E0E22EF12CEC0EFD1E77
:1075B000A7012AE030E00E94DCF0BC018B2D40E006
:1075C00021E00E94FF398B2D6EE773E040E050E030
:1075D00098010E94A2328B2D6FE873E040E120E019
:1075E0000E94FF398B2D64E973E040E050E0980180
:1075F0000E94A232E7E9F6E0CE1ADF0A8BE19AECAC
:10760000C89E802D11246F0123E1829F4001112427
:107610008E0E9F1EAE2CEF2CF02E012F2101662422
:1076200077249DC0F601628170E080E090E04A2DF1
:107630005E2D2AE030E00E94DCF0BC018B2D44E09E
:1076400021E00E94FF39F6016381748180E090E0BF
:107650004A2D5E2D2AE030E00E94DCF0BC018B2D2B
:1076600047E021E00E94FF398B2D69EB73E040E099
:1076700050E02F2D302F0E94A232F60160817181DF
:107680008B2D40E120E00E94FF39F6016581768173
:10769000878190854A2D5E2D2AE030E00E94DCF043
:1076A000BC018B2D47E021E00E94FF3921143104F9
:1076B00051F48B2D6CEB73E040E050E02F2D302F18
:1076C0000E94A2321DC0F6016189728980E090E0BB
:1076D00024E630E040E050E00E94F2F3A301920182
:1076E0000E9446F4CA01B9014A2D5E2D2AE030E01D
:1076F0000E94DCF0BC018B2D48E021E00E94FF39A4
:10770000F60165857685878590894A2D5E2D2AE06C
:1077100030E00E94DCF0BC018B2D49E021E00E94AA
:10772000FF39F60161857285838594854A2D5E2D2A
:107730002AE030E00E94DCF0BC018B2D49E021E022
:107740000E94FF398B2D65EC73E040E050E02F2D57
:10775000302F0E94A23283E190E0C80ED91EC814D7
:10776000D90409F05FCF2C960FB6F894DEBF0FBE98
:10777000CDBFCF91DF911F910F91FF90EF90DF90E0
:10778000CF90BF90AF909F908F907F906F905F90C1
:107790004F903F902F90089549E228E130E00FB6D6
:1077A000F894A895209360000FBE4093600010925B
:1077B0007F071092800710928107109282076093D2
:1077C0007B0770937C0780937D0790937E070895D5
:1077D000EF92FF920F931F93EFB7F89420917F07DA
:1077E000309180074091810750918207262B372BDB
:1077F000482B592B20937F073093800740938107B4
:1078000050938207E0907F07F090800700918107F6
:1078100010918207EFBF80917B0790917C07A09128
:107820007D07B0917E0720917B0730917C074091C6
:107830007D0750917E078E219F21A023B1238217BF
:107840009307A407B50761F48FB7F89410927F07E8
:107850001092800710928107109282078FBFA8951F
:107860001F910F91FF90EF9008950895CF93DF93AC
:10787000EC01DB0120E030E012971DC0FE01E20FB9
:10788000F31F80814827842F82958427082E8695B0
:1078900086958025082E869580258770042E452F95
:1078A000869507948795502D4827069487955025EF
:1078B00048272F5F3F4F2A173B0700F3AC0FBD1F30
:1078C0008D919C914817590711F48FEF01C080E00A
:1078D000DF91CF910895DC0120E030E01DC0FD0173
:1078E000E20FF31F80814827842F82958427082E7A
:1078F000869586958025082E869580258770042E8E
:10790000452F869507948795502D4827069487958F
:10791000502548272F5F3F4F2617370700F3CA012E
:1079200008950F931F93DF93CF930F92CDB7DEB7D8
:107930008C018FEF8983D80112968C91813C08F0DD
:107940005BC0809151199091521960E070E0AE01D6
:107950004F5F5F4F0E94C2288091930790E026E31B
:1079600031E0829FF001839FF00D929FF00D112472
:10797000E35AF645D80112964C91129750E04E5EAC
:107980005F4F518340834251504083E090E09383A6
:10799000828313968C911397848714968C911497F5
:1079A00085875787468770966C9111967C91CF0199
:1079B00050E00E941CF080919307873020F48F5F85
:1079C0008093930702C01092930790919307809140
:1079D0009407981741F4973020F49F5F9093940791
:1079E00002C01092940780915119909152190E94EF
:1079F00036278FEF898301C0198289810F90CF913B
:107A0000DF911F910F9108951F93182F88E18093A4
:107A1000C1008093C9008093D1008093310107C0D9
:107A200080E060E040E024E630E00E942A2E809171
:107A30009EA18823A9F388E10FB6F8948093600093
:107A4000109260000FBEF8941230A9F0133021F1AB
:107A5000113099F58091C00087FF04C08091C60065
:107A60008093CE008091C80087FFF4CF8091CE0034
:107A70008093C600EFCF8091C00087FF04C0809143
:107A8000C6008093D6008091D00087FFF4CF80910C
:107A9000D6008093C600EFCF8091C00087FF04C05E
:107AA0008091C600809336018091300187FFF4CF2A
:107AB000809136018093C600EFCFFFCFAF92BF9287
:107AC000CF92DF92EF92FF920F931F93DF93CF93AA
:107AD0000F92CDB7DEB78C01D62EC72E19828091BA
:107AE00051199091521960E070E0AE014F5F5F4F05
:107AF0000E94C2288091950790E026E331E0829FA2
:107B00007001839FF00C929FF00C11248DE093EB99
:107B1000E80EF91E80E290E0D70113969C938E93B5
:107B2000129782E01C968C931C97F80184819581B2
:107B30001E969C938E931D978091E4039091E5038C
:107B400050969C938E931F972091E70383EFA82E66
:107B500088E1B82E2A3008F062C0AD2DBC2DFD01A1
:107B600001900020E9F7EA1BFB0B7D96D7011196E7
:107B7000FC93EE938DE351968C93AD2DBC2DFD01BE
:107B800001900020E9F73197EA1BFB0BD7015B96C8
:107B9000FC93EE935A9783E059968C935997589695
:107BA0001C928701045E1F4FED2DFC2DDF010D900F
:107BB0000020E9F71197AE1BBF0BC8016D2D7C2D7E
:107BC000AD010E941CF0ED2DFC2DDF010D90002079
:107BD000E9F71197AE1BBF0BC501B801AD010E94BB
:107BE0001CF0AD2DBC2DFD0101900020E9F731976F
:107BF000EA1BFB0BEA0DFB1D1082EDB7FEB73897B1
:107C00000FB6F894FEBF0FBEEDBF3196ADB7BEB74D
:107C10001296BC92AE92119783EB92E023C08DE155
:107C200090E0D70111969C938E9386E251968C93A7
:107C3000519781E090E059969C938E9358975A966D
:107C40002C93EDB7FEB738970FB6F894FEBF0FBE72
:107C5000EDBF3196ADB7BEB71296BC92AE921197FA
:107C600081E992E093838283D7011F968D919C9145
:107C70005097958384831D968D919C911E97978331
:107C800086830E9451F1EDB7FEB738960FB6F8948F
:107C9000FEBF0FBEEDBF80916E9D90916F9DA09134
:107CA000709DB091719DF701828B938BA48BB58BE6
:107CB000808191814A97978B868B8091950783303D
:107CC00020F48F5F8093950702C0109295079091E2
:107CD000950780919607981741F4933020F49F5FA1
:107CE0009093960702C01092960780915119909137
:107CF00052190E9436270F90CF91DF911F910F915B
:107D0000FF90EF90DF90CF90BF90AF900895CF920B
:107D1000DF92EF92FF920F931F93CF93DF936C014B
:107D20007B0160E270E04BE050E00E9425F0D7015B
:107D30000D900020E9F78D01015010400E191F0928
:107D400020E030E00AC0F701E20FF31F80818E329D
:107D500011F4E90107C02F5F3F4F201731079CF353
:107D6000CFEFDFEFC80101970C9710F080E022C041
:107D70001C161D06CCF4C601B701AE010E941CF012
:107D8000C017D107B4F4A601485F5F4FFE01E0952C
:107D9000F095E00FF11F9E012F5F3F4F2E0D3F1D0D
:107DA000CA01B901AF0103C0C601B701A8010E9411
:107DB0001CF08FEFDF91CF911F910F91FF90EF900B
:107DC000DF90CF900895CF93DF93AC01EB018DE06E
:107DD000FB0111928A95E9F7DB01FA0188E0019035
:107DE0000D928150E1F767E070E0FA01E60FF71FAE
:107DF0008081803239F09B012F5F3F4F12161306AE
:107E00004CF027C061507040FFEF6F3F7F0769F76C
:107E100080E020C0FE01E20FF31F8EE28083D901D3
:107E20001196AC0FBD1FFA01389683E001900D92B8
:107E30008150E1F7FE01E60FF71F20E030E084817A
:107E4000803209F414822F5F3F4F31972330310580
:107E5000B1F78FEFDF91CF91089586E5E7EFF8E86E
:107E6000DF011D928A95E9F71092F78808952F9205
:107E70003F924F925F926F927F928F929F92AF92BA
:107E8000BF92CF92DF92EF92FF920F931F93DF93F7
:107E9000CF93CDB7DEB760970FB6F894DEBF0FBEB5
:107EA000CDBFF82ECB01788B6F874A0163EA78EB60
:107EB000AE01415F5F4F0E94A0F0988B8F8700D08A
:107EC00000D0EDB7FEB7319603EF18E1ADB7BEB7FE
:107ED00012961C930E9311978EEF93E093838283F7
:107EE000F48215820E9451F1EDB7FEB73196ADB71D
:107EF000BEB712961C930E93119789EE93E093836D
:107F000082838F859889958384830E9451F1EDB790
:107F1000FEB736960FB6F894FEBF0FBEEDBFF4E481
:107F2000FF1609F4AFC2FF15B0F023E3F21659F1C2
:107F30002F1540F031E3F31649F162E3F61609F02C
:107F400001C326C082E4F81609F450C293E4F9167E
:107F500009F0F8C2F5C0A3E6FA1609F4F1C0AF15AE
:107F600048F0B9E4FB1609F4B0C2E2E6FE1609F0E7
:107F7000E9C23CC2F4E6FF1609F484C229E6F2160F
:107F800009F0E0C2A2C222E0D22E05C081E001C009
:107F900082E0D82EDA940F85188981E49BE10E9453
:107FA000C6EFAC01C80161E47BE10E94CFEF892BF1
:107FB00009F4A5C081EA9BE10E94C6EFAC01C801AB
:107FC00061EA7BE10E94CFEF892B19F496E0F92E4C
:107FD00097C082E19CE00E94C6EFAC01C80162E15B
:107FE0007CE00E94CFEF892B19F484E0F82E88C042
:107FF00088EE90E10E94C6EFAC01C80165E57DE026
:108000000E94CFEF892B19F403E0F02E79C084EDA4
:1080100091E10E94C6EFAC01C80164ED71E10E94DC
:10802000CFEF892B19F417E0F12E6AC088E59AE1A9
:108030000E94C6EFAC01C80168E57AE10E94CFEF6B
:10804000892B19F4B5E0FB2E5BC08AE399E00E940E
:10805000C6EFAC01C8016AE379E00E94CFEF892B3B
:1080600019F4A8E0FA2E4CC0C80164EE73E044E0B5
:1080700050E00E94CFEF892B19F4FF24F39440C005
:10808000C80160EE73E043E050E00E94CFEF892B1F
:1080900019F4F2E0FF2E34C0D8018C91805323EF05
:1080A00038E18A30B0F400D00F92EDB7FEB73283DA
:1080B000218386ED93E0948383830E9451F10F9096
:1080C0000F900F900F908F8598890E9459EFF82E8E
:1080D00017C000D00F92ADB7BEB712963C932E9347
:1080E00011978BEC93E014969C938E9313970E94B8
:1080F00051F180E00F900F900F900F9024C2FF2459
:10810000EE24EA94E9820D2D10E00F5E1F4F680106
:10811000E4E0CC0CDD1CEA95E1F701511040C6010A
:10812000BE016F5F7F4F0E9438378981F81611F1C9
:108130000E561E45F801E082C6016F2D0E949F3742
:1081400070E1C72E71E0D72E61E0E62EF12C5AEFD8
:10815000A52E58EBB52E8E010B5F1F4F48EA242E3B
:1081600043E0342E33E0432E512C2FE9622E23E0DE
:10817000722E29C02DB73EB7285030400FB6F89464
:108180003EBF0FBE2DBFEDB7FEB7319683EF98E12E
:10819000ADB7BEB712969C938E93119781EB93E087
:1081A000938382830F5F1F4F15830483F6821782A8
:1081B0000E9451F1EDB7FEB738960FB6F894FEBFA6
:1081C0000FBEEDBFBDCFC601BE016C5F7F4F0E94E9
:1081D0003837D501E4E11D92EA95E9F7D801EAE0E4
:1081E0001D92EA95E9F78C81843009F463C08530EB
:1081F00050F48130F1F0813098F08230C1F1833059
:1082000009F086C04EC0863009F466C0863008F496
:108210005AC0873009F469C0883009F079C06EC04F
:1082200081E49BE10E94C6EFAC01C80161E47BE1FF
:108230006DC000D000D0EDB7FEB73196ADB7BEB778
:1082400012961C930E9311972CEA33E0338322830A
:1082500088E090E0958384830E9451F1ADB7BEB76A
:1082600016960FB6F894BEBF0FBEADBF51C000D07A
:1082700000D0EDB7FEB73196ADB7BEB712961C93DE
:108280000E93119733822282558244820E9451F1CB
:10829000EDB7FEB736960FB6F894FEBF0FBEEDBF32
:1082A00037C085E59DE00E94C6EFAC01C80165E5D9
:1082B0007DE02CC082E19CE00E94C6EFAC01C801C9
:1082C00062E17CE023C088E59AE10E94C6EFAC0140
:1082D000C80168E57AE11AC081EA9BE10E94C6EF15
:1082E000AC01C80161EA7BE111C084ED91E10E941B
:1082F000C6EFAC01C80164ED71E108C08AE399E002
:108300000E94C6EFAC01C8016AE379E00E94ABEFBE
:108310002DB73EB7285030400FB6F8943EBF0FBE81
:108320002DBFEDB7FEB73196ADB7BEB71296BC9272
:10833000AE92119773826282F582E482178306837C
:108340000E9451F1EDB7FEB738960FB6F894FEBF14
:108350000FBEEDBFC401B5010E942CF020E130E05A
:10836000C20ED31E0894E11CF11C30E4C31631E0A8
:10837000D30609F028CF82E091E0BE016E5F7F4F07
:108380000E94383700D000D0EDB7FEB73196ADB7B8
:10839000BEB71296BC92AE92119781E893E0938398
:1083A00082838A81848315820E9451F1EDB7FEB7E2
:1083B00036960FB6F894FEBF0FBEEDBFC401B501EF
:1083C0000E942CF000D000D0EDB7FEB7319683EFBD
:1083D00098E1ADB7BEB712969C938E93119780E744
:1083E00093E0938382839582848240C08F859889AD
:1083F00060E070E040E050E00E942AEE9B01AC019A
:10840000DC01CB0180509140A040B04080509E4F95
:10841000A040B04040F4222331F4232F342F452FC5
:10842000552747FD5A95DA01C9010197A109B109FC
:108430008E3F9105A105B10508F084C02B8381E032
:1084400091E0622F0E949F3700D000D0EDB7FEB7B9
:108450003196ADB7BEB712969C928E9211978FE36C
:1084600093E0938382838B81848315820E9451F1F0
:108470008FEFEDB7FEB736960FB6F894FEBF0FBE7E
:10848000EDBF61C0EF85F8898081882309F45AC067
:10849000CF010E9459EF682F8F3F09F453C08A83A0
:1084A00082E091E00E949F3700D000D0EDB7FEB788
:1084B0003196ADB7BEB712969C928E92119786E117
:1084C00093E0938382838A81CFCF81E091E0BE01E4
:1084D0006D5F7F4F0E94383782E091E0BE016E5F92
:1084E0007F4F0E9438372DB73EB72E5030400FB621
:1084F000F8943EBF0FBE2DBFEDB7FEB73196ADB7B6
:10850000BEB712969C928E92119785ED92E093835E
:10851000828382E090E09583848381E090E097837A
:1085200086838BE891E0918780878B818287138691
:108530008A81848715860E9451F18FEFEDB7FEB7CF
:108540003E969ACF80E060960FB6F894DEBF0FBEDD
:10855000CDBFCF91DF911F910F91FF90EF90DF90F2
:10856000CF90BF90AF909F908F907F906F905F90D3
:108570004F903F902F900895CF92DF92EF92FF920D
:108580000F931F93DF93CF930F920F92CDB7DEB768
:108590006C0122E73DE93A83298300D000D0EDB792
:1085A000FEB7319683EF98E1ADB7BEB712969C93B4
:1085B0008E93119782E394E093838283358324839F
:1085C0000E9451F1E981FA81E150FF4F108233EAB4
:1085D000E32E38EBF32E87E0F70111928A95E9F745
:1085E0002DB73EB72A5F3F4F0FB6F8943EBF0FBE80
:1085F0002DBFC7016FE372E00E94B4EF89819A81B9
:10860000B7018E010F5F1F4FA8010E94A0F00097D5
:1086100021F420E090E011E01CC06EE274E043E041
:1086200050E00E94CFEF892B21F020E090E012E093
:1086300010C0C80166E472E048E027E00EE712E0EF
:108640000E941F38282F882311F09FEF01C090E06F
:1086500013E0EAEAF8EB80E5DF011D928A95E9F77D
:108660009F3F51F469817A81822FAF010E94373F89
:10867000182F8F3F79F11DC000D000D0EDB7FEB7A5
:10868000319683EF98E1ADB7BEB712969C938E9367
:1086900011978FE094E093838283148315820E9464
:1086A00051F1EDB7FEB736960FB6F894FEBF0FBE88
:1086B000EDBF113039F0113058F0123029F013307D
:1086C00039F404C08DE007C08EE005C08AE003C025
:1086D0008FE001C081E08093E703C6016AEA78EB8E
:1086E0000E945E3D80E091E0E2E7FDE9DF019C0150
:1086F0001D9221503040E1F710926A9D1092699DC1
:1087000010926B9D10926D9D10926C9D10926E9DBB
:1087100010926F9D1092709D1092719D0F900F900E
:10872000CF91DF911F910F91FF90EF90DF90CF904D
:1087300008954F925F926F927F928F929F92AF9225
:10874000BF92CF92DF92EF92FF920F931F93DF932E
:10875000CF930F920F92CDB7DEB77C01A62E3A01D0
:108760004C010894811C911C198243E0C42ED12C29
:108770001A8200E010E0BB242E010894411C511C19
:108780008A2DB301A2010E94B832982F89818823D3
:1087900019F000E010E03EC08A818F3F69F59D37F7
:1087A00019F4BB24BA9412C0BB2059F0EFEFBE16E7
:1087B00069F49062F70191937F010F5F1F4FBB2413
:1087C00005C0F70191937F010F5F1F4F0330110523
:1087D00061F4F401C080D180F0E3CF16F2E0DF064F
:1087E00020F0CC24DD2420E001C02FEFC60101964B
:1087F0000817190778F40BC09E3711F6F70191930B
:108800007F010F5F1F4FFFEFFA83BB24B9CF2F3FCC
:1088100009F4B6CFC8010F900F90CF91DF911F914F
:108820000F91FF90EF90DF90CF90BF90AF909F900F
:108830008F907F906F905F904F9008956F927F928E
:108840008F929F92BF92CF92DF92EF92FF920F93FF
:108850001F93DF93CF930F920F92CDB7DEB77C01BA
:108860004C010894811C911C198253E0C52ED12C17
:108870001A8200E010E0BB243E010894611C711CC8
:1088800080E060E070E0A3010E94B8329A819F3FCF
:1088900069F58D3719F4BB24BA9412C0BB2059F086
:1088A000EFEFBE1669F48062F70181937F010F5FDD
:1088B0001F4FBB2405C0F70181937F010F5F1F4F3E
:1088C0000330110561F4F401C080D180F0E3CF16CC
:1088D000F2E0DF0620F0CC24DD2420E001C02FEF01
:1088E000C60101960817190778F40BC08E3741F6B8
:1088F000F70181937F010F5F1F4FFFEFFA83BB24C6
:10890000BFCF2F3F09F4BCCFC8010F900F90CF917C
:10891000DF911F910F91FF90EF90DF90CF90BF906C
:108920009F908F907F906F9008958F929F92AF92BB
:10893000BF92CF92DF92EF92FF920F931F93CF934C
:10894000DF93EC015B01D42E7901CB0101978F52AB
:10895000924008F051C0842F63E00E947A318D2C40
:108960009924F401EA56F7448081823099F41AE0A0
:1089700005C08D2D60E0A7010E94F3311150C8F7AA
:108980008D2D65E5A7010E94F3318D2D6AEAA701BF
:108990000E94F3318D2D6EE7A7010E94F3318823E9
:1089A00029F0AA24BB24CC24CA9429C0CC2427C0F3
:1089B0006881862F8D57823060F48D2D6DE7A70179
:1089C0000E94F331982F88818F7D8883F8019082EF
:1089D00011C08D2DA7010E94F331982FF8018081DD
:1089E000882321F0888180628883108221960894F0
:1089F000A108B108992341F0CC24CA9408C084018D
:108A00000456184F99249A94A114B10489F68C2D18
:108A1000DF91CF911F910F91FF90EF90DF90CF905A
:108A2000BF90AF909F908F9008955F926F927F92CA
:108A30008F929F92AF92BF92CF92DF92EF92FF926E
:108A40000F931F93CF93DF937C01FEEFCF2EF4EAB9
:108A5000DF2E10929807C1E0D0E03601089461083B
:108A60007108E0E38E2EE2E09E2E7AE2572E6AE253
:108A7000A62EB12CFE01EA56F74480818150823047
:108A800008F087C010E00C2FF301C4011192019788
:108A9000E9F7F70160817181C701402F20E030E0E4
:108AA0000E949544882309F070C08DEF94EA602FEE
:108AB00040E450E00E949943892B09F466C08091FC
:108AC000FEA49091FFA4EEEFF4EA20E030E0DC0198
:108AD0001297AC0144505B4518C081912827822F22
:108AE00082958227082E869586958025082E869564
:108AF00080258770022E232F869507948795302D29
:108B000028270694879530252827E417F50729F7A5
:108B1000A250BB458D919C9128173907B1F530E0E3
:108B200029C0259DD0011124359DF0011124A251A9
:108B3000B844E25FFA458AE201900D928150E1F774
:108B400020919807822F90E08A9DF0018B9DF00D77
:108B50009A9DF00D1124E251F84404873F5F2F5F86
:108B60002093980780910AA590910BA50197F60193
:108B70009587848720919807243058F480910AA51E
:108B800090910BA5892B69F604C01F5F123009F084
:108B90007BCF2196C430D10509F06CCFDF91CF9106
:108BA0001F910F91FF90EF90DF90CF90BF90AF900B
:108BB0009F908F907F906F905F9008950F931F9379
:108BC000CF93DF938C01C1E0D0E0FE01EA56F74479
:108BD00080818150823048F4F80160817181C80140
:108BE0004C2F2AE030E00E9495442196C430D105F4
:108BF00061F7DF91CF911F910F910895FF920F932D
:108C00001F93CF93DF93EC018B01CB0101978F5220
:108C1000924070F580E06EE740E050E00E94F33152
:108C2000FF24FA9422C06881862F8D57823060F429
:108C300080E06DE740E050E00E94F33188818F7D55
:108C40008883F092A00711C080E040E050E00E94CD
:108C5000F3318091A007882329F08881806288837E
:108C60001092A00721960150104001151105D9F668
:108C7000DF91CF911F910F91FF900895EF92FF9296
:108C80000F931F93CF93DF93EC01EA80FB8000D01A
:108C90000F9203EF18E1ADB7BEB712961C930E9377
:108CA000119782EC94E014969C938E9313970E94F4
:108CB00051F10F900F900F900F908A8D9B8D8F3FE9
:108CC000910509F008F4A1C100D00F92EDB7FEB7ED
:108CD0001283018381EB94E0948383830E9451F19A
:108CE0001EE115C0F3E0FE1508F073C000D00F922E
:108CF000ADB7BEB712961C930E9311978DE994E011
:108D000014969C938E9313970E9451F11FE10F903C
:108D10000F900F900F9000D00F9283EF98E1ADB7B6
:108D2000BEB712969C938E9311978DE594E014969E
:108D30009C938E9313970E9451F18C819D81909307
:108D4000E1888093E0888A819B819093E388809377
:108D5000E2888E819F819093E5888093E48889E101
:108D600090E09093DF888093DE8884E090E0909399
:108D7000E7888093E688888599859093E988809331
:108D8000E8881092EA888E859F85A889B9898093A2
:108D9000EC889093ED88A093EE88B093EF8883E001
:108DA00090E09093F1888093F08886E28093EB883E
:108DB00081E090E09093F3888093F2881093F48898
:108DC000E0E0F8E820E030E00F900F900F900F9077
:108DD000F4C04E2D50E08A0103571E45F8018081F2
:108DE0008F3FA1F400D00F9283EF98E1ADB7BEB7EB
:108DF00012969C938E9311978BE894E014969C9313
:108E00008E9313970E9451F111E181CF89E091E097
:108E1000489F9001499F300D589F300D1124F90152
:108E2000E759F2468C819D8191838083898D82836D
:108E30008A8D9B8D948383838E859F85A889B9892C
:108E400085839683A783B0872E58324680E091E0D1
:108E5000F901AC01119241505040E1F7FE017C96BE
:108E60004A8D5B8DC901BF010E941CF08FEFD801B4
:108E70008C938C819D8190930388809302888A8152
:108E80009B8190930588809304888E819F81909325
:108E900007888093068885E190E09093018880930D
:108EA000008881E090E09093098880930888888505
:108EB000998590930B8880930A888E859F85A889D1
:108EC000B98980930D8890930E88A0930F88B093F2
:108ED0001088109212881092118883E180930C8878
:108EE000E0E0F8E820E030E018C081912827822FE8
:108EF00082958227082E869586958025082E869550
:108F000080258770022E232F869507948795302D14
:108F100028270694879530252827B8E8E331FB07F2
:108F200021F731832083CF01439765E170E00E94F0
:108F3000FE45EDB7FEB738970FB6F894FEBF0FBEEB
:108F4000EDBF319683EF98E1ADB7BEB712969C9313
:108F50008E93119789E694E09383828380910288AF
:108F600090910388958384838091048890910588EB
:108F7000978386830E9451F1EDB7FEB738960FB6FE
:108F8000F894FEBF0FBEEDBF38C081912827822F15
:108F900082958227082E869586958025082E8695AF
:108FA00080258770022E232F869507948795302D74
:108FB00028270694879530252827B8E8E731FB074E
:108FC00021F73093F6882093F58877976081718137
:108FD000CF010E94FE4500D00F9283EF98E1EDB7DC
:108FE000FEB79283818381E594E0948383830E941A
:108FF00051F10F900F900F900F90EE2061F4CE0181
:109000000E94BC4210928DA106C08091E6038F158C
:1090100009F068CEDECEDF91CF911F910F91FF90C6
:10902000EF9008951F93CF93DF93EC018A858130F1
:10903000B9F58B859C850197B9F58D858A30A1F5A9
:109040008C89803189F58D899E898550904961F59B
:10905000388D5F899A8D80E0298D820F911D01974F
:1090600029F5FE017B964B8D433000F5932F80E070
:109070009C01250F311D8091E4039091E503281791
:109080003907A1F4858196818217930779F480E0EE
:10909000413009F481E00E943CEB4FEF1FEF08C024
:1090A000882311F44FEF03C041E001C042E010E01B
:1090B0002885398537FD67C08091E4039091E503E9
:1090C000909332A7809331A78C819D81909330A794
:1090D00080932FA78E819F81909334A7809333A78D
:1090E000109236A7109235A74F3F31F481E090E0FF
:1090F000909336A7809335A787E397EA4F3F39F4DB
:10910000309338A7209337A7DC01129608C030931C
:1091100038A7209337A7409339A7DC011396CD01D8
:109120008B52974A90932EA780932DA7EDE2F7EAF2
:1091300020E030E0AC01455D584518C081912827FA
:10914000822F82958227082E869586958025082E67
:10915000869580258770022E232F86950794879504
:10916000302D28270694879530252827E417F50702
:1091700029F72D933C9360912DA770912EA78DE236
:1091800097EA0E94FE45112319F08FEF0E9458EBD9
:10919000DF91CF911F910895BF92CF92DF92EF920E
:1091A000FF920F931F93DF93CF93CDB7DEB72D9729
:1091B0000FB6F894DEBF0FBECDBF8C01FE01319615
:1091C0008DE0DF011D928A95E9F7D8011296BC90D7
:1091D00012979496CD90DD90ED90FC909797BFEF0D
:1091E000CB16BFEFDB06BFEFEB06BFEFFB0611F0C0
:1091F000898105C0C8014996BF010E94E33E8823CA
:1092000009F0A0C0F801848195819093E188809352
:10921000E088828193819093E3888093E2888681BD
:1092200097819093E5888093E48889E190E090931A
:10923000DF888093DE8884E090E09093E7888093D5
:10924000E688808591859093E9888093E8881092DC
:10925000EA8886859785A089B1898093EC88909368
:10926000ED88A093EE88B093EF8883E090E0909330
:10927000F1888093F08884E28093EB8881E090E02D
:109280009093F3888093F28885E08093F488E0E0FF
:10929000F8E820E030E038C081912827822F8295BD
:1092A0008227082E869586958025082E869580250E
:1092B0008770022E232F869507948795302D2827B7
:1092C000069487953025282788E8EE32F80721F79D
:1092D00031832083BE9721C081912827822F8295D8
:1092E0008227082E869586958025082E86958025CE
:1092F0008770022E232F869507948795302D282777
:109300000694879530252827A8E8E731FA0721F742
:109310003093F6882093F588779760817181CF012B
:109320000E94FE452D960FB6F894DEBF0FBECDBF4E
:10933000CF91DF911F910F91FF90EF90DF90CF9031
:10934000BF900895EB2DF0E0EE0FFF1FEF5AF246AD
:109350002081318140E050E0F80184819581909333
:1093600003888093028882819381909305888093FB
:10937000048886819781909307888093068880E38C
:1093800090E0909301888093008861E070E0709392
:109390000988609308888085918590930B888093D5
:1093A0000A8886859785A089B18980930D889093D6
:1093B0000E88A0930F88B09310888BE190E0909373
:1093C00012888093118881E380930C888FEF8093BB
:1093D00017887093198860931888109216881092D5
:1093E00015888789908D90931488809313881092A4
:1093F0002D88C0922588D0922688E0922788F09206
:1094000028882093298830932A8840932B8850936A
:109410002C888AE198E8BE016F5F7F4F0E94873EEB
:10942000E0E0F8E820E030E04FCFCF92DF92FF920B
:109430000F931F93DF93CF93CDB7DEB72D970FB662
:10944000F894DEBF0FBECDBF8C016E010894C11C25
:10945000D11C8DE0F60111928A95E9F7F801F280AE
:10946000C8014996B6010E94E33EF8016481758106
:10947000A681B781882309F099C07093E188609331
:10948000E088828193819093E3888093E288B0930F
:10949000E588A093E48889E190E09093DF88809349
:1094A000DE8884E090E09093E7888093E68880856A
:1094B00091859093E9888093E8881092EA88868560
:1094C0009785A089B1898093EC889093ED88A093CB
:1094D000EE88B093EF8883E090E09093F1888093DA
:1094E000F08884E28093EB8881E090E09093F388A9
:1094F0008093F28885E08093F488E0E0F8E820E04B
:1095000030E038C081912827822F82958227082E4B
:10951000869586958025082E869580258770022E53
:10952000232F869507948795302D282706948795B5
:109530003025282788E8EE32F80721F73183208389
:10954000BE9721C081912827822F82958227082EDD
:10955000869586958025082E869580258770022E13
:10956000232F869507948795302D28270694879575
:109570003025282788E8E731F80721F73093F68867
:109580002093F588779760817181CF010E94FE4515
:109590002D960FB6F894DEBF0FBECDBFCF91DF91F1
:1095A0001F910F91FF90DF90CF900895EF2DF0E085
:1095B000EE0FFF1FEF5AF2462081318140E050E06C
:1095C0007093038860930288F8018281938190935D
:1095D000058880930488B0930788A093068880E369
:1095E00090E0909301888093008861E070E0709330
:1095F0000988609308888085918590930B88809373
:109600000A8886859785A089B18980930D88909373
:109610000E88A0930F88B09310888BE190E0909310
:1096200012888093118881E380930C888FEF809358
:109630001788709319886093188810921688109272
:1096400015888789908D9093148880931388109241
:109650002D888FEF9FEFAFEFBFEF8093258890931A
:109660002688A0932788B093288820932988309350
:109670002A8840932B8850932C888AE198E8B60179
:109680000E94873EE0E0F8E820E030E053CF4F92C0
:109690005F926F927F929F92AF92BF92CF92DF9232
:1096A000EF92FF920F931F93DF93CF93CDB7DEB767
:1096B0002D970FB6F894DEBF0FBECDBF7C01FE0123
:1096C00031968DE0DF011D928A95E9F7D701129658
:1096D0009C90129713960C91C7014996BF010E9466
:1096E000E33E882321F410E065E070E00CC0809137
:1096F000E603801709F456C1B3E0B91508F052C16A
:1097000010E06AE070E0CC24DD240AC06901D7FCD7
:1097100004C01FEF60E070E003C010E065E070E09F
:10972000E92DF0E09601442737FD4095542FD701ED
:1097300098964D905D906D907C909B97240D351D73
:10974000461D571DEE0FFF1FEF5AF2468081918193
:10975000A0E0B0E0281739074A075B0710F0118234
:1097600010826115710509F098C01F3F09F095C07E
:10977000F701848195819093038880930288828188
:109780009381909305888093048886819781909334
:109790000788809306888EED90E0909301888093EF
:1097A000008881E090E09093098880930888808504
:1097B000918590930B8880930A8886859785A089E8
:1097C000B18980930D8890930E88A0930F88B093F1
:1097D000108889EC90E090931288809311888BE137
:1097E00080930C882AE1A22E28E8B22EC0921A8813
:1097F000D0921B8880A591A5A2A5B3A580931588BA
:1098000090931688A0931788B0931888A5014E5F8F
:109810005F4F992D990F990F80E020A531A5280F52
:10982000391F2F5A3247CA01B901A6010E941CF004
:1098300010931988D70157968D919C9158979093C2
:10984000148880931388F5017A9720E030E018C0DF
:1098500081912827822F82958227082E86958695CA
:109860008025082E869580258770022E232F8695C9
:1098700007948795302D282706948795302528272B
:10988000B8E8EC3DFB0721F7318320836091008825
:109890007091018880E098E86DC0F701848195811E
:1098A0009093E1888093E088828193819093E3880C
:1098B0008093E288868197819093E5888093E488FD
:1098C00089E190E09093DF888093DE8884E090E0E7
:1098D0009093E7888093E688808591859093E988C6
:1098E0008093E8881092EA8886859785A089B18957
:1098F0008093EC889093ED88A093EE88B093EF88E6
:1099000083E090E09093F1888093F08884E28093E4
:10991000EB8881E090E09093F3888093F2886093E5
:10992000F488E0E0F8E820E030E018C081912827D2
:10993000822F82958227082E869586958025082E6F
:10994000869580258770022E232F8695079487950C
:10995000302D2827069487953025282788E8E73179
:10996000F80721F73093F6882093F5887797608180
:109970007181CF010E94FE452D960FB6F894DEBF8F
:109980000FBECDBFCF91DF911F910F91FF90EF9050
:10999000DF90CF90BF90AF909F907F906F905F903F
:1099A0004F900895E92DF0E0EE0FFF1FEF5AF246B9
:1099B000C080D180D70198968D919C919997C81AB3
:1099C000D90A9C962D913D914D915C919F97C6012E
:1099D000AA2797FDA095BA2F281739074A075B07D2
:1099E00008F494CE94CE0F931F93DF93CF93CDB70B
:1099F000DEB72D970FB6F894DEBF0FBECDBF8C013A
:109A0000FE0131968DE0DF011D928A95E9F7D801BC
:109A100094962D913D914D915C9197972F5F3F4F7B
:109A20004F4F5F4F11F0898105C0C8014996BF01B2
:109A30000E94E33E882309F09EC0F801848195814D
:109A40009093E1888093E088828193819093E3886A
:109A50008093E288868197819093E5888093E4885B
:109A600089E190E09093DF888093DE8884E090E045
:109A70009093E7888093E688808591859093E98824
:109A80008093E8881092EA8886859785A089B189B5
:109A90008093EC889093ED88A093EE88B093EF8844
:109AA00083E090E09093F1888093F08884E2809343
:109AB000EB8881E090E09093F3888093F28885E0D2
:109AC0008093F488E0E0F8E820E030E03BC081914A
:109AD0002827822F82958227082E869586958025B5
:109AE000082E869580258770022E232F8695079451
:109AF0008795302D2827069487953025282788E8D4
:109B0000E331F80721F731832083CF01439765E1E3
:109B100070E024C081912827822F82958227082E09
:109B2000869586958025082E869580258770022E3D
:109B3000232F869507948795302D2827069487959F
:109B400030252827A8E8E731FA0721F73093F6886F
:109B50002093F588779760817181CF010E94FE453F
:109B60002D960FB6F894DEBF0FBECDBFCF91DF911B
:109B70001F910F910895F801848195819093038836
:109B800080930288828193819093058880930488D2
:109B900086819781909307888093068885E190E07D
:109BA000909301888093008881E090E090930988E9
:109BB000809308888085918590930B8880930A888C
:109BC00086859785A089B18980930D8890930E88AA
:109BD000A0930F88B0931088109212881092118869
:109BE00083E180930C88E0E0F8E820E030E087CF64
:109BF0007F928F929F92AF92BF92CF92DF92EF921D
:109C0000FF920F931F93DF93CF93CDB7DEB72D97BE
:109C10000FB6F894DEBF0FBECDBF6C01FE013196CA
:109C20008DE0DF011D928A95E9F7D60112967C90AE
:109C3000129713962C91139759968D909D90AD90F5
:109C4000BC905C978091F7888130B1F48091238932
:109C500090912489A0912589B0912689881699062A
:109C6000AA06BB0649F4DF01E8EFF8E88DE00190B1
:109C70000D928150E1F701C019828981882319F47E
:109C800025E030E0CCC08091E603821721F0B3E0FC
:109C9000B71508F4C2C0D6019196ED91FC91929748
:109CA0007F010027F7FC0095102F5D964D915D9187
:109CB0006D917C919097D801C701840F951FA61FC5
:109CC000B71F81509140A040B04018F025E030E02F
:109CD00010C0372D20E0240F351F2F5A3647A6011C
:109CE0004D5D5F4FC901BA01AF010E941CF020E039
:109CF00030E0F601858D968DA78DB0A1E80EF91E96
:109D00000A1F1B1F8091278990912889A09129897A
:109D1000B0912A89E816F9060A071B07D0F086E5F4
:109D2000E7EFF8E8DF011D928A95E9F71092F788CE
:109D3000A72DB0E0FD01EE0FFF1FEE0FFF1FED5747
:109D4000F84F80829182A282B382AF59B2468FEFE0
:109D50008C932115310509F062C0F601848195814B
:109D600090930388809302888281938190930588E1
:109D700080930488868197819093078880930688D2
:109D800085E190E0909301888093008881E090E0E5
:109D900090930988809308888085918590930B889B
:109DA00080930A8886859785A089B18980930D88DC
:109DB00090930E88A0930F88B09310881092128809
:109DC0001092118883E180930C88E0E0F8E820E0AD
:109DD00030E018C081912827822F82958227082E93
:109DE000869586958025082E869580258770022E7B
:109DF000232F869507948795302D282706948795DD
:109E00003025282788E8E331F80721F731832083BC
:109E1000CF01439765E170E080C02AE030E086E53D
:109E2000E7EFF8E8DF011D928A95E9F7E72DF0E00A
:109E3000EE0FFF1FE75AF246118210821092F78848
:109E4000F601848195819093E1888093E0888281F6
:109E500093819093E3888093E288868197819093A1
:109E6000E5888093E48889E190E09093DF8880938F
:109E7000DE8884E090E09093E7888093E688808590
:109E800091859093E9888093E8881092EA88868586
:109E90009785A089B1898093EC889093ED88A093F1
:109EA000EE88B093EF8883E090E09093F188809300
:109EB000F08884E28093EB8881E090E09093F388CF
:109EC0008093F2882093F488E0E0F8E820E030E026
:109ED00018C081912827822F82958227082E869587
:109EE00086958025082E869580258770022E232F43
:109EF000869507948795302D2827069487953025D9
:109F0000282788E8E731F80721F73093F68820936F
:109F1000F588779760817181CF010E94FE452D966B
:109F20000FB6F894DEBF0FBECDBFCF91DF911F916A
:109F30000F91FF90EF90DF90CF90BF90AF909F90E8
:109F40008F907F900895BF92CF92DF92EF92FF9211
:109F50000F931F93DF93CF93CDB7DEB72D970FB637
:109F6000F894DEBF0FBECDBF8C01FE0131968DE0AF
:109F7000DF011D928A95E9F7D8011296BC901297DD
:109F80001396FC9039E1C32ED12CC00ED11ED60100
:109F90008BE00D9001928150E1F7FE0131968DE04A
:109FA000DF011D928A95E9F78091F788882309F0EF
:109FB000ABC1C601BF010E94E33E882309F095C1F1
:109FC00025E030E002C18091E6038F1521F0B3E077
:109FD000BB1508F4F8C0EB2CFF24F701E35BF64750
:109FE0008081882309F4EFC0F701EE0FFF1FEF5ABD
:109FF000F24680819181892B09F086C1A5E0B9E8FC
:10A00000FE0131968DE001900D928150E1F7F8014B
:10A0100082AD93AD90933A8980933989ABE3B9E8E7
:10A02000FC9680E101900D928150E1F7ABE2B9E836
:10A03000F801BC9686E001900D928150E1F7A1E312
:10A04000B9E8F801F29686E001900D928150E1F7AF
:10A05000D801D8968C91D8978093378994968D9112
:10A060009D910D90BC91A02D80932389909324897C
:10A07000A0932589B0932689A8E1B9E8F6018BE081
:10A0800001900D928150E1F7C60168EF78E80E94D7
:10A09000E33EF80180A591A5A2A5B3A580932789E9
:10A0A00090932889A0932989B0932A8981E080938D
:10A0B000F78881AD882319F428E030E086C09B2D15
:10A0C00080E08F5A9647FC0180E091E0DF019C011F
:10A0D0001D9221503040E1F7EE0CFF1C89E59DE90F
:10A0E000E80EF91ED80198968D919C919997F701E9
:10A0F0009183808314968D919C91159790930388FA
:10A100008093028812968D919C9113979093058865
:10A110008093048816968D919C9117979093078849
:10A120008093068885E190E0909301888093008871
:10A1300081E090E0909309888093088818968D912B
:10A140009C91199790930B8880930A881E968D9105
:10A150009D910D90BC91A02D80930D8890930E88B9
:10A16000A0930F88B09310881092128810921188D3
:10A1700083E180930C88E0E0F8E820E030E018C04C
:10A1800081912827822F82958227082E8695869591
:10A190008025082E869580258770022E232F869590
:10A1A00007948795302D28270694879530252827F2
:10A1B00088E8E331F80721F731832083CF01439703
:10A1C00065E170E080C02AE030E086E5E7EFF8E87E
:10A1D000DF011D928A95E9F7EB2DF0E0EE0FFF1FEE
:10A1E000E75AF246118210821092F788F8018481B2
:10A1F00095819093E1888093E08882819381909308
:10A20000E3888093E288868197819093E5888093A4
:10A21000E48889E190E09093DF888093DE8884E091
:10A2200090E09093E7888093E6888085918590936D
:10A23000E9888093E8881092EA8886859785A089C6
:10A24000B1898093EC889093ED88A093EE88B093C9
:10A25000EF8883E090E09093F1888093F08884E227
:10A260008093EB8881E090E09093F3888093F2886C
:10A270002093F488E0E0F8E820E030E018C0819115
:10A280002827822F82958227082E869586958025FD
:10A29000082E869580258770022E232F8695079499
:10A2A0008795302D2827069487953025282788E81C
:10A2B000E731F80721F73093F6882093F5887797F0
:10A2C00060817181CF010E94FE452D960FB6F894F2
:10A2D000DEBF0FBECDBFCF91DF911F910F91FF90D9
:10A2E000EF90DF90CF90BF900895F80180A591A5E1
:10A2F000A2A5B3A58F3F9105A105B10509F008F40A
:10A3000062CE2DE030E061CF21E130E05ECFFC0194
:10A310008589968920E98430920709F43DC020E9B7
:10A3200085309207A0F420E98130920729F120E9D5
:10A330008230920720F480509049C9F519C020E975
:10A3400082309207E9F08350904989F51DC020E9D9
:10A3500088309207E9F020E98930920720F485508F
:10A36000904929F51DC080509149029700F51CC005
:10A37000CF010E94A34F0895CF010E94F84D089588
:10A38000CF010E94F34C0895CF010E94474B0895DE
:10A39000CF010E94154A0895CF010E94CC4808952C
:10A3A000CF010E9412480895CF010E943E460895B1
:10A3B000FC0188E190E09093A2A28093A1A2848105
:10A3C00095819093A4A28093A3A24091E40350911D
:10A3D000E5035093A6A24093A5A28681978190930E
:10A3E000A8A28093A7A221E030E03093AAA22093F4
:10A3F000A9A2808591859093ACA28093ABA2309363
:10A40000AEA22093ADA23093B0A22093AFA25093FE
:10A41000B2A24093B1A28091E6038093B3A291E0EF
:10A420009093B4A2809143198093B5A29093B6A261
:10A43000E1EAF2EA20E030E018C081912827822F7B
:10A4400082958227082E869586958025082E8695EA
:10A4500080258770022E232F869507948795302DAF
:10A460002827069487953025282782EAE73BF807B6
:10A4700021F731832083CF01469768E170E00E9485
:10A48000FE450895AF92BF92DF92EF92FF920F9335
:10A490001F93DF93CF930F92CDB7DEB77C015B01A3
:10A4A0008A01198210929DB810929CB810929FB8A0
:10A4B00010929EB81092A1B81092A0B88091511934
:10A4C0009091521960E070E0AE014F5F5F4F0E94C3
:10A4D000C22820919607809195078217F9F086E9A6
:10A4E00097E090939DB880939CB885E997E090930E
:10A4F0009FB880939EB830E086E391E0289FA0014A
:10A50000299F500D389F500D1124435F5C44509398
:10A51000A1B84093A0B874E0D72E20C084E997E09A
:10A5200090939DB880939CB883E997E090939FB8EF
:10A5300080939EB88091940790E026E331E0829F5B
:10A54000A001839F500D929F500D1124435A5645F0
:10A550005093A1B84093A0B868E0D62EE0919CB883
:10A56000F0919DB820812F5F2D1508F020E0A0917B
:10A57000A0B8B091A1B8007012968D919C911397DC
:10A58000802B912B13969C938E9312978091E403CA
:10A590009091E50315969C938E9314971796BC9211
:10A5A000AE92169781E090E019969C938E9318973F
:10A5B0001B96FC92EE921A97E0919EB8F0919FB88C
:10A5C0008081281741F080E090E8E82AF92A1B965C
:10A5D000FC92EE921A972D913C911197FA2E9B2F97
:10A5E000FD0160E070E0225030408D01020F131F2A
:10A5F0002E5F3F4F18C081916827862F829586274E
:10A60000082E869586958025082E8695802587704C
:10A61000062E672F869507948795702D68270694D8
:10A62000879570256827E017F10729F7420F531F18
:10A6300042505040FA01718360836D917C918F2D5F
:10A640000E94FE45E0919CB8F0919DB84081242F76
:10A6500030E08D2D90E00197281739071CF44F5FEB
:10A66000408301C0108280915119909152190E942B
:10A6700036270F90CF91DF911F910F91FF90EF90B0
:10A68000DF90BF90AF9008952EE130E0309384A228
:10A69000209383A2509386A2409385A24091E40325
:10A6A0005091E503509388A2409387A270938AA2A9
:10A6B000609389A221E030E030938CA220938BA29A
:10A6C00090938EA280938DA2309390A220938FA21C
:10A6D000309392A2209391A2309394A2209393A2BC
:10A6E0009091930780919407981731F49091950772
:10A6F00080919607981731F081E090E8909394A2AA
:10A70000809393A2509396A2409395A2109298A200
:10A71000109297A2109299A210929AA280914A192F
:10A7200080939BA28091441980939CA280914819A8
:10A7300080939DA28091461980939EA2E3E8F2EA5D
:10A7400020E030E018C081912827822F829582274F
:10A75000082E869586958025082E869580258770FB
:10A76000022E232F869507948795302D282706944F
:10A7700087953025282782EAEF39F80721F73183BA
:10A780002083CF014C976EE170E00E94FE45089552
:10A79000CF93DF9310929BB810929AB8AFE9B1EAC9
:10A7A00024EEED0119922A95E9F7E0919807F0E07F
:10A7B00031962AE230E0E901EC9F9001ED9F300DE7
:10A7C000FC9F300D11242E5E3F4F3093A0A12093AB
:10A7D0009FA15093A2A14093A1A14091E403509165
:10A7E000E5035093A4A14093A3A17093A6A1609305
:10A7F000A5A121E030E03093A8A12093A7A19093D8
:10A80000AAA18093A9A1F093ACA1E093ABA1F0938E
:10A81000AEA1E093ADA13093B0A12093AFA130934E
:10A82000B2A12093B1A15093B4A14093B3A1569685
:10A83000E8ECF3E086E001900D928150E1F7109290
:10A84000BBA184E190E0A0E0B0E08093BCA1909334
:10A85000BDA1A093BEA1B093BFA11092C0A182E000
:10A860008093C1A181E08093C2A18BE891E0909395
:10A87000C4A18093C3A1A5ECB1EAEFECF3E084E1BD
:10A8800001900D928150E1F740E050E020E030E08F
:10A890000FC0D901A752BE45F901E251F8448AE23E
:10A8A00001900D928150E1F74F5F5F4F265D3F4F62
:10A8B0008091980790E0481759075CF3E0919FA1B9
:10A8C000F091A0A1E356FE45F0939BB8E0939AB8AF
:10A8D000AFE9B1EA20E030E0AF0118C08D91282740
:10A8E000822F82958227082E869586958025082EB0
:10A8F000869580258770022E232F8695079487954D
:10A90000302D28270694879530252827A417B507CA
:10A9100029F73183208360919FA17091A0A18FE9D5
:10A9200091EA0E94FE45DF91CF9108950F931F9306
:10A93000CF93DF93DC011296CD91DC91139718969B
:10A940008D919C91199720E280319207F9F0E0E215
:10A9500081319E0760F4F0E280309F07A0F020E292
:10A960008530920798F08650904269F40FC0F0E26B
:10A9700080329F0740F020E28332920738F0805304
:10A980009042039718F000E410E002C000E816E1DE
:10A990004FEF5FEF20E030E06AE270E0269FF001C9
:10A9A000279FF00D369FF00D1124E251F844848169
:10A9B00095818C279D278070892B19F4A90124E0AB
:10A9C00030E02F5F3F4F2430310544F344305105D0
:10A9D000B0F58AE290E0489FE001499FD00D589F72
:10A9E000D00D1124C251D8448C819D81892BE1F076
:10A9F0006D917C911197CD014C852AE030E00E9449
:10AA00009544882371F58DEF94EA6C85A8010E9426
:10AA10009943892B31F16091FEA47091FFA48EEFD0
:10AA200094EA0E94FE451DC000D00F9283EF98E18A
:10AA3000EDB7FEB79283818385EF94E00AC000D022
:10AA40000F9283EF98E1EDB7FEB7928381838FED8C
:10AA500094E0948383830E9451F10F900F900F90A4
:10AA60000F90DF91CF911F910F9108952F923F92F8
:10AA70004F925F926F927F928F929F92AF92BF920E
:10AA8000CF92DF92EF92FF920F931F93DF93CF93BA
:10AA9000CDB7DEB762970FB6F894DEBF0FBECDBF5D
:10AAA0008DE297EA9093CCA28093CBA2B1E9EB2EF2
:10AAB000B1EAFB2E10E0812F63E00E947A31D701CA
:10AAC0001D927D011F5F1430B1F75524A3EF6A2E4C
:10AAD000A8E17A2E44244A94F1E02F2E312CEDEC9B
:10AAE000F2EA20E332E0119221503040E1F78DECA0
:10AAF00092EA0E941E44892B91F38091CEA29091FC
:10AB0000CFA2EEECF2EA20E030E0DC011297AC01DB
:10AB100044535D4518C081912827822F8295822752
:10AB2000082E869586958025082E86958025877027
:10AB3000022E232F869507948795302D282706947B
:10AB4000879530252827E417F50729F7A253BD4537
:10AB50008D919C912817390709F0C1CF1092F318F5
:10AB60004DB75EB74A5050400FB6F8945EBF0FBE67
:10AB70004DBFEDB7FEB73196ADB7BEB712967C921A
:10AB80006E92119726EF35E0338322838091D2A213
:10AB90009091D3A2958384838091D0A29091D1A2E9
:10ABA000978386838091D6A29091D7A29F77918731
:10ABB00080870E9451F12091D0A23091D1A2809142
:10ABC000E4039091E5038227932780704DB75EB729
:10ABD000465F5F4F0FB6F8945EBF0FBE4DBF892B27
:10ABE00061F0207020503F4F09F067C28091D6A2DB
:10ABF0009091D7A2409709F060C28091D6A290911F
:10AC0000D7A29F778432910509F42DC18532910531
:10AC100040F48031910599F08232910509F02EC2FD
:10AC20003CC08034910509F4C5C0AFE08D3A9A0765
:10AC300009F436C18033910509F020C2EFC000D07D
:10AC40000F92EDB7FEB77282618222EE35E0348357
:10AC500023830E9451F10F900F900F900F9080E08E
:10AC600061E00E947A318091CEA29091CFA240976C
:10AC700009F054C28EEC92EA0E9415456091D4A26C
:10AC80007091D5A24091D2A25091D3A28091D6A228
:10AC90009091D7A20E94C85341C200D00F92ADB785
:10ACA000BEB712967C926E921197E6ECF5E0149680
:10ACB000FC93EE9313970E9451F10F900F900F9019
:10ACC0000F9080E061E00E947A318091D8A29927AC
:10ACD00087FD9095882E9A8389838091D9A29927A0
:10ACE00087FD9095A82E9C838B838091DAA299276B
:10ACF00087FD9095C82E9E838D838091DBA2992736
:10AD000087FD9095E82E98878F838091DCA2992704
:10AD100087FD9095082F9A8789878091DDA290E022
:10AD20008053984F282F9C878B879A80BC80DE8029
:10AD3000F8841A853C854D855E856F85788989897B
:10AD40009A890E9448340E942F348091DEA290910B
:10AD5000DFA2A091E0A2B091E1A28093E5B7909329
:10AD6000E6B7A093E7B7B093E8B78091E2A29091DD
:10AD7000E3A2A091E4A2B091E5A28093E9B79093F9
:10AD8000EAB7A093EBB7B093ECB78091E6A28093BB
:10AD9000EDB76091D4A27091D5A24091D2A250910A
:10ADA000D3A28091D6A29091D7A20E944453409200
:10ADB0009707B4C100D00F92ADB7BEB712967C9280
:10ADC0006E921197E6EAF5E01496FC93EE931397D2
:10ADD0000E9451F10F900F900F900F9080E061E072
:10ADE0000E947A319091930780919407981739F4D3
:10ADF0009091950780919607981709F4E1C16091A9
:10AE0000D4A27091D5A24091D2A25091D3A28091A8
:10AE1000D6A29091D7A20E94425280C100D00F9238
:10AE2000ADB7BEB712967C926E921197EAE8F5E044
:10AE30001496FC93EE9313970E9451F10F900F908C
:10AE40000F900F9080E061E00E947A31409295A1CE
:10AE5000409296A1409297A1409298A18EEC92EADE
:10AE60000E94D8515BC100D00F92ADB7BEB7129609
:10AE70007C926E921197E1E7F5E01496FC93EE93C5
:10AE800013970E9451F10F900F900F900F9080E058
:10AE900061E00E947A318EEC92EA0E9487513EC1B5
:10AEA00000D00F92ADB7BEB712967C926E921197FA
:10AEB000E7E4F5E01496FC93EE9313970E9451F1AA
:10AEC00010929DA1E091D8A2F0E0E756FE454082A5
:10AED00010E00F900F900F900F9008C01F5F80E060
:10AEE00060E041E020E030E00E942A2E80919DA1A8
:10AEF000882319F41F3091F707C08F3F29F430924F
:10AF0000C2A22092C1A204C01092C2A21092C1A2F9
:10AF100022E130E03093BAA22093B9A28091D2A26C
:10AF20009091D3A29093BCA28093BBA28091E403A2
:10AF30009091E5039093BEA28093BDA28091D4A28C
:10AF40009091D5A29093C0A28093BFA28091D6A2E7
:10AF50009091D7A29093C4A28093C3A23092C6A22C
:10AF60002092C5A23092C8A22092C7A2E9EBF2EAD1
:10AF700020E030E018C081912827822F8295822717
:10AF8000082E869586958025082E869580258770C3
:10AF9000022E232F869507948795302D2827069417
:10AFA00087953025282742EAE93CF40721F73183C9
:10AFB0002083CF01409762E170E00E94FE4580E06F
:10AFC00060E042E020E030E00E942A2E80919DA1C6
:10AFD0008F3F09F04CC08091DEA2863039F0873077
:10AFE00049F0853049F41092990709C052E0509316
:10AFF000990705C084E001C086E08093990780919D
:10B00000DFA2823021F498E090939A0702C0109258
:10B010009A078091DDA28F3471F0803518F4853461
:10B0200071F405C0853619F08F3649F404C0A0E2EA
:10B03000A0939B0706C0B0E3B0939B0702C0109299
:10B040009B074091D9A25091DAA26091DBA2709146
:10B05000DCA280E02091990700919A07E0909B077D
:10B060000E94EE2F8091D8A20E94043D57C0E0912B
:10B07000D8A2F0E0E756FE45108250C000D000D0C4
:10B08000EDB7FEB73196ADB7BEB712967C926E9211
:10B09000119723E235E033832283958384830E94D2
:10B0A00051F1552453944DB75EB74A5F5F4F0FB6C9
:10B0B000F8945EBF0FBE4DBF34C080E061E00E94D7
:10B0C0007A312091D0A23091D1A2C90180708050F4
:10B0D0009F4F29F48EEC92EA0E94DE451FC000D0FB
:10B0E00000D0EDB7FEB73196ADB7BEB712967C92E1
:10B0F0006E92119744E055E0538342833583248355
:10B100000E9451F18DB79EB706960FB6F8949EBF78
:10B110000FBE8DBF8EEC92EA0E949654552009F422
:10B12000DECC80E061E00E947A31E091CBA2F09128
:10B13000CCA28091D2A29091D3A29383828380915A
:10B14000D0A29091D1A2958384838091D4A2909132
:10B15000D5A29783868311861086AFE0B0E0B183D5
:10B16000A08354861E2F9F2FDF0120E030E0AF0127
:10B17000435F5F4F18C08D912827822F82958227C9
:10B18000082E869586958025082E869580258770C1
:10B19000022E232F869507948795302D2827069415
:10B1A000879530252827A417B50729F730933BA7A3
:10B1B00020933AA760817181812F0E94FE458FCC38
:10B1C000E2E05E2EAECFCF92DF92EF920F93DF934D
:10B1D000CF930F92CDB7DEB780EB99E0EDE5F9EABA
:10B1E000DF019C011D9221503040E1F780E040E0FA
:10B1F00052EC61E070E026E000E0EE240E9438337B
:10B200001092519D1092529D1092539D1092549DF8
:10B210001092599D10925A9D10925B9D10925C9DC8
:10B220001092629D1092619D88E0E3E8F7E0DF01F3
:10B230001D928A95E9F71092669D1092659D109275
:10B240008EA110928DA110929AA1109299A11092A4
:10B250009DA110929EA188EAEEEEF7EBDF011D9210
:10B260008A95E9F781E091E0BE016F5F7F4F0E9410
:10B270003837898181508E3F38F06091E5036983CA
:10B2800081E091E00E949F3782E091E063E479E100
:10B290000E943837809143198F3F41F481E08093B9
:10B2A000431982E091E061E00E949F378981809399
:10B2B000E6031092E4038093E50380E094E0E1E587
:10B2C000F9E8DF019C011D9221503040E1F780E058
:10B2D00090E1E1E5FDE8DF019C011D922150304045
:10B2E000E1F7109299A110929AA110929BA110924D
:10B2F0009CA101E0C02ED12CF601EA56F744E08172
:10B30000E13019F0E230C1F408C08C2D40E052EC7D
:10B3100061E070E026E000E007C08C2D40E052ECD8
:10B3200061E070E026E008E0EE240E9438338C2DC6
:10B330006FEF4FEF0E94A2380894C11CD11C34E07B
:10B34000C316D104C9F60F90CF91DF910F91EF9002
:10B35000DF90CF900895DF93CF930F92CDB7DEB7F4
:10B36000809164008B7F8093640080916400877F6C
:10B370008093640084B1876284B9289A81E58CBD8A
:10B3800080E48093800088E08093810010928500A3
:10B39000109284008AE790E090938900809388005F
:10B3A00085E18EBD0DB407FEFDCF85E58EBD8EB562
:10B3B00089830DB407FEFDCF80E48EBD8EB58983F1
:10B3C0000DB407FEFDCF8EB589838CB58B7F8CBD08
:10B3D0008DE18EBD0DB407FEFDCF80E58EBD8EB52F
:10B3E00089830DB407FEFDCF8EB589838CB584604B
:10B3F0008CBD1EBC0DB407FEFDCF1EBC3EB50DB40A
:10B4000007FEFDCF2EB5932F80E0622F70E0682BF2
:10B41000792B8CB58B7F8CBD8DE18EBD0DB407FE75
:10B42000FDCF80E68EBD8EB589830DB407FEFDCFBE
:10B430008EB589838CB584608CBD1EBC0DB407FEAF
:10B44000FDCF1EBC3EB50DB407FEFDCF2EB5932F2C
:10B4500080E0422F50E0482B592B8CB58B7F8CBD60
:10B460008DE18EBD0DB407FEFDCF80E98EBD8EB59A
:10B4700089830DB407FEFDCF8EB589838CB58460BA
:10B480008CBD1EBC0DB407FEFDCF1EBC3EB50DB479
:10B4900007FEFDCF2EB5932F80E0E22FF0E0E82BE2
:10B4A000F92B8CB58B7F8CBD8DE18EBD0DB407FE65
:10B4B000FDCF80EA8EBD8EB589830DB407FEFDCF2A
:10B4C0008EB589838CB584608CBD1EBC0DB407FE1F
:10B4D000FDCF1EBC3EB50DB407FEFDCF2EB5932F9C
:10B4E00080E030E0282B392BCB01A4E0969587959E
:10B4F000AA95E1F78854944F9093A2078093A107EF
:10B5000067707070762F6627770F770FCA01A6E0F5
:10B5100096958795AA95E1F7682B792B605F784D12
:10B520007093A4076093A307CF0176E09695879563
:10B530007A95E1F788539F4F9093A6078093A507CC
:10B54000C901880F892F881F990B91958A5F9040B8
:10B550009093A8078093A7074F73507096E0440F0D
:10B56000551F9A95E1F7EF73F0704E2B5F2B4E51FC
:10B570005B4F83E0440F551F8A95E1F75093AA076C
:10B580004093A9072F7730702C593F4F3093AC0769
:10B590002093AB070F90CF91DF910895FC019B01A1
:10B5A0008091B1079091B2076AE070E00E9411F4B7
:10B5B000718360838091B3079091B4076AE070E073
:10B5C0000E9411F4F901718360830895AF92BF92D4
:10B5D000CF92DF92EF92FF920F931F93DF93CF935F
:10B5E0000F92CDB7DEB7809164008B7F80936400AB
:10B5F00080916400877F80936400809181008160E6
:10B60000809381008CB58B7F8CBD8FE08EBD0DB497
:10B6100007FEFDCF80E48EBD8EB589830DB407FE95
:10B62000FDCF8EB5898380E060E040E022E330E02A
:10B630000E942A2E8CB584608CBD1EBC0DB407FE02
:10B64000FDCF1EBC3EB50DB407FEFDCF2EB5932F2A
:10B6500080E030E0822B932B9093AE078093AD0770
:10B660008CB58B7F8CBD8FE08EBD0DB407FEFDCFFA
:10B6700080E28EBD8EB589830DB407FEFDCF8EB5F9
:10B68000898380E060E040E022E330E00E942A2EDF
:10B690008CB584608CBD1EBC0DB407FEFDCF1EBCF6
:10B6A0002EB50DB407FEFDCFEEB4922F80E0FF243F
:10B6B000E82AF92AF092B007E092AF078091800063
:10B6C000887F809380008091A9079091AA07E81A4B
:10B6D000F90AF092B607E092B5070027F7FC00954B
:10B6E000102F2091AB073091AC07442737FD4095D0
:10B6F000542FC801B7010E94F2F33BE0959587955E
:10B70000779567953A95D1F768537F4F7093B20755
:10B710006093B107A090AD07B090AE078091A307EA
:10B720009091A407A81AB90A2091A7073091A807F9
:10B73000442737FD4095542FC801B7010E94F2F30A
:10B740002CE095958795779567952A95D1F7A61A58
:10B75000B70ACC24B7FCC094DC2C2091A50730910B
:10B76000A607442737FD4095542FC801B7010E9412
:10B77000F2F31DE095958795779567951A95D1F722
:10B780002091A1073091A207260F371F442737FDCC
:10B790004095542FC601B5010E94F2F3BCE0959587
:10B7A000879577956795BA95D1F768517C4F7093D7
:10B7B000B4076093B307809164008860809364004D
:10B7C000809164008460809364000F90CF91DF913A
:10B7D0001F910F91FF90EF90DF90CF90BF90AF90AF
:10B7E00008950E94155C0E94AB5908950E94F15B78
:10B7F00080E060E040E024EF31E00E942A2E0E94C9
:10B80000E65A0E94985C8AE499E164E479E10E9436
:10B81000895C88E499E166E479E10E94CE5A80E08F
:10B8200061E040E020E030E0E8CF6F9A089588239F
:10B8300091F0779A7798779A7798779A7798779A16
:10B840007798779A7798779A7798779A7798779A78
:10B850007798779A7798779A6E9A7798779A6E987A
:10B8600077980895809560959DB187FB96F99DB96D
:10B87000779AE8946699689487F9779886FB96F9A1
:10B880009DB9779AE8946699689486F9779885FBCC
:10B8900096F99DB9779AE8946699689485F97798AE
:10B8A00084FB96F99DB9779AE8946699689484F92F
:10B8B000779883FB96F99DB9779AE894669968948E
:10B8C00083F9779882FB96F99DB9779AE8946699FF
:10B8D000689482F9779881FB96F99DB9779AE894F4
:10B8E0006699689481F9779880FB96F99DB9779A63
:10B8F000E8946699689480F9779860FB96F99DB909
:10B90000779AE8946699689460F977986E9890E0D1
:10B910000895FC01DB0180914E1990914F1991839C
:10B92000808380914C1990914D198D939C9308952B
:10B930000F931F9381E00E94175C85E061E00E94F5
:10B94000325C8150914010F080E0B3C080E060E054
:10B9500040E020E931E00E942A2E8FEF60E00E9453
:10B96000325C182F8FEF61E00E94325C682F70E02C
:10B97000912F80E0682B792B7093B8076093B707FD
:10B9800080E898E3861B970B0E9443D8DC01CB012B
:10B990005AE0B695A795979587955A95D1F76DEC8E
:10B9A00072E90E9443D841E196958795779567950E
:10B9B0004A95D1F76059714070934D1960934C19B5
:10B9C00080E00E94175C83E061E00E94325C80E0CE
:10B9D00060E040E020E931E00E942A2E8FEF60E035
:10B9E0000E94325C182F00E010934F1900934E19FB
:10B9F0008FEF61E00E94325C90E0802B912B8E579C
:10BA00009F4090934F1980934E196091B7077091A2
:10BA1000B8076E517B4F845C99400E9454D8DC017A
:10BA2000CB0100914C1910914D193AE0B595A795AD
:10BA3000979587953A95D1F76CE173E40E9454D8B5
:10BA400025E195958795779567952A95D1F7060F06
:10BA5000171F10934D1900934C1917FF04C0109233
:10BA60004D1910924C1980914C1990914D1981519A
:10BA7000974234F080E197E290934D1980934C19EE
:10BA800080914C1990914D1964E670E00E9411F478
:10BA900070934D1960934C1980914E1990914F19E4
:10BAA00064E670E00E9411F470934F1960934E1990
:10BAB0008FEF1F910F91089580E197E2A0E0B0E031
:10BAC0000197A109B109E1F780E060E040E024E6D8
:10BAD00030E00E942A2EF0CF80E060E04AE020E0D3
:10BAE00030E00E942A2EF8CF2F923F924F925F9221
:10BAF0006F927F928F929F92AF92BF92CF92DF927E
:10BB0000EF92FF920F931F93DF93CF93CDB7DEB7E2
:10BB100029970FB6F894DEBF0FBECDBF0E9416372F
:10BB20000E94E7330E9491398DE13E010894611C27
:10BB3000711CB3010E94E829909352198093511906
:10BB40000F920F9281E090E0ADB7BEB712969C9332
:10BB50008E93119786EF9BE560E070E048EB50E133
:10BB60002CE309EE13E0E9EBEE2EEFE0FE2EA12C24
:10BB700031E0B32EC12CD12C882499240E94972C1B
:10BB80000F900F908CE368EE73E0A3010E941F2CCE
:10BB900081E0809396B817E9E12E18EBF12EB3E01F
:10BBA000CB2ED12CCC0EDD1E00E111E0A2E0AA2E9E
:10BBB000B12CAC0EBD1EC801B5010E9438378A8178
:10BBC0008F3F29F41A82C80160E00E949F378A8162
:10BBD000F6018083813019F0823039F403C0D70137
:10BBE0008C9305C0F701808302C0D7011C92005FCF
:10BBF0001F4F0894E11CF11C0894C11CD11CB1E03A
:10BC000000341B07C1F610924D890E94E3580F9231
:10BC10000F9281E090E0EDB7FEB79283818386E3D7
:10BC200095E560E070E048EB5FE024E10AEE13E0A8
:10BC3000F9EBEF2EFDE0FF2EA12CE2E0BE2EC12C91
:10BC4000D12C882499240E94972C0F900F9084E186
:10BC500065EF73E0AE014F5F5F4F0E941F2C2EEE29
:10BC600037EE398728878EE099EB9F838E835EE4D9
:10BC7000452E59E8552E2224332441E0642E712CA0
:10BC8000E3E0F0E0EC0FFD1FE20DF31D80818A83FD
:10BC9000ADB7BEB718970FB6F894BEBF0FBEADBF15
:10BCA000EDB7FEB7319623EF38E112963C932E9311
:10BCB0001197ADEDB8E0B383A283358224828683E9
:10BCC00017820E9451F180E5E5E0F8EE11928A9525
:10BCD000E9F72DB73EB7285F3F4F0FB6F8943EBF48
:10BCE0000FBE2DBF8A81843009F46FC0853058F4AF
:10BCF0008130B1F0813008F4B4C0823039F1833042
:10BD000009F045C13CC0863009F4D0C0863008F443
:10BD100082C0873009F4EFC0883009F038C111C102
:10BD2000D2011C92EDB7FEB738970FB6F894FEBF5C
:10BD30000FBEEDBF319625E038EEADB7BEB7129617
:10BD40003C932E93119781E998E039C1F20110825A
:10BD50002DB73EB7285030400FB6F8943EBF0FBE07
:10BD60002DBFEDB7FEB7319625E038EEADB7BEB7C3
:10BD700012963C932E93119789E498E020C18FEF9F
:10BD8000F20180832DB73EB7285030400FB6F894AB
:10BD90003EBF0FBE2DBFEDB7FEB7319625E038EEA2
:10BDA000ADB7BEB712963C932E93119781E098E001
:10BDB000938382838091E6038483158277826682EF
:10BDC0000E9451F104EA13E106C18FEFF201808372
:10BDD0002DB73EB7285030400FB6F8943EBF0FBE87
:10BDE0002DBFEDB7FEB7319625E038EEADB7BEB743
:10BDF00012963C932E9311978CEB97E0938382835A
:10BE00008091E60384831582778266820E9451F1D5
:10BE10000EE31FE0E0C08FEFF20180832DB73EB745
:10BE2000285030400FB6F8943EBF0FBE2DBFEDB77F
:10BE3000FEB7319625E038EEADB7BEB712963C930B
:10BE40002E9311978FE697E0938382838091E60388
:10BE500084831582778266820E9451F104EC18E196
:10BE6000BAC0F20110822DB73EB7285030400FB64D
:10BE7000F8943EBF0FBE2DBFEDB7FEB7319625E05B
:10BE800038EEADB7BEB712963C932E93119789E268
:10BE900097E0938382838091E6038483158277827F
:10BEA00066820E9451F106E91AE195C0F201108202
:10BEB0002DB73EB7285030400FB6F8943EBF0FBEA6
:10BEC0002DBFEDB7FEB7319625E038EEADB7BEB762
:10BED00012963C932E93119780EE96E09383828383
:10BEE0008091E60384831582778266820E9451F1F5
:10BEF0000AE617ED70C08FEFF20180832DB73EB7D1
:10BF0000285030400FB6F8943EBF0FBE2DBFEDB79E
:10BF1000FEB7319625E038EEADB7BEB712963C932A
:10BF20002E93119780EA96E0938382838091E603B3
:10BF300084831582778266820E9451F100EA15E1BE
:10BF40004AC08FEFF20180832DB73EB728503040B2
:10BF50000FB6F8943EBF0FBE2DBFEDB7FEB73196BA
:10BF600025E038EEADB7BEB712963C932E931197ED
:10BF70008CE596E0938382838091E6038483158227
:10BF8000778266820E9451F105E01EE024C0F20132
:10BF900010822DB73EB7285030400FB6F8943EBF00
:10BFA0000FBE2DBFEDB7FEB7319625E038EEADB729
:10BFB000BEB712963C932E9311978FE196E0938330
:10BFC00082838091E60384831582778266820E9451
:10BFD00051F100E010E0ADB7BEB718960FB6F89477
:10BFE000BEBF0FBEADBFA3EFB8E1E5E0F8EE80E560
:10BFF00001900D928150E1F7E5E0F8EEF09301E851
:10C00000E09300E801900020E9F73197E550F84E01
:10C01000E09302E8109203E885E0809304E880E072
:10C0200098EE0E94913C0115110509F488C0A8857D
:10C03000B9856C9211966C921197EE81FF811596DD
:10C04000FC93EE931497F1E02F16310471F122E086
:10C050002216310409F44AC02114310409F06FC0DA
:10C060000F920F9281E090E0ADB7BEB712969C930D
:10C070008E931197C8016EEE77EE48EB5DE02EE1EE
:10C080000BEE13E039EBE32E3BE0F32EA12CB2E0F4
:10C09000BB2EC12CD12C882499240E94972C0F9060
:10C0A0000F908EE16FEF73E045C00F920F92EDB7E6
:10C0B000FEB732822182C80164EF77EE48EB5BE085
:10C0C00028E20CEE13E0A9EBEA2EA9E0FA2EA12C4F
:10C0D000F2E0BF2EC12CD12C882499240E94972CE9
:10C0E0000F900F9088E263E074E024C00F920F92EB
:10C0F00081E090E0ADB7BEB712969C938E931197F6
:10C10000C8016AEF77EE48EB59E022E30DEE13E049
:10C11000E9EBEE2EE7E0FE2EA12C32E0B32EC12C8F
:10C12000D12C882499240E94972C0F900F9082E3A1
:10C1300067E074E0AE014F5F5F4F0E941F2C0894D0
:10C14000211C311C0894611C711CE885F985369608
:10C15000F987E8872E813F812056304F3F832E8319
:10C160000894411C511C33E02316310409F088CD9A
:10C1700080E065E040E020E030E00E942A2E8091DF
:10C180009707882319F00E947FEB07C00E941CEBE1
:10C19000882319F080E00E9458EB80E090E0299617
:10C1A0000FB6F894DEBF0FBECDBFCF91DF911F91C8
:10C1B0000F91FF90EF90DF90CF90BF90AF909F9046
:10C1C0008F907F906F905F904F903F902F90089549
:10C1D00014BE88E10FB6F89480936000109260005E
:10C1E0000FBE12B811B815B814B818B817B81BB8E4
:10C1F0001AB81EB81DB811BA10BA14BA13BA1092F0
:10C20000020110920501109204011092080110928F
:10C21000070110920B0110920A01E4E6F0E0808120
:10C220008F6E8083E5E6F0E080818F6380830E94DB
:10C23000DE330E94CB300E9448EC0E942EEB8093AC
:10C24000501908958FEF80939EA181E060E040E057
:10C2500020E030E00E942A2EF8CFCF93DF93EC014C
:10C26000898160E040E00E94A238282F8F3FD9F4F6
:10C27000EC81FD81E050FB4F1082EC81FD81EF5F8E
:10C28000FA4F1082EC81FD81EE5FFA4F1082EC8153
:10C29000FD81ED5FFA4F8FEF9FEFAFEFBFEF808330
:10C2A0009183A283B383822FDF91CF910895CF92A0
:10C2B000DF92EF92FF921F93DF93CF930F92CDB750
:10C2C000DEB77C01198210E06E010894C11CD11CFC
:10C2D000D70111968C9160E470E0A6010E94B832FB
:10C2E000982F8981882351F08FEF0F90CF91DF91A4
:10C2F0001F91FF90EF90DF90CF900895D701149693
:10C30000ED91FC911597E10FF11DE050FF4F9083E7
:10C310001F5FDECFEF92FF920F931F93DF93CF93B8
:10C320000F92CDB7DEB77C0119828091511990919F
:10C33000521960E070E0AE014F5F5F4F0E94C2286B
:10C340008091950790E026E331E0829F8001839FF2
:10C35000100D929F100D1124035F1C4480E290E0A9
:10C36000D80113969C938E93129782E01C968C931F
:10C37000D7011496ED91FC911597E25EF94F8191EA
:10C380009191D8011E969C938E931D97D7018C9105
:10C3900090E02091E4033091E503822B932BD801A8
:10C3A00050969C938E931F972081E052F6402A303E
:10C3B00018F5EE5DF94F408150E0425E5F4F1196F7
:10C3C0005C934E934E5150408DE351968C93519710
:10C3D0005B965C934E935A9759962C9359978291FA
:10C3E00058968C939801245E3F4F3696C901BF0141
:10C3F00050E00E941CF00CC08DE190E0F8019183A8
:10C40000808386E2818B81E090E0918F808F228F04
:10C41000D7011496ED91FC911597ED5DF94F808150
:10C420009181A281B381F801828B938BA48BB58B10
:10C43000808191814A97978B868B80919507833075
:10C4400020F48F5F8093950702C01092950790911A
:10C45000950780919607981741F4933020F49F5FD9
:10C460009093960702C0109296078091511990916F
:10C4700052190E9436270F90CF91DF911F910F9193
:10C48000FF90EF900895EF92FF920F931F93DF9329
:10C49000CF930F92CDB7DEB77C01198280915119ED
:10C4A0009091521960E070E0AE014F5F5F4F0E94C3
:10C4B000C2288091930790E026E331E0829F8001BB
:10C4C000839F100D929F100D1124035A164580E989
:10C4D00090E0A0E0B0E0F8018787908BA18BB28B51
:10C4E0008091E603838BD7018C91848B81E3858BCC
:10C4F00081E0868B1496ED91FC911597E85FFA4FD9
:10C50000808190E08596F8019183808322E030E07D
:10C510003383228321E924874197968785878091F9
:10C52000E5B79091E6B7A091E7B7B091E8B7878BF0
:10C53000908FA18FB28F8091E9B79091EAB7A091C7
:10C54000EBB7B091ECB7838F948FA58FB68F0E9415
:10C550003C34D8015F966D937D938D939C93929715
:10C56000D7011496ED91FC9115970D5D1F4FE85F73
:10C57000FA4F4191BF01C80150E00E941CF0809128
:10C580009307873020F48F5F8093930702C0109247
:10C5900093079091930780919407981741F49730EF
:10C5A00020F49F5F9093940702C0109294078091AB
:10C5B0005119909152190E9436278FEF0F90CF9109
:10C5C000DF911F910F91FF90EF900895CF92DF922E
:10C5D000EF92FF920F931F93DF93CF930F92CDB7FC
:10C5E000DEB77C0119828E010F5F1F4FD7011196B4
:10C5F0008C9160E470E0A8010E94B832982F8E37C9
:10C6000019F08981882391F38981882309F057C023
:10C610009E3709F054C0F70104811581085F1A4F55
:10C62000D8011C92818160E470E06E010894C11C05
:10C63000D11CA6010E94B832F80180838981882329
:10C64000F1F5D7011496ED91FC911597E85FFA4F3B
:10C6500080818823A1F100E010E017C0F7018181FB
:10C6600060E470E0A6010E94B832982F8981882387
:10C6700031F5D7011496ED91FC911597E00FF11F5C
:10C68000E75FFA4F90830F5F1F4FD7011496ED912C
:10C69000FC911597E85FFA4F8081682F70E0CB011D
:10C6A000029608171907D0F26D5F7F4FCF014FEF49
:10C6B0005FEF0E94363C882311F08FEF01C080E0CD
:10C6C0000F90CF91DF911F910F91FF90EF90DF902E
:10C6D000CF900895CF93DF93EC018C819D81885F8B
:10C6E0009A4FFC0182E091E0DF019C011D922150F4
:10C6F0003040E1F7CE010E94E6628F3F19F4CE018F
:10C700000E944362DF91CF9108950F931F93CF93BF
:10C71000DF93EC01062F662399F010E00DC0EC8149
:10C72000FD81E10FF11D898160814AE050E00E94A6
:10C73000F331882329F41F5F101788F38FEF01C0AE
:10C7400080E0DF91CF911F910F910895FF920F9399
:10C750001F938C01DC011496EC9114971596FC91B3
:10C7600080E091E0DF019C011D9221503040E1F713
:10C7700000D00F92D80114968D919C911597EDB72A
:10C78000FEB7928381838CE999E0948383830E942E
:10C7900051F10F900F900F900F90C8016BE00E9425
:10C7A0008563F82ED8011496ED91FC911597EE5FF4
:10C7B000FA4F8FEF808314960D911C9115970E946C
:10C7C00023340D5F1A4F645C7F4F8F4F9F4FF801EA
:10C7D00060837183828393838F2D1F910F91FF90CC
:10C7E0000895CF92DF92EF92FF920F931F93DF9302
:10C7F000CF9300D0CDB7DEB77C015B834A83683529
:10C8000009F44CC06935B8F4693409F45AC16A3482
:10C8100050F4633409F4C5C0663409F43FC0613490
:10C8200009F05FC283C1623511F16335F1F16F34F4
:10C8300009F057C21CC0693609F443C16A3648F48E
:10C84000633609F4AEC0663649F1613609F049C273
:10C850006DC1623761F0633720F46F3609F041C271
:10C8600006C0633711F1683709F03BC217C0D70122
:10C8700011968C916FEF40E00E94A238D701149678
:10C88000ED91FC911597E050FB4F8FEF808314964C
:10C89000ED91FC911597EF5FFA4F11C1C7010E940E
:10C8A000A6638F3F09F01EC2FCC1F701A481B581C8
:10C8B000A050BB4F8C91A050B540882319F42BE0B9
:10C8C00034E00CC0AE5FBA4F8C91A250B5408823C3
:10C8D00019F42FE034E002C022E134E0AF5FBA4F38
:10C8E0008C91A150B540882319F46BE074E002C02C
:10C8F0006FE074E0A95FBA4F8C91A750B5408130CA
:10C9000019F04BE054E002C04FE054E08DB79EB701
:10C910000A970FB6F8949EBF0FBE8DBF0DB71EB716
:10C920000F5F1F4FA95DB94FEDB7FEB7B283A1836B
:10C9300081E799E0D80113969C938E9312971596F0
:10C940003C932E93149717967C936E931697199693
:10C950005C934E9318970E9451F1D7011496ED9174
:10C96000FC911597E05EF94F81E0808314960D905D
:10C97000BC91A02DCD01895D994FFC010190002053
:10C98000E9F73197E81BF90BAE5DB94FEC938FEFE8
:10C99000EDB7FEB73A960FB6F894FEBF0FBEEDBFE7
:10C9A000A1C180E060E040E024E630E00E942A2E51
:10C9B000D7011496CD90DC9015970A811B81011543
:10C9C000110519F42EE134E014C0B601665F794F09
:10C9D000C8010E9477F09C01200F311FF9010190DE
:10C9E0000020E9F73197E21BF30BE20FF31FFB8303
:10C9F000EA83D9010D900020E9F78D010150104024
:10CA0000021B130B09F46DC1C60180509F4FFC013E
:10CA100080E094E0DF01AC011D9241505040E1F70D
:10CA2000D70114968C91149715969C91B901A80181
:10CA30000E941CF019826E010894C11CD11C07C011
:10CA4000F701818160E470E0A6010E94B83289811B
:10CA50008823B1F3C701602F0E948563C7010E943C
:10CA60005761D70114962D913C911597A90140501B
:10CA70005F4FDA010D900020E9F71197A41BB50B69
:10CA8000295D394FC901BA01AD010E941CF0F701BF
:10CA9000A481B581CD01895D994FFC0101900020F1
:10CAA000E9F73197E81BF90BAE5DB94FEC93D7016D
:10CAB0001496ED91FC911597E05EF94F81E080832B
:10CAC000F0C000D00F92F70184819581895D994F64
:10CAD000ADB7BEB712969C938E93119780E699E0FE
:10CAE00014969C938E9313970E9451F1D70114963C
:10CAF000ED91FC911597E05EF94F81E080831496EB
:10CB00000D90BC91A02DCD01895D994FFC01019044
:10CB10000020E9F73197E81BF90BAE5DB94FEC93B4
:10CB20008FEF0F900F900F900F90DCC0F701848172
:10CB30009581865F994FFC0184E1DF011D928A9502
:10CB4000E9F7F70184819581865F994F68E372E088
:10CB50000E94B4EFD70114966D917C911597665F92
:10CB6000794F8A819B81AE014E5F5F4F0E94A0F09A
:10CB7000FC01009709F4B5C080818F3611F08F3425
:10CB800031F48181863611F0863409F48083808106
:10CB90008F34F9F0803570F48133D9F0823320F48A
:10CBA000803309F09EC01FC08634E9F08E3409F04E
:10CBB00098C019C08E36B9F08F3630F4893549F0F7
:10CBC000863609F08EC00FC08F3619F0893709F00C
:10CBD00088C0D7011496ED91FC911597E95FFA4F43
:10CBE00081E0808308C0D7011496ED91FC911597E0
:10CBF000E95FFA4F1082F701828193810480F58109
:10CC0000E02DE95FFA4F805C9F4F60810E949F3763
:10CC1000F701A481B581A95FBA4F8C91A750B540A7
:10CC2000813019F02BE034E002C02FE034E000D076
:10CC300000D04DB75EB74F5F5F4FA95DB94FEDB7FD
:10CC4000FEB7B283A18382E599E0DA0113969C9343
:10CC50008E93129715963C932E9314970E9451F140
:10CC6000F701A481B581CD01895D994FFC01019047
:10CC70000020E9F73197E81BF90BAE5DB94FEC9353
:10CC8000D7011496ED91FC911597E05EF94F81E084
:10CC90008083EDB7FEB736960FB6F894FEBF0FBE91
:10CCA000EDBFD70114968D919C911597895D994F91
:10CCB0006FE479E042E050E00E94ABEFD7011496B8
:10CCC000ED91FC911597E05EF94F81E08083149619
:10CCD000ED91FC911597EE5DF94F82E080838FEF27
:10CCE00001C080E00F900F900F90CF91DF911F91C6
:10CCF0000F91FF90EF90DF90CF900895CF92DF9249
:10CD0000EF92FF920F931F93DF93CF930F920F92A7
:10CD1000CDB7DEB76C01DC018C9190E029E031E009
:10CD2000829FF001839FF00D929FF00D1124CF019F
:10CD30008E5892469A838983EF58F1461082149652
:10CD40008D919C911597865F994FFC0184E1DF01DD
:10CD50001D928A95E9F7F60184819581865F994F46
:10CD600068E372E00E94B4EFD60114966D917C9155
:10CD70001597665F794F89819A817E010894E11C3D
:10CD8000F11CA7010E94A0F08C01009711F481E032
:10CD900026C08AE399E00E94C6EFAC01C8016AE3AD
:10CDA00079E00E94CFEF892B29F5D6011496ED91F9
:10CDB000FC911597E65FF94FC7016AEE78E04AE00B
:10CDC00028E00EE319E07F010E941F38682F8823B6
:10CDD00009F082C018C0823069F08330A1F0D6011A
:10CDE0001496ED91FC9115978130B1F4E05EF94F06
:10CDF0008DE015C0D6011496ED91FC911597E05E7B
:10CE0000F94F8EE00CC0D6011496ED91FC91159768
:10CE1000E05EF94F8AE003C0E05EF94F8FE0808367
:10CE2000C6010E948A61F601808190E029E031E02C
:10CE3000AC01429FC001439F900D529F900D112461
:10CE40008E589246FC0180E091E0DF01AC011D921A
:10CE500041505040E1F7D6018C9190E0829FF00163
:10CE6000839FF00D929FF00D1124E759F246118235
:10CE700010828C9190E0829FF001839FF00D929F31
:10CE8000F00D1124E759F24612828C9190E0829FB6
:10CE9000F001839FF00D929FF00D1124E759F246A7
:10CEA000148213828C9190E0829FF001839FF00D99
:10CEB000929FF00D1124E759F246158216821782CF
:10CEC00010860F900F90CF91DF911F910F91FF90DF
:10CED000EF90DF90CF90089549815A81C6010E945A
:10CEE000F1638F3F09F077CF9BCFCF92DF92EF9224
:10CEF0000F93DF93CF930F920F92CDB7DEB76C01F4
:10CF0000DC0111968C911197813031F480E093E02F
:10CF100013969C938E931297F6018181823021F4AF
:10CF200080E095E093838283D60111968C911197CE
:10CF3000833031F480E097E013969C938E931297A0
:10CF4000D6011496ED91FC911597309741F087E248
:10CF500097E0DF019C011D9221503040E1F7D6019E
:10CF600011968C9140E056E960E070E026E000E028
:10CF7000EE240E94383380E060E041E020E030E0C1
:10CF80000E942A2EF601818160E040E00E94A238D2
:10CF9000D6011496ED91FC911597E050FB4F11923C
:10CFA000108236968FEF808312968D919C91139705
:10CFB000805C9F4FBF010E943837D6011496ED91D7
:10CFC000FC911597E95FFA4F8081823058F081E03B
:10CFD000808312968D919C911397805C9F4F61E0A6
:10CFE0000E949F37D6011496ED91FC911597E05061
:10CFF000FB4F1192108236968081813069F48091C6
:10D000001F04909120049A838983C60162E7AE01D0
:10D010004F5F5F4F0E94F163809143198C3318F486
:10D020008CE3809343198FEF0F900F90CF91DF9196
:10D030000F91EF90DF90CF9008958FEF80939EA196
:10D0400081E060E040E020E030E00E942A2EF8CF4E
:10D05000CF92DF92EF92FF920F931F93DF93CF93C4
:10D06000CDB7DEB762970FB6F894DEBF0FBECDBF67
:10D070006C011982809151199091521960E070E011
:10D08000AE014F5F5F4F0E94C2288091930790E0EE
:10D0900026E331E0829F8001839F100D929F100D47
:10D0A0001124035A16458AE5D8011D928A95E9F79D
:10D0B0008CE590E0F8019183808385E090E0938394
:10D0C000828380E684870E943C346A837B838C83DE
:10D0D0009D83D6011196EC91F0E0EE0FFF1FEF5A01
:10D0E000F24680819181A0E0B0E0F801828F938FB9
:10D0F000A48FB58F92E0E92EF12CEC0EFD1EC70136
:10D100000E943235FC018681D80192968C939297C9
:10D1100084815E968C935E9782815F968C935F97F5
:10D1200080858F5F91968C939197808190968C9358
:10D1300090978285845693968C93C7010E943235CE
:10D14000FC018681D80198968C9398978481949657
:10D150008C939497828195968C93959780858F5F19
:10D1600097968C939797808196968C9396978285C5
:10D17000845699968C9399979A961C92C801CF964B
:10D1800020E1DC01822F1D928A95E9F7C8018D9676
:10D19000DC011D922A95E9F7F80116AE15AE14A62A
:10D1A00013A6D60111968C9190E02091E403309162
:10D1B000E503822B932B96878587EDB7FEB73897CB
:10D1C0000FB6F894FEBF0FBEEDBF2DB73EB72F5F71
:10D1D0003F4F86E0E82EF12CEC0EFD1EF282E1823C
:10D1E00081E294E0D90113969C938E931297D60115
:10D1F0001496ED91FC911597E05FF64F8081918137
:10D20000A281B381F90184839583A683B7830E94A9
:10D210002DF18DB79EB708960FB6F8949EBF0FBE3E
:10D220008DBFC8010F96B7010E94873E809193077A
:10D23000873020F48F5F8093930702C0109293078A
:10D240009091930780919407981741F4973020F4B8
:10D250009F5F9093940702C0109294078091511998
:10D26000909152190E94362780E062960FB6F8948A
:10D27000DEBF0FBECDBFCF91DF911F910F91FF9009
:10D28000EF90DF90CF900895EF92FF920F931F934E
:10D29000CF93DF93EC018C819D818057984FFC01E7
:10D2A00080ECDF011D928A95E9F78C819D81805F7A
:10D2B000974FFC0180E091E0DF019C011D9221501D
:10D2C0003040E1F78C819D816F3F29F48057984F62
:10D2D00064ED7AE004C08057984F6DED7AE00E94CB
:10D2E000B4EF8C819D818057984F65EE7AE00E9463
:10D2F000B4EFEC81FD81E85AFA4F8081E85CFD4F84
:10D300008F3F21F4CF016DEC7AE003C0CF0160EDD7
:10D310007AE00E94B4EF8C819D818057984F6BEE2C
:10D320007AE00E94B4EFEC81FD81E95AFA4F8081E6
:10D33000E75CFD4F8F3F21F4CF016DEC7AE003C035
:10D34000CF0160ED7AE00E94B4EFEC81FD81EB5FEC
:10D35000FA4F80819181E557FD4F8F3F910529F06C
:10D3600020F0CF0163EF7AE003C0CF0161E47BE0FE
:10D370000E94B4EF8C819D818057984F6EE87BE0CE
:10D380000E94B4EFEC81FD81E75AFA4F8081E95C9D
:10D39000FD4F813021F0CF0167EA7BE003C0CF0170
:10D3A00063EA7BE00E94B4EF8C819D818057984FA7
:10D3B00068E97BE00E94B4EFEC81FD81E050FB4F17
:10D3C0008081E057FD4F813021F4CF016DEC7AE090
:10D3D00003C0CF0160ED7AE00E94B4EFAC81BD8163
:10D3E000AF5FBA4F0D911D916D917C911197AA5E1F
:10D3F000BB4F4D915C91119717962D913C911197D0
:10D400008E91AF51B940882319F48BE294E002C0A9
:10D410008FE294E0EDB7FEB770970FB6F894FEBFB9
:10D420000FBEEDBFEDB6FEB60894E11CF11CA05F87
:10D43000B74FB283A183A058B040F701B383A28352
:10D4400015830483778366835187408733872287D8
:10D4500095878487AB58B2408D919C91978786873A
:10D460000E942DF1EC81FD81EB58F84F81E0808323
:10D47000AC81BD81CD01805F974FFC010190002000
:10D48000E9F73197E81BF90BA958B84FEC932DB782
:10D490003EB7205F3F4F0FB6F8943EBF0FBE2DBF83
:10D4A0008FEFDF91CF911F910F91FF90EF90089533
:10D4B000CF93DF93EC018C819D81805F974FFC01BE
:10D4C00080E091E0DF019C011D9221503040E1F7A6
:10D4D0008C819D81FC01E95EFA4F2081805F974F2E
:10D4E000222321F0BF010E942CF004C06FE67CE0F3
:10D4F0000E94B4EFEC81FD81CF01805F974FDC018A
:10D500000D900020E9F71197A81BB90BE958F84FC7
:10D51000A0838FEFDF91CF910895EF92FF920F9349
:10D520001F93DF93CF930F92CDB7DEB77C011982A3
:10D53000809151199091521960E070E0AE014F5FF7
:10D540005F4F0E94C2288091950790E026E331E06A
:10D55000829F8001839F100D929F100D1124035F05
:10D560001C4480E290E0D80113969C938E9312970E
:10D5700082E01C968C93D7011496ED91FC9115973F
:10D58000ED58F84F81919191D8011E969C938E93FE
:10D590001D97D7018C9190E02091E4033091E50331
:10D5A000822B932BD80150969C938E931F972081AA
:10D5B000E557F7402A3020F5E958F84F408150E010
:10D5C000425E5F4F11965C934E934E5150408DE3F7
:10D5D00051968C9351975B965C934E935A975996BC
:10D5E0002C935997829158968C939801245E3F4FC3
:10D5F000E656FF4FC901BF0150E00E941CF00CC06D
:10D600008DE190E0F8019183808386E2818B81E057
:10D6100090E0918F808F228FD7011496ED91FC912D
:10D620001597E858F84F80819181A281B381F80164
:10D63000828B938BA48BB58B808191814A97978B3A
:10D64000868B80919507833020F48F5F80939507B8
:10D6500002C01092950790919507809196079817B0
:10D6600041F4933020F49F5F9093960702C010928C
:10D67000960780915119909152190E9436270F9068
:10D68000CF91DF911F910F91FF90EF9008950F932D
:10D690001F93DF93CF930F92CDB7DEB78C01198222
:10D6A000809151199091521960E070E0AE014F5F86
:10D6B0005F4F0E94C2288091930790E026E331E0FB
:10D6C000829FD001839FB00D929FB00D1124A35A69
:10D6D000B645FD01C90111920197E9F781E190E09A
:10D6E00011969C938E93F80184819581865A994F67
:10D6F000FC0190818CE1989FF0011124799611969C
:10D70000FC93EE9382E090E013969C938E93129795
:10D7100081E91C968C931C9771971E96FC93EE934F
:10D720001D97AD01415F5F4FD80114962D913C913B
:10D7300015972D5A394FCA01B901AF010E941CF04B
:10D7400080919307873020F48F5F8093930702C006
:10D75000109293079091930780919407981741F442
:10D76000973020F49F5F9093940702C01092940723
:10D7700080915119909152190E94362780E00F90A4
:10D78000CF91DF911F910F9108950F931F93DF9316
:10D79000CF930F92CDB7DEB78C01198280915119CA
:10D7A0009091521960E070E0AE014F5F5F4F0E94B0
:10D7B000C2288091930790E026E331E0829FD00158
:10D7C000839FB00D929FB00D1124A35AB645FD0161
:10D7D000C90111920197E9F781E190E011969C93BC
:10D7E0008E93F801848195818E599A4FFC01908126
:10D7F00088E1989FF001112479961196FC93EE939D
:10D8000082E090E013969C938E93129781E91C9688
:10D810008C931C9771971E96FC93EE931D97AD0108
:10D82000415F5F4FD80114962D913C911597255A71
:10D830003A4FCA01B901AF010E941CF080919307D1
:10D84000873020F48F5F8093930702C01092930774
:10D850009091930780919407981741F4973020F4A2
:10D860009F5F9093940702C0109294078091511982
:10D87000909152190E94362780E00F90CF91DF914E
:10D880001F910F9108950F931F93CF93DF938C01F6
:10D89000EB016F36710510F080E013C0DC011296C9
:10D8A0008D919C911397805B9F4F0E94D637D80132
:10D8B0001496ED91FC911597E05EF64FD183C083ED
:10D8C0008FEFDF91CF911F910F9108950F931F93C9
:10D8D000CF93DF938C01EB0188EA613C780710F06D
:10D8E00080E013C0D80112968D919C911397895BAB
:10D8F0009F4F0E94D637D8011496ED91FC91159751
:10D90000E75EF64FD183C0838FEFDF91CF911F91F8
:10D910000F9108950F931F93CF93DF938C01EB0129
:10D920006115710511F4C2E0D0E0CE0101978F5F5F
:10D930009E4F10F080E014C0D80112968D919C91FA
:10D9400013978C5B9F4FBE010E94D637D801149667
:10D95000ED91FC911597ED5FFA4FD183C0838FEF66
:10D96000DF91CF911F910F9108951F93CF93DF9374
:10D97000EC01162F862F81508A3010F080E00EC007
:10D980008A819B818E5B9F4F70E00E94D637EC812D
:10D99000FD81ED5FFA4F108311828FEFDF91CF9100
:10D9A0001F910895CF93DF93EC01EC81FD81E95A3B
:10D9B000FA4F11921082898160E040E00E94A23803
:10D9C000EC81FD81EE59FA4F8081E256F5408823C3
:10D9D000A1F0E55AFA4F80E790E0A0E0B0E0819333
:10D9E0009193A193B1938091E60381938881819370
:10D9F00088E48083CE010E94C56BEC81FD81E65AEC
:10DA0000F94F8081EA55F6408823A1F0ED5AF94F8D
:10DA100080E790E0A0E0B0E081939193A193B1936F
:10DA20008091E60381938881819389E48083CE018C
:10DA30000E94476BEC81FD81EE59FA4F108280E025
:10DA4000DF91CF9108959F92AF92BF92CF92DF92D4
:10DA5000EF92FF920F931F93DF93CF93CDB7DEB773
:10DA600027970FB6F894DEBF0FBECDBF5C011982B9
:10DA7000FE01329686E0DF011D928A95E9F7F501F5
:10DA80008481958180509F4FFC0186E1DF011D92CA
:10DA90008A95E9F7D5011496ED91FC911597E05020
:10DAA000FF4F1082CC24DD247E010894E11CF11C80
:10DAB00024C0F5010481158181816CE070E0A7012B
:10DAC0000E94B8320C0D1D1D00501F4FD8018C93C1
:10DAD000992D9F5FD5011496ED91FC911597EC0D52
:10DAE000FD1DE050FF4F80818A3061F00894C11C19
:10DAF000D11CB6E1CB16D10429F09C2C8981882356
:10DB0000C1F204C0992EE6E19E1721F0F1E19F16C3
:10DB100009F078C1D5011496CD90DC901597F601E7
:10DB2000E90DF11DE150FF4F80818A3009F06AC193
:10DB30009601265A394FF901808190E06CE1E62E7A
:10DB4000F12C8E9DF0018F9DF00D9E9DF00D112406
:10DB5000EC0DFD1DE55AF94F8091E5B79091E6B7C0
:10DB6000A091E7B7B091E8B780839183A283B38394
:10DB7000D9018C9190E08E9DF0018F9DF00D9E9DBE
:10DB8000F00D1124EC0DFD1DE15AF94F8091E9B71C
:10DB90009091EAB7A091EBB7B091ECB780839183F5
:10DBA000A283B383F901008110E00E943C340E9DF2
:10DBB00090010F9D300D1E9D300D1124C20ED31EFD
:10DBC00023E636E0C20ED31ED6016D937D938D936E
:10DBD0009C9313979E012E5F3F4F86E0F9011192AF
:10DBE0008A95E9F7F501A481B581F901A050BF4FED
:10DBF00085E00D9001928150E1F7D50114960D91C9
:10DC00001C911597065A194FF801E0800A551640E5
:10DC1000FF2452E0C52ED12CCC0EDD1EC60160E0E3
:10DC200070E040E150E00E942AEE2CE130E0A901D2
:10DC3000E49E9001E59E300DF49E300D1124020FFC
:10DC4000131F0959194FD8016D937D938D939C93A0
:10DC5000139786E0F60111928A95E9F7D50114969B
:10DC6000ED91FC911597D601EB5FFE4F85E0019099
:10DC70000D928150E1F7F50104811581065A194F83
:10DC8000D801EC900A551640FF2442E0C42ED12C56
:10DC9000CC0EDD1EC60160E070E040E150E00E9465
:10DCA0002AEE2CE130E0F901EE9E9001EF9E300D5E
:10DCB000FE9E300D1124020F131F0559194FD80174
:10DCC0006D937D938D939C93139786E0F60111924B
:10DCD0008A95E9F7D5011496ED91FC911597D60137
:10DCE000E65FFE4F85E001900D928150E1F7F5016E
:10DCF00004811581065A194FD801EC900A55164037
:10DD0000FF2432E0C32ED12CCC0EDD1EC60160E014
:10DD100070E040E150E00E942AEE0894E11CF11C02
:10DD20004CE150E0E49E9001E59E300DF49E300DF4
:10DD30001124020F131F0D5A194FF80160837183CC
:10DD400082839383D5011496ED91FC911597B6E1EA
:10DD50009B16A1F586E0D6011D928A95E9F7D601BA
:10DD6000E15FFE4F85E001900D928150E1F7F501F2
:10DD700004811581065A194FD801EC900A551640B6
:10DD8000FF24CE01029660E070E040E150E00E9486
:10DD90002AEE2CE130E0F901EE9E9001EF9E300D6D
:10DDA000FE9E300D1124020F131F0D58194FD8017C
:10DDB0006D937D938D939C9313971AC0E65AF94FF8
:10DDC0008081EA55F64090E09C01249FC001259F88
:10DDD000900D349F900D1124E80FF91FED58F94F65
:10DDE0008FEF9FEFAFEFBFEF80839183A283B38369
:10DDF000D5011496ED91FC911597E65AF94F808163
:10DE00008F5F08C0D5011496ED91FC911597E65AE5
:10DE1000FA4F8FEF808327960FB6F894DEBF0FBEC0
:10DE2000CDBFCF91DF911F910F91FF90EF90DF90C9
:10DE3000CF90BF90AF909F900895AF92BF92CF9236
:10DE4000DF92EF92FF920F931F93DF93CF93CDB7A3
:10DE5000DEB727970FB6F894DEBF0FBECDBF5C01CB
:10DE60001982FE01329686E0DF011D928A95E9F75C
:10DE7000F5018481958180509F4FFC0180E091E005
:10DE8000DF019C011D9221503040E1F7EE24FF2478
:10DE90006E010894C11CD11C1BC0D50114960D91B4
:10DEA0001C91159711968C916CE070E0A6010E9470
:10DEB000B8320E0D1F1D00501F4FF80180838E2DAC
:10DEC0008F5F0894E11CF11CF1E1EF16F10421F0E1
:10DED0008981882311F32CC1813109F029C1D50131
:10DEE0001496ED90FC901597E0E1F1E0EE0EFF1E28
:10DEF000D7018C91E0EFFEEFEE0EFF1E8A3009F0A5
:10DF000017C197012E593A4FD9018C9190E0FC012D
:10DF1000EE0FFF1FE80FF91F319613E0EE0FFF1F02
:10DF20001A95E1F7EE0DFF1DE55AFA4F8091E5B71E
:10DF30009091E6B7A091E7B7B091E8B7808391835D
:10DF4000A283B383F901808190E0FC01EE0FFF1FF3
:10DF5000E80FF91FA3E0EE0FFF1FAA95E1F7EE0D02
:10DF6000FF1DE959FA4F8091E9B79091EAB7A09166
:10DF7000EBB7B091ECB780839183A283B383D901CF
:10DF80000C9110E00E943C349801220F331F200FA7
:10DF9000311FE3E0220F331FEA95E1F7E20EF31E93
:10DFA000EBE6F5E0EE0EFF1ED7016D937D938D93AA
:10DFB0009C9313979E012E5F3F4F86E0F9011192CB
:10DFC0008A95E9F7F501A481B581F901A050BF4F09
:10DFD00085E00D9001928150E1F7D50114960D91E5
:10DFE0001C9115970E591A4FF801E0800256154002
:10DFF000FF2462E0C62ED12CCC0EDD1EC60160E0EF
:10E0000070E040E150E00E942AEE9701220F331F9A
:10E010002E0D3F1D43E0220F331F4A95E1F7020FFB
:10E02000131F01591A4FD8016D937D938D939C93C3
:10E03000139786E0F60111928A95E9F7D5011496B7
:10E04000ED91FC911597D601EB5FFE4F85E00190B5
:10E050000D928150E1F7F501048115810E591A4F97
:10E06000D801EC9002561540FF2482E0C82ED12C36
:10E07000CC0EDD1EC60160E070E040E150E00E9481
:10E080002AEE0894E11CF11C9701220F331F2E0D7C
:10E090003F1DA3E0220F331FAA95E1F7020F131FC4
:10E0A000055A1A4FF801608371838283938386E057
:10E0B000D6011D928A95E9F7D5011496ED91FC9150
:10E0C0001597D601E65FFE4F85E001900D928150D5
:10E0D000E1F7F501048115810E591A4FD801EC9032
:10E0E00002561540FF24CE01029660E070E040E148
:10E0F00050E00E942AEE9701220F331F2E0D3F1D84
:10E10000E3E0220F331FEA95E1F7020F131F0958CE
:10E110001A4FF8016083718382839383D50114962B
:10E12000ED91FC911597EE59FA4F80818F5F08C0F1
:10E13000D5011496ED91FC911597E65AFA4F8FEFA1
:10E14000808327960FB6F894DEBF0FBECDBFCF9168
:10E15000DF911F910F91FF90EF90DF90CF90BF90D4
:10E16000AF900895EF92FF920F931F93DF93CF9399
:10E170000F92CDB7DEB78C0119827E010894E11CA5
:10E18000F11C09C0F80181816CE070E0A7010E94D8
:10E19000B8328A3019F089818823A1F30F90CF918A
:10E1A000DF911F910F91FF90EF9008958F929F92B2
:10E1B000AF92BF92CF92DF92EF92FF920F931F9395
:10E1C000DF93CF930F92CDB7DEB76C011982DC01DC
:10E1D0001496ED90FC901597D7010D900020E9F76B
:10E1E0008D01015010400E191F09C80101978F3F82
:10E1F000910508F058C085E0B82E4E010894811CA6
:10E20000911C2EC0F6018181D7016C914AE050E04B
:10E210000E94F331882309F046C0F60181811982FA
:10E2200060E870E0A4010E94B832A82E898188239A
:10E2300051F0BB20C1F1BA9480E060E040E024E6F8
:10E2400030E00E942A2ED7018C91A81639F4089448
:10E25000E11CF11C01501040BB2402C0BB2019F18D
:10E260000115110579F6F60181816DE04AE050E073
:10E270000E94F3318823B9F4D60111968C9119824A
:10E280006AE070E08E010F5F1F4FA8010E94B83254
:10E29000F60181816AE070E0A8010E94B8328A30FC
:10E2A00011F48FEF01C080E00F90CF91DF911F91AB
:10E2B0000F91FF90EF90DF90CF90BF90AF909F9025
:10E2C0008F9008954F925F926F927F928F929F925C
:10E2D000AF92BF92CF92DF92EF92FF920F931F9374
:10E2E000DF93CF930F92CDB7DEB74C012B017A01AC
:10E2F000FC01048115811982CB010E94C6EFB82E62
:10E30000F70111821082F401818160E872E03E0120
:10E310000894611C711CA3010E94B83200501F4F69
:10E32000F80180830050114089818823F9F491E03D
:10E33000C92ED92EC00ED11EF70180819181019680
:10E3400091838083AB2CBB2486010A191B090F5FC4
:10E350001F4F28C0F401818160E470E0A3010E9496
:10E36000B832F60180838981882321F0F701118278
:10E3700010821EC00894C11CD11CF70180819181BC
:10E380000196918380838A159B0550F0C801B201E4
:10E39000A5010E94E7EF882311F48FEF0AC089835B
:10E3A0000F5F1F4FF701808191818050944090F260
:10E3B00080E00F90CF91DF911F910F91FF90EF9030
:10E3C000DF90CF90BF90AF909F908F907F906F9095
:10E3D0005F904F9008950F931F93DF93CF9300D0DA
:10E3E00000D0CDB7DEB78C010E943C346B837C83B8
:10E3F0008D839E83CE0103960E943235AC01D801F5
:10E4000014966C91149715967C91159780E091E085
:10E41000FB019C01119221503040E1F714968D913F
:10E420009C91159780509F4FBC0180E094E0DB01E8
:10E43000FC011D923197E9F72DB73EB720513040CE
:10E440000FB6F8943EBF0FBE2DBFEDB7FEB73196A5
:10E45000D80114968D919C911597ADB7BEB71296C1
:10E460009C938E9311978DED99E093838283DA01CB
:10E4700018968D919C911997019695838483169691
:10E480008D919C911797978386831A968D919C9175
:10E490001B978459984F9187808714968D919C91F2
:10E4A00015979387828712968D919C9113979587E4
:10E4B00084878D919C91978786870E9451F1EDB753
:10E4C000FEB770960FB6F894FEBF0FBEEDBFC80141
:10E4D0000E94D6708F3F41F4C80168E97AE0AE012E
:10E4E0004F5F5F4F0E94627126960FB6F894DEBFB1
:10E4F0000FBECDBFCF91DF911F910F910895AF92C5
:10E50000BF92DF92EF92FF920F931F93DF93CF930F
:10E510000F920F92CDB7DEB78C017B01CB010E9429
:10E520004FF0C7016AE67CE00E94F5EF892B19F4F1
:10E53000DD24DA940AC0D8011496ED91FC91159768
:10E54000EB58F84F84E18083DD24C70168E57CE067
:10E550000E94F5EF892B51F0D8011496ED91FC91B2
:10E560001597EB58F84F84E18083DD24C70162E5FD
:10E570007CE00E94F5EF892B51F0D8011496ED91C3
:10E58000FC911597EB58F84F84E18083DD24C70197
:10E590006AE47CE00E94F5EF892B51F0D8011496D3
:10E5A000ED91FC911597EB58F84F84E18083DD24C1
:10E5B000C70166E47CE00E94F5EF892B51F0D80199
:10E5C0001496ED91FC911597EB58F84F84E18083F8
:10E5D000DD24C70169E37CE00E94F5EF892B51F04F
:10E5E000D8011496ED91FC911597EB58F84F84E102
:10E5F0008083DD24C70161E37CE00E94F5EF892B75
:10E6000059F0D8011496ED91FC911597EB58F84FFD
:10E6100084E18083DD249DC0DD2009F49AC0A12C13
:10E6200021E0B22ED8011496EC9114971596FC9126
:10E63000DF0195011D9221503040E1F7D801149679
:10E640008D919C91159780509F4FFC0180E094E044
:10E65000DF019C011D9221503040E1F7D801149652
:10E660008D919C911597B7010E942CF0C8010E94D2
:10E67000D670D82EBFEF8B1709F06BC0C80168E9C0
:10E680007AE0AE014F5F5F4F0E946271D82EEFEFCC
:10E690008E1709F05EC089819A81892B09F459C0CF
:10E6A000D80114968D919C911597805F974FDC014E
:10E6B00095011D9221503040E1F7E980FA80D801A0
:10E6C0001496ED91FC911597B1E0EB16B1E0FB06C5
:10E6D00090F4EB58F84F81E08083F8012481358174
:10E6E000A901405F574F20503F4FCA01B901A70110
:10E6F0000E941CF01CC0EB58F84F82E08083D801C8
:10E7000014968D919C911597DC01A05FB74FFC0189
:10E71000E050FF4F8FEF01900D928150E1F7D8014B
:10E720001496ED91FC911597E15FF64F1082D80198
:10E730001496ED91FC911597CF01805F974FDC0106
:10E740000D900020E9F71197A81BB90BE958F84F75
:10E75000A0838D2D0F900F90CF91DF911F910F917E
:10E76000FF90EF90DF90BF90AF900895CF92DF922F
:10E77000FF920F931F93DF93CF930F920F92CDB71A
:10E78000DEB78C016B01CB01019780519E4010F0E8
:10E79000FF2467C0D80114968C91149715969C910C
:10E7A0001A821982FC0180E091E0DF019C011D9238
:10E7B00021503040E1F7D80114968D919C91159726
:10E7C00080509F4FFC0180E094E0DF019C011D928E
:10E7D00021503040E1F700D000D0EDB7FEB73196C0
:10E7E000D80114968D919C911597ADB7BEB712962E
:10E7F0009C938E93119788E49AE093838283758328
:10E8000064830E9451F1EDB7FEB736960FB6F894C7
:10E81000FEBF0FBEEDBFC8010E94D670F82EFFEFFD
:10E820008F17F9F4C80168E97AE0AE014F5F5F4FD6
:10E830000E946271F82E2FEF821799F4D801129678
:10E840008D919C911397805C9F4FB6010E94D637A3
:10E85000D8011496ED91FC911597EF5FFA4FD18294
:10E86000C0828F2D0F900F90CF91DF911F910F914C
:10E87000FF90DF90CF900895EF92FF920F931F9338
:10E88000DF93CF930F920F92CDB7DEB77C011A8240
:10E890001982DC0114960D911C9115970E591A4F8F
:10E8A000F80110820B501040D8011C9207551540FA
:10E8B00080E091E0F8019C01119221503040E1F795
:10E8C000D70114968D919C91159780509F4FFC0114
:10E8D00080E094E0DF019C011D9221503040E1F77F
:10E8E000D70114968D919C9115976AE87AE00E9461
:10E8F000B4EFF80101900020E9F73197E01BF10B2C
:10E90000FA83E98311C0F7018181D8016C914AE053
:10E9100050E00E94F331882359F489819A8101974C
:10E920009A8389830F5F1F4F89819A81892B59F7B9
:10E93000F70181816DE04AE050E00E94F331C701A8
:10E9400068E97AE0AE014F5F5F4F0E946271D701C4
:10E950001496ED91FC911597EE5DF64F8FEF808345
:10E960000F900F90CF91DF911F910F91FF90EF903B
:10E9700008950F931F93DF93CF930F920F92CDB70C
:10E98000DEB78C011A821982DC011496EC9114977F
:10E990001596FC9180E091E0DF019C011D922150D1
:10E9A0003040E1F7D80114968D919C9115978050D5
:10E9B0009F4FFC0180E094E0DF019C011D922150FB
:10E9C0003040E1F7D80114968D919C9115976FE82E
:10E9D0007AE00E94B4EFC8010E94D670982F8F3F52
:10E9E00049F4C80168E97AE0AE014F5F5F4F0E94C9
:10E9F0006271982FD8011496ED91FC911597EE5DF8
:10EA0000F64F8FEF8083892F0F900F90CF91DF917A
:10EA10001F910F910895EF92FF920F931F93DF9331
:10EA2000CF930F920F92CDB7DEB77C011A82198275
:10EA3000DC0114960D911C9115970E591A4FF8018F
:10EA40008081025615408823D1F0055A1A4F80E77D
:10EA500090E0A0E0B0E0F80181939193A193B1938D
:10EA60008091E603DF018D93F70180818D938D0105
:10EA700088E48C9301561540C7010E94C56BD701ED
:10EA80001496ED91FC911597E65AF94F8081EA555D
:10EA9000F6408823A9F0ED5AF94F80E790E0A0E016
:10EAA000B0E081939193A193B1938091E603819318
:10EAB000D7018C91819389E48083C7010E94476BC1
:10EAC000D7011496ED91FC911597EE59FA4F1082EB
:10EAD0003B971082E755F54080E091E09C01119250
:10EAE00021503040E1F7D70114968D919C911597F4
:10EAF00080509F4FFC0180E094E0DF019C011D925B
:10EB000021503040E1F7D70114968D919C911597D3
:10EB10006AE87AE00E94B4EFF80101900020E9F77A
:10EB20003197E01BF10BFA83E98320E012C0F70173
:10EB30008181D8016C914AE050E00E94F331882332
:10EB400009F589819A8101979A8389830F5F1F4F05
:10EB50002FEF89819A81892B51F72F3FA1F4F7017B
:10EB600081816DE04AE050E00E94F331882351F446
:10EB7000C70168E97AE0AE014F5F5F4F0E946271A2
:10EB8000282F01C020E0D7011496ED91FC91159734
:10EB9000EE5DF64F1082822F0F900F90CF91DF9194
:10EBA0001F910F91FF90EF900895EF92FF920F93B6
:10EBB0001F93DF93CF930F920F92CDB7DEB78C01E7
:10EBC000DC011496EC9114971596FC9180E091E08D
:10EBD000DF019C011D9221503040E1F7D8011496CD
:10EBE0008D919C91159780509F4FFC0180E094E09F
:10EBF000DF019C011D9221503040E1F7D8011496AD
:10EC00008D919C9115976AEC79E00E94B4EFC80150
:10EC10000E94D6708F3F29F5C80168E97AE0AE01FD
:10EC20004F5F5F4F0E9462718F3FD9F489819A8153
:10EC3000892BB9F0F80104811581E12C31E0F32E24
:10EC4000E00EF11EC70169EA7AE00E94F5EF009735
:10EC500041F08E159F0529F0075A1A4F81E0D8011F
:10EC60008C930F900F90CF91DF911F910F91FF9098
:10EC7000EF9008950F931F93DF93CF930F920F920E
:10EC8000CDB7DEB78C011A8219820E943C74C8018C
:10EC90000E94D575D8011496ED91FC911597EF5F00
:10ECA000FA4F60817181C8010E94B673D801149631
:10ECB000ED91FC911597EE59FA4F10823B978FEF2B
:10ECC0008083E755F54080E091E09C01119221504E
:10ECD0003040E1F7D80114968D919C9115978050A2
:10ECE0009F4FFC0180E094E0DF019C011D922150C8
:10ECF0003040E1F7D80114968D919C91159764E806
:10ED00007AE00E94B4EFC8010E94D6708F3F41F4B0
:10ED1000C80168E97AE0AE014F5F5F4F0E946271FF
:10ED2000D8011496ED91FC911597EE5DF64F108287
:10ED30000F900F90CF91DF911F910F910895BF9287
:10ED4000CF92DF92EF92FF920F931F93DF93CF93B7
:10ED50000F920F92CDB7DEB77C01DC0114968D9136
:10ED60009C9115978458984FFC0184E1DF011D9216
:10ED70008A95E9F7F701848195818458984F61EA73
:10ED80007AE00E94B4EFD7011496EC91149715968F
:10ED9000FC9180E091E0DF019C011D922150304008
:10EDA000E1F7D70114968D919C91159780509F4F54
:10EDB000FC0180E094E0DF019C011D922150304075
:10EDC000E1F7D70114968D919C9115976EEB79E040
:10EDD0000E94B4EFC7010E94D670B82EBFEF8B1708
:10EDE00009F085C0C70168E97AE0AE014F5F5F4F67
:10EDF0000E946271B82EEFEF8E1709F078C08981FA
:10EE00009A81892B09F473C0D70114960D911C9136
:10EE10001597C12C41E0D42EC00ED11EC6016CEB5B
:10EE20007AE00E94F5EF009741F08C159D0529F0DE
:10EE3000075A1A4F81E0F8018083D7011496CD90CC
:10EE4000DC901597860100501F4FC8016EE97AE0EB
:10EE50000E94F5EF009709F44AC001966EE97AE046
:10EE60000E94F5EF009709F442C0FC01E01BF10B92
:10EE7000E034F105E0F59601295E3A4FC901B80189
:10EE8000AF010E941CF0F70184819581895E9A4F41
:10EE90000E9467F0D7011496CD90DC9015978601FB
:10EEA000095E1A4FC80164E07DE00E94F5EF00970B
:10EEB000A9F0FC01E01BF10BE031F10578F49601BB
:10EEC000295F3A4FC901B801AF010E941CF0F70158
:10EED00084819581895F9A4F0E9467F0D7011496CB
:10EEE0008D919C911597895E9A4F0E9467F08B2DAA
:10EEF0000F900F90CF91DF911F910F91FF90EF90A6
:10EF0000DF90CF90BF900895CF92DF92EF92FF9263
:10EF10000F931F93DF93CF930F920F92CDB7DEB76E
:10EF20008C011A821982DC011496ED91FC911597DF
:10EF3000E95AFA4F119210823A96108211968C91EA
:10EF40006FEF40E00E94A23853E0E52E6E01089476
:10EF5000C11CD11C80E060E041E020E030E00E9474
:10EF60002A2EF80181816DE04AE050E00E94F331E1
:10EF7000C80168E97AE0A6010E946271F82EFFEFED
:10EF80008F1771F0EA9431F78F2D0F900F90CF917A
:10EF9000DF911F910F91FF90EF90DF90CF90089538
:10EFA000C8010E949F7680E060E040E024E630E007
:10EFB0000E942A2ED8011496ED91FC911597E85ADB
:10EFC000FA4FF082E1CF8F929F92AF92BF92CF9291
:10EFD000DF92EF92FF920F931F93DF93CF9300D0B6
:10EFE0000F92CDB7DEB75C01062F5C834B831A828C
:10EFF0001982DC0114968D919C9115978458984F35
:10F00000FC0184E1DF011D928A95E9F7F501848115
:10F0100095818458984F68E372E00E94B4EF602FA6
:10F0200070E0FB01E154F040EA33F10508F0CDC295
:10F03000EE58FF4FEE0FFF1F0590F491E02D19944D
:10F04000C5010E948477C1C2C5010E94D26CC0C0B4
:10F05000D5011496ED91FC911597E85AFA4F8081ED
:10F06000882319F4C5010E948477D5011496ED9187
:10F07000FC911597E95AFA4F80818F3F51F4C501F1
:10F080000E940B7580E060E041E020E030E00E94EB
:10F090002A2EF501848195818458984FFC0184E1E2
:10F0A000DF011D928A95E9F7F501848195818458E5
:10F0B000984F68E372E00E94B4EFD50114966D9109
:10F0C0007C9115976458784F8E010D5F1F4F8B818F
:10F0D0009C81A8010E94A0F09A838983EE244E01AE
:10F0E0000894811C911CD02E012F29C0B40140E04E
:10F0F00050E00E942AEEB1E0EB1651F0EB1620F042
:10F10000E2E0EE1661F408C0C5010E94B67307C0C4
:10F11000C5010E94B56C03C0C5010E948A6CE394CE
:10F12000D50114966D917C9115976458784F80E0C5
:10F1300090E04D2D502F0E94A0F09A838983898101
:10F140009A81009719F0B3E0EB1681F6C5010E9491
:10F15000EB71F501C480D58029E139E0C20ED31EE0
:10F16000D6014D915C91E7EEF6EFCE0EDF1E411514
:10F17000510539F1F601ED5FFA4F21E035E0C20E9D
:10F18000D31ED6012D913C9180819181289F7001E1
:10F19000299FF00C389FF00C1124E40EF51E00E0BE
:10F1A00010E00E942334EAE1F4E0CE0EDF1EE60E0A
:10F1B000F71E081F191FD601ED92FD920D931C93A7
:10F1C0001397C5010E943A7600C2C5010E940B75D3
:10F1D000D5011496ED91FC911597E15EF64F1082E2
:10F1E000F4C1D5011496ED91FC911597E85AFA4FA8
:10F1F0008081882319F4C5010E948477F5018481F8
:10F2000095818458984FFC0184E1DF011D928A9515
:10F21000E9F7F501848195818458984F68E372E09D
:10F220000E94B4EFD50114966D917C9115976458A6
:10F23000784F89819A81AE014D5F5F4F0E94A0F0A7
:10F240009A838983009709F4C0C1BE016F5F7F4F25
:10F2500040E050E00E942AEE9B01AC01C501B901DB
:10F260000E94B673B2C1F501848195818458984F8C
:10F27000FC0184E1DF011D928A95E9F7F5018481A3
:10F2800095818458984F68E372E00E94B4EFD501ED
:10F2900014966D917C9115976458784F89819A8165
:10F2A000AE014D5F5F4F0E94A0F09A838983009763
:10F2B00009F48BC1BE016F5F7F4F40E050E00E94B8
:10F2C0002AEEC5010E94B56C80C1F501848195814B
:10F2D0008458984FFC0184E1DF011D928A95E9F77B
:10F2E000F501848195818458984F68E372E00E940B
:10F2F000B4EFD50114966D917C9115976458784FB1
:10F3000089819A81AE014D5F5F4F0E94A0F09A8380
:10F310008983009709F459C1BE016F5F7F4F40E0B8
:10F3200050E00E942AEE9B01AC01C501B9010E9488
:10F330008A6C4BC1D5011496ED91FC911597E85A52
:10F34000FA4F8081882319F4C5010E948477C50192
:10F350000E94586A082FD5011496ED91FC911597DB
:10F36000EB58F84F81E0BDC0F50184819581845848
:10F37000984FFC0184E1DF011D928A95E9F7F501C0
:10F38000848195818458984F68E372E00E94B4EFBD
:10F39000D50114966D917C9115976458784F8981A9
:10F3A0009A81AE014D5F5F4F0E94A0F09A838983DE
:10F3B000009709F40AC160E070E040E050E00E946C
:10F3C0002AEE9B01AC01C501B9010E94666CFDC02B
:10F3D000F501848195818458984FFC0184E1DF0117
:10F3E0001D928A95E9F7F501848195818458984F9B
:10F3F00068E372E00E94B4EFD50114966D917C91A0
:10F4000015976458784F89819A81AE014D5F5F4F9F
:10F410000E94A0F09A838983009709F4D6C060E027
:10F4200070E040E050E00E942AEE9B01AC01C50173
:10F43000B9010E94436CC9C0D5011496ED91FC91AD
:10F440001597E85AFA4F8081882311F000E00BC02D
:10F45000C5010E948477082F80E060E042E020E050
:10F4600030E00E942A2ED5011496ED91FC9115975B
:10F47000E95AFA4F8081E755F5408823A1F5CF017D
:10F480008458984FFC0184E1DF011D928A95E9F7C9
:10F49000F501848195818458984F68E372E00E9459
:10F4A000B4EFD50114966D917C9115976458784FFF
:10F4B0008B819C81AE014D5F5F4F0E94A0F0BC012B
:10F4C000009739F09A838983C5010E947F72082FC3
:10F4D00081C0D5011496ED91FC911597EB58F84F2A
:10F4E0008DE0808377C0EB58F84F8BE0FACFF501C1
:10F4F000848195818458984FFC0184E1DF011D923D
:10F500008A95E9F7F501848195818458984F68E3DD
:10F5100072E00E94B4EFD50114966D917C9115971D
:10F520006458784F8B819C81AE014D5F5F4F0E9484
:10F53000A0F0FC01009709F448C080818F3611F0DB
:10F540008F3431F48181863611F0863409F480835A
:10F5500080818F34D9F0803560F48133B9F0823303
:10F5600018F4803391F51CC08634D1F08E3469F5DF
:10F5700017C08E36A9F08F3628F4893539F08636D3
:10F5800021F50EC08F3611F08937F9F4D5011496A4
:10F59000ED91FC911597E050FB4F81E0808308C00E
:10F5A000D5011496ED91FC911597E050FB4F108218
:10F5B000F501828193810480F581E02DE050FB4FBD
:10F5C000875B9F4F60810E949F37C5016FEF0E944C
:10F5D00044690FEF802F0F900F900F900F90CF91F5
:10F5E000DF911F910F91FF90EF90DF90CF90BF9030
:10F5F000AF909F908F900895BF92CF92DF92EF923D
:10F60000FF920F931F93DF93CF930F920F92CDB77B
:10F61000DEB76C01B62E1A82198221E0621729F03A
:10F6200032E0631709F0D9C110C0DC018C9190E081
:10F6300029E031E0FC01E29FC001E39F900DF29FC1
:10F64000900D11248E58924605C0DC019C9180E0FB
:10F650008F5A96479A838983E981FA81E150FF4F57
:10F660001082F601848195818458984FFC0184E1D1
:10F67000DF011D928A95E9F7F6018481958184580E
:10F68000984F68E372E00E94B4EFD60114966D9132
:10F690007C9115976458784F89819A817E010894EE
:10F6A000E11CF11CA7010E94A0F08C01009759F108
:10F6B00082E19CE00E94C6EFAC01C80162E17CE0FF
:10F6C0000E94CFEF892B09F04DC0D6011496ED9121
:10F6D000FC911597E458F84FC7016AEA7BE048E0CF
:10F6E0002DE006E11CE07F010E941F38682F88236F
:10F6F00009F06AC167C08230A9F1833009F462C0A1
:10F70000813009F08EC0B1E0BB1649F4D6011496E1
:10F71000ED91FC911597EB58F84F8DE02EC0F60156
:10F720002181922F990F990F80E08F5A9247FC0107
:10F7300080E091E0DF019C011D9221503040E1F713
:10F7400000D00F92D60111962C91922F990F990FFC
:10F7500080E08F5A9247EDB7FEB7928381838AEE9D
:10F760009CE08DC0F1E0BF1651F4D6011496ED91E6
:10F77000FC911597EB58F84F8EE08083A8C0F601F6
:10F780002181922F990F990F80E08F5A9247FC01A7
:10F7900080E091E0DF019C011D9221503040E1F7B3
:10F7A00000D00F92D60111962C91922F990F990F9C
:10F7B00080E08F5A9247EDB7FEB79283818383EC46
:10F7C0009CE05DC0F1E0BF1649F4D6011496ED91BE
:10F7D000FC911597EB58F84F8AE0CFCFF6012181C5
:10F7E000922F990F990F80E08F5A9247FC0180E089
:10F7F00091E0DF019C011D9221503040E1F700D0E3
:10F800000F92D60111962C91922F990F990F80E0AB
:10F810008F5A9247EDB7FEB7928381838EEA9CE0C0
:10F820002EC0F1E0BF1649F4D6011496ED91FC917B
:10F830001597EB58F84F8FE0A0CFF6012181922F5A
:10F84000990F990F80E08F5A9247FC0180E091E078
:10F85000DF019C011D9221503040E1F700D00F9252
:10F86000D60111962C91922F990F990F80E08F5A03
:10F870009247EDB7FEB7928381838FE99CE0948332
:10F8800083830E9451F1F601A181FA2FFF0FFF0F30
:10F89000E0E09F012F5A3247F90101900020E9F77B
:10F8A000CF010197821B930BB0E0AA0FBB1FAF5A89
:10F8B000B2468D939C930F900F900F900F90F1E0B4
:10F8C000BF1629F022E0B21609F087C004C0C601B5
:10F8D0000E948D6A2AC0D6011496ED91FC9115976D
:10F8E00011968C91382F330F330F20E02F5A324767
:10F8F000E958F84F4081E756FF4FC901BF0150E07A
:10F900000E941CF0F601A181B0E0AA0FBB1FAF5A04
:10F91000B246848195818958984FFC0180818C93EF
:10F9200011961C92C6010E942868D6018C9190E025
:10F9300029E031E0FC01E29FC001E39F900DF29FBE
:10F94000900D11248E589246FC0180E091E0DF0179
:10F95000AC011D9241505040E1F7D6018C9190E0EE
:10F96000829FF001839FF00D929FF00D1124E759C3
:10F97000F246118210828C9190E0829FF001839F69
:10F98000F00D929FF00D1124E759F24612828C91EE
:10F9900090E0829FF001839FF00D929FF00D112463
:10F9A000E759F246148213828C9190E0829FF00115
:10F9B000839FF00D929FF00D1124E759F2461582B6
:10F9C00016821782108609C049815A81C6010E9499
:10F9D000E3778F3F09F08FCE72CF0F900F90CF91CA
:10F9E000DF911F910F91FF90EF90DF90CF90BF902C
:10F9F0000895CF92DF92EF920F931F93DF93CF93EF
:10FA000000D00F92CDB7DEB76C01DC0111968C915E
:10FA10001197813019F480E093E00DC0823031F409
:10FA200080E095E0F6019383828309C0833039F446
:10FA300080E097E0D60113969C938E931297D6019F
:10FA40001496ED91FC911597309741F080EA9FE074
:10FA5000DF019C011D9221503040E1F7D601119643
:10FA60008C9140E855E260E070E026E000E0EE2492
:10FA70000E943833D6011496ED91FC911597EF5FF3
:10FA8000FA4F0CE310E0019311938AE090E0819328
:10FA9000919382E090E091838083EC5AFF4F119222
:10FAA0001082E853FC4F108212962D913C911397CF
:10FAB0002115310509F40AC18FEF9FEF9A838983DD
:10FAC000C901805C9F4FBE016F5F7F4F0E944D3721
:10FAD00089819A81019780519E4058F01A83098349
:10FAE000F60182819381805C9F4F6CE370E00E94FD
:10FAF000D637D6011496ED91FC911597EF5FFA4F2A
:10FB000089819A81918380838FEF9FEF9A83898384
:10FB100012968D919C9113978E5B9F4FBE016F5FE4
:10FB20007F4F0E944D3789819A8101978E5F9F4F49
:10FB300068F08AE090E09A838983F601828193815C
:10FB40008E5B9F4F6AE070E00E94D637D601149614
:10FB5000ED91FC911597ED5FFA4F89819A81918320
:10FB600080838FEF9FEF9A83898312968D919C916A
:10FB700013978C5B9F4FBE016F5F7F4F0E944D3785
:10FB800089819A8101978E5F9F4F68F082E090E0B3
:10FB90009A838983F601828193818C5B9F4F62E017
:10FBA00070E00E94D637D6011496ED91FC9115971E
:10FBB000EB5FFA4F89819A81918380838FEF9FEF6A
:10FBC0009A83898312968D919C911397895B9F4F9D
:10FBD000BE016F5F7F4F0E944D3789819A81815CA2
:10FBE000984A58F01A821982F60182819381895BC2
:10FBF0009F4F60E070E00E94D637D6011496ED91D9
:10FC0000FC911597E75EF64F89819A8191838083F5
:10FC1000E951F4408FEF808312968D919C91139758
:10FC2000875B9F4FBF010E943837D6011496ED9134
:10FC3000FC911597E050FB4F8081823050F010828C
:10FC400012968D919C911397875B9F4F60E00E9465
:10FC50009F378FEF9FEF9A838983F601828193818B
:10FC6000805B9F4FBE016F5F7F4F0E944D37898140
:10FC70009A818F36910568F01A821982D601129600
:10FC80008D919C911397805B9F4F60E070E00E9484
:10FC9000D637D6011496ED91FC911597E05EF64F9C
:10FCA00089819A8191838083E052F4408081813000
:10FCB00069F480913204909133049C838B83C60154
:10FCC00062E7AE014D5F5F4F0E94E3778FEF0F90C9
:10FCD0000F900F900F90CF91DF911F910F91EF90A8
:10FCE000DF90CF9008958FEF80939EA181E060E038
:10FCF00040E020E030E00E942A2EF8CF8F929F92C1
:10FD0000AF92BF92CF92DF92EF92FF920F931F9329
:10FD1000DF93CF93CDB7DEB762970FB6F894DEBF0F
:10FD20000FBECDBF4C015A016B0119828091511950
:10FD30009091521960E070E0AE014F5F5F4F0E94FA
:10FD4000C2288091930790E026E331E0829F8001F2
:10FD5000839F100D929F100D1124035A16458AE5BA
:10FD6000D8011D928A95E9F78CE590E0F80191831E
:10FD7000808385E090E09383828380E684870E947D
:10FD80003C346A837B838C839D83D4011196EC91F0
:10FD9000F0E0EE0FFF1FEF5AF24680819181A0E064
:10FDA000B0E0F801828F938FA48FB58F92E0E92E97
:10FDB000F12CEC0EFD1EC7010E943235FC0186813C
:10FDC000D80192968C93929784815E968C935E97DD
:10FDD00082815F968C935F9780858F5F91968C93DD
:10FDE0009197808190968C93909782858456939674
:10FDF0008C93C7010E943235FC018681D801989608
:10FE00008C939897848194968C93949782819596FD
:10FE10008C93959780858F5F97968C939797808129
:10FE200096968C9396978285845699968C939997FB
:10FE30009A961C92C801CF9620E1DC01822F1D9278
:10FE40008A95E9F7C8018D96DC011D922A95E9F79C
:10FE5000F80116AE15AE14A613A6D40111968C9116
:10FE600090E02091E4033091E503822B932B968759
:10FE70008587EDB7FEB738970FB6F894FEBF0FBE73
:10FE8000EDBF319686E0E82EF12CEC0EFD1EADB7ED
:10FE9000BEB71296FC92EE92119784E394E093839E
:10FEA0008283A482B582C682D7820E942DF1EDB7EB
:10FEB000FEB738960FB6F894FEBF0FBEEDBFC8016F
:10FEC0000F96B7010E94873E80919307873020F4F8
:10FED0008F5F8093930702C01092930790919307CE
:10FEE00080919407981741F4973020F49F5F909386
:10FEF000940702C010929407809151199091521961
:10FF00000E94362780E062960FB6F894DEBF0FBEDF
:10FF1000CDBFCF91DF911F910F91FF90EF90DF90B8
:10FF2000CF90BF90AF909F908F900895FF920F93C6
:10FF30001F93CF93DF938C016EE374E043E050E0B6
:10FF40000E9459F0EC01C80162E474E043E050E023
:10FF50000E9459F0009719F492E0F92E05C0FF2491
:10FF6000CD2B11F4FF24F394C80166E474E043E060
:10FF700050E00E9459F0009711F483E0F82EC80178
:10FF80006AE474E043E050E00E9459F0009711F4F5
:10FF9000B4E0FB2EC8016EE474E043E050E00E9440
:10FFA00059F0009711F4A5E0FA2EC80162E574E05B
:10FFB00043E050E00E9459F0009711F4F6E0FF2E64
:10FFC000C80166E574E043E050E00E9459F00097F4
:10FFD00011F4E7E0FE2EC8016AE574E043E050E06A
:10FFE0000E9459F0009711F478E0F72EC8016EE5F1
:10FFF00074E043E050E00E9459F0009711F469E08A
:020000021000EC
:10000000F62EC80162E674E043E050E00E9459F029
:10001000009711F45AE0F52EC80166E674E043E05B
:1000200050E00E9459F0009711F44BE0F42EC80103
:100030006AE674E043E050E00E9459F0009711F442
:100040003CE0F32E8F2DDF91CF911F910F91FF9008
:100050000895EF92FF920F931F93DF93CF930F9228
:10006000CDB7DEB77C011982809151199091521958
:1000700060E070E0AE014F5F5F4F0E94C228809148
:10008000950790E026E331E0829F8001839F100D69
:10009000929F100D1124035F1C4480E290E0D80170
:1000A00013969C938E93129782E01C968C93D701A3
:1000B0001496ED91FC911597E156FA4F819191912B
:1000C000D8011E969C938E931D97D7018C9190E03A
:1000D0002091E4033091E503822B932BD8015096B5
:1000E0009C938E931F972081E15AF5402A3098F512
:1000F000ED55FA4F408150E0425E5F4F11965C93A0
:100100004E934E5150408DE351968C9351975B9690
:100110005C934E935A9759962C935997829158967F
:100120008C939801245E3F4F7A96C901BF0150E03D
:100130000E941CF0D7011496ED91FC91159723EFC6
:1001400038E1ED55FA4F40817996C901BF0150E081
:100150000E941CF00CC08DE190E0F8019183808337
:1001600086E2818B81E090E0918F808F228FD70192
:100170001496ED91FC911597EC55FA4F8081918181
:10018000A281B381F801828B938BA48BB58B808184
:1001900091814A97978B868B80919507833020F4C5
:1001A0008F5F8093950702C01092950790919507F5
:1001B00080919607981741F4933020F49F5F9093B5
:1001C000960702C01092960780915119909152198A
:1001D0000E9436270F90CF91DF911F910F91FF90D2
:1001E000EF9008950F931F93DF93CF930F92CDB7A6
:1001F000DEB78C011982809151199091521960E0FB
:1002000070E0AE014F5F5F4F0E94C228809193075C
:1002100090E026E331E0829FA001839F500D929FE2
:10022000500D1124435A5645D8011496ED91FC9176
:100230001597E25DFA4F80812EE0829FC001112464
:100240008B96FA019183808322E030E0338322830E
:1002500020E8248741979687858780E290E0A0E098
:10026000B0E08787908BA18BB28B81E0838BD80124
:100270001496ED91FC911597DA015496E65EFA4FCB
:1002800085E801900D928150E1F7809193078730C6
:1002900020F48F5F8093930702C010929307909190
:1002A000930780919407981741F4973020F49F5F4B
:1002B0009093940702C010929407809151199091E5
:1002C00052190E94362780E00F90CF91DF911F9145
:1002D0000F910895CF93DF93EC01EC81FD81E25DF6
:1002E000FA4F80818823D1F0CE010E94F2808C8168
:1002F0009D81865E9A4FFC0185E8DF011D928A95FB
:10030000E9F78C819D81DC01A25EBA4FFC01EC5FB4
:10031000FA4F80E101900D928150E1F78FEFDF916C
:10032000CF9108950F931F93CF93DF938C01009784
:10033000C1F0DC01CD91DC91209799F0CE010E94B3
:1003400077F09C012C0F3D1FF90101900020E9F787
:100350003197E21BF30BE20FF31FD801ED93FC93EF
:1003600002C02EE634E0C901DF91CF911F910F91B9
:100370000895EF92FF920F931F93CF93DF938C0119
:100380007B010097C1F0DC01CD91DC91209799F0C1
:10039000CE010E9477F0C80FD91FCE01B7010E948D
:1003A00040F0FE01E80FF91F808181111192D80100
:1003B000ED93FC9302C0CEE6D4E0CE01DF91CF9165
:1003C0001F910F91FF90EF9008958F929F92AF929F
:1003D000BF92CF92DF92EF92FF920F931F93DF9322
:1003E000CF930F92CDB7DEB75C018B014A01198222
:1003F000FC01818160E075E06E010894C11CD11C94
:10040000A6010E94B832982F8981882361F5F801EE
:10041000908321E0E22EF12CF501818164E670E009
:10042000A6010E94B832982F89818823E1F4F8014F
:1004300091830894E11CF11CC80164E974E042E076
:1004400050E00E9459F0009711F48FEF08C00F5F41
:100450001F4FF0E0EF16F4E0FF06F1F680E0F40144
:10046000F182E08201C080E00F90CF91DF911F9177
:100470000F91FF90EF90DF90CF90BF90AF909F9043
:100480008F9008958F929F92AF92BF92CF92DF92FA
:10049000EF92FF920F931F93DF93CF930F92CDB7FD
:1004A000DEB76C017B018A01CA0101978F3F91057C
:1004B00008F058C0198233E0B32E4E010894811C15
:1004C000911C2EC0F6018181F70160814AE050E065
:1004D0000E94F331882309F045C0F6018181198219
:1004E00060E870E0A4010E94B832A82E89818823B8
:1004F00051F0BB20B9F1BA9480E060E040E024E61E
:1005000030E00E942A2EF7018081A81639F4089461
:10051000E11CF11C01501040BB2402C0BB2011F1B2
:100520000115110579F6F60181816DE04AE050E090
:100530000E94F3318823B1F4F601818119826AE0C7
:1005400070E08E010F5F1F4FA8010E94B832F601C4
:1005500081816AE070E0A8010E94B8328A3011F40B
:100560008FEF01C080E00F90CF91DF911F910F912D
:10057000FF90EF90DF90CF90BF90AF909F908F90C3
:1005800008954F925F926F927F928F929F92AF9257
:10059000BF92CF92DF92EF92FF920F931F93DF9360
:1005A000CF93CDB7DEB728970FB6F894DEBF0FBE56
:1005B000CDBF6C012A013B011A821982DC01119620
:1005C0002C91922F990F990F80E08F5A9247FC013E
:1005D00080E094E0DF019C011D9221503040E1F762
:1005E000D60111969C9180E08F5A96470E94D2F0D6
:1005F000F601918180E0DC01AF5AB647FD01019020
:100600000020E9F73197EA1BFB0BFA83E983359762
:1006100008F433C1BC83AB8380E28D8389E08E8391
:100620008DE08F838AE08887F3E0AF2EB12CAC0E8B
:10063000BD1EE5E08E2E912C8C0E9D1EC501B401D1
:100640000E94B9818C016FE674E043E050E00E94A3
:1006500059F0009709F090C0C501B4010E94B9811A
:100660008C0163E774E043E050E00E9459F000978A
:1006700049F4D6011496ED91FC911597EC5EFA4F72
:10068000108254C0C80167E774E043E050E00E9464
:1006900059F0009709F0F1C0C501B4010E94B98179
:1006A0008C010E9477EF282FF8018081882309F4BC
:1006B000E4C07B01022F192FE114F104010511059B
:1006C00009F4DBC0C501B4010E94B981FC0180813D
:1006D000882329F428E030E040E050E008C0CF0152
:1006E0000E9477EFAC01CB01DA019C01AD01DA0188
:1006F000C9010197A109B1090897A105B10508F041
:10070000BCC0D6011496ED91FC911597EC5EFA4FA2
:100710008FEF80831496ED91FC911597E050FB4F7D
:10072000E082F18202831383799620831496ED91FF
:10073000FC911597EB5EFA4F1082118212821382A0
:10074000C6010E946A81F6012181922F990F990FAB
:1007500080E08F5A924767E97DE042E050E00E94D6
:10076000ABEFD6011196EC91F0E0EE0FFF1FEF5AC0
:10077000F24682E090E099C0C8016BE774E043E084
:1007800050E00E9459F0009709F077C0C501B4010C
:100790000E949281F82EE92EE82FF92FDF010D90AB
:1007A0000020E9F78D01015010400E1B1F0B09F4CA
:1007B00064C0D6011496ED91FC911597EC5EFA4F4A
:1007C0008081882309F040C060E040E024E630E00A
:1007D0000E942A2EC6016F2D7E2DA8010E94428202
:1007E0001A821982F6016481758160507F4FC601BB
:1007F000AE014F5F5F4F0E94E581E981FA81CF0131
:1008000001978F5F9340C8F5D60111968C9111978F
:10081000382F330F330F20E02F5A324714964D9163
:100820005C91159740505F4FC901BA01AF010E941A
:100830001CF0D6011196EC91F0E0EE0FFF1FEF5A7D
:10084000F24689819A8131C0F6012181922F990F58
:10085000990F80E08F5A92476AE77DE04CE150E0C3
:100860000E94ABEFD6011196EC91F0E0EE0FFF1F66
:10087000EF5AF2468CE190E018C0F6012181922FE8
:10088000990F990F80E08F5A924765E67DE044E129
:1008900050E00E94ABEFD6011196EC91F0E0EE0F24
:1008A000FF1FEF5AF24684E190E091838083C601F6
:1008B000B301A2010E947E7E8FEF28960FB6F894B6
:1008C000DEBF0FBECDBFCF91DF911F910F91FF9083
:1008D000EF90DF90CF90BF90AF909F908F907F90E0
:1008E0006F905F904F9008956F927F928F929F923A
:1008F000AF92BF92CF92DF92EF92FF921F93DF935E
:10090000CF93CDB7DEB766970FB6F894DEBF0FBEB4
:10091000CDBF6C01DC011496ED90FC901597E0E0E2
:10092000F1E0EE0EFF1EDE011796E7E8F4E086E048
:1009300001900D928150E1F784E48D8383E58E83ED
:1009400080E060E040E024E630E00E942A2E1C8235
:100950001B82C601BE016B5F7F4F42E050E00E94E8
:100960004282D60114966D917C91159760507F4F0D
:10097000C601AE014D5F5F4F0E94E581BDE0AB2E29
:10098000B12CAC0EBD1E10E0A7E06A2E712C6C0ECF
:100990007D1E4E010894811C911CC701B301A40166
:1009A0000E94A0F0009709F442C0F5018193919351
:1009B0005F011F5FEE24FF24153079F78B899C8936
:1009C0006FE774E00E9437F0009789F58D899E8962
:1009D0000E9477EF2DB73EB7285030400FB6F894FD
:1009E0003EBF0FBE2DBFEDB7FEB73196D6011496B0
:1009F0002D913C9115972C5F3A4FADB7BEB712962B
:100A00003C932E93119723E834E03383228364834D
:100A10007583868397830E942DF18FEFEDB7FEB724
:100A200038960FB6F894FEBF0FBEEDBF01C080E050
:100A300066960FB6F894DEBF0FBECDBFCF91DF91A3
:100A40001F91FF90EF90DF90CF90BF90AF909F905D
:100A50008F907F906F900895AF92BF92CF92DF9268
:100A6000EF92FF920F931F93DF93CF9300D00F92DB
:100A7000CDB7DEB76C01162F5C834B838DB79EB765
:100A800008970FB6F8949EBF0FBE8DBFEDB7FEB7A7
:100A9000319683EF98E1ADB7BEB712969C938E93D3
:100AA000119787E59EE093838283648315828B810F
:100AB0009C81978386830E9451F1EDB7FEB73896EB
:100AC0000FB6F894FEBF0FBEEDBF183509F4A5C0F0
:100AD000193578F4193409F47AC11A3420F413342E
:100AE00009F051C2DDC01235B1F0133509F04BC227
:100AF000EDC1123781F0133738F4133609F4D0C042
:100B0000193609F040C263C1133709F4DFC1183741
:100B100009F039C282C000D00F9283EF98E1ADB7DF
:100B2000BEB712969C938E9311978BE49EE0149619
:100B30009C938E9313970E9451F10F900F900F90FA
:100B40000F9013E0A12EB12CAC0EBD1EF6016481F6
:100B5000758168557A4FC5010E94B9818C010E9448
:100B600077EF282FD8018C91882309F40CC27B01E0
:100B7000022F192FE114F1040105110509F403C234
:100B8000F6016481758168557A4FC5010E94B9816B
:100B9000FC018081882329F428E030E040E050E027
:100BA00008C0CF010E9477EFAC01CB01DA019C01B4
:100BB000AD01DA01C9010197A109B1090897A105A1
:100BC000B10508F0E0C1D6011496ED91FC9115979E
:100BD000EC5EFA4F8FEF80831496ED91FC911597A0
:100BE000E050FB4FE082F1820283138379962083E9
:100BF0001496ED91FC911597EB5EFA4F10821182DD
:100C000012821382C6010E946A81F6018481958155
:100C100084549A4F68E47EE02EC000D00F9283EF98
:100C200098E1EDB7FEB7928381838BE39EE09483D6
:100C300083830E9451F1D6011496ED91FC91159792
:100C4000EC5EFA4F10821496ED91FC911597EB5ED5
:100C5000FA4F10821182128213820F900F900F9020
:100C60000F90C6010E946A81F601848195818454A7
:100C70009A4F68E37EE042E050E00E94ABEFD6017D
:100C80001496ED91FC911597EF55FA4F81E0808312
:100C90001496ED91FC911597ED55FA4F82E079C0CD
:100CA00000D00F9283EF98E1EDB7FEB79283818376
:100CB00089E29EE0948383830E9451F10F900F900C
:100CC0000F900F90D60114966D917C9115976855F1
:100CD0007A4FCE0103960E949281F82EE92EE82FDA
:100CE000F92FDF010D900020E9F78D010150104030
:100CF0000E1B1F0B09F447C1D6011496ED91FC9110
:100D00001597EC5EFA4F8081E451F540882309F095
:100D100043C060E040E024E630E00E942A2EC60195
:100D20006F2D7E2DA8010E9442821A821982F6013F
:100D30006481758160507F4FC601AE014F5F5F4F88
:100D40000E94E581E981FA81CF0101978F5F93408D
:100D500008F019C1D60114962D913C911597A9015F
:100D600044545A4F20503F4FCA01B901AF010E946D
:100D70001CF0D6011496ED91FC911597ED55FA4FA4
:100D8000898180831496ED91FC911597EF55FA4F68
:100D900081E080831FEFF8C0CF0184549A4F6CE04C
:100DA0007EE04CE150E00E94ABEFF601A481B581FA
:100DB000CD0184549A4FFC0101900020E9F731974E
:100DC000E81BF90BAD55BA4FEC93D601DBCF00D041
:100DD0000F9283EF98E1EDB7FEB79283818381E0B4
:100DE0009EE0948383830E9451F10F900F900F90A7
:100DF0000F90C6010E947484182FD60114962D916D
:100E00003C9115978F3F89F500D000D0EDB7FEB724
:100E1000319624543A4FADB7BEB712963C932E93F9
:100E2000119787EE9DE093838283285B3040358362
:100E300024830E9451F1F601A481B581CD0184542F
:100E40009A4FFC0101900020E9F73197E81BF90B5C
:100E5000AD55BA4FEC93D6011496ED91FC911597D0
:100E6000EF55FA4F81E0808385C000D00F92245463
:100E70003A4FADB7BEB712963C932E93119781ECC3
:100E80009DE014969C938E9313970E9451F1F60166
:100E9000A481B581CD0184549A4FFC0101900020BA
:100EA000E9F73197E81BF90BAD55BA4FEC93D60132
:100EB0001496ED91FC911597EF55FA4F81E08083E0
:100EC0001FEF0F900F900F900F905EC000D00F9209
:100ED00083EF98E1EDB7FEB79283818382EB9DE0CB
:100EE000948383830E9451F1F601A481B581AC5EA5
:100EF000BA4F0F900F900F900F908C91A451B54066
:100F0000882319F42DE834E002C021E934E000D050
:100F100000D04DB75EB74F5F5F4FA454BA4FEDB7E7
:100F2000FEB7B283A1838AE99DE0DA0113969C9310
:100F30008E93129715963C932E9314970E9451F11D
:100F4000F601A481B581CD0184549A4FFC01019032
:100F50000020E9F73197E81BF90BAD55BA4FEC9338
:100F6000D6011496ED91FC911597EF55FA4F81E05B
:100F700080831FEFEDB7FEB736960FB6F894FEBF2D
:100F80000FBEEDBF01C010E0812F0F900F900F90AA
:100F90000F90CF91DF911F910F91FF90EF90DF9015
:100FA000CF90BF90AF9008958F929F92AF92BF92D3
:100FB000CF92DF92EF92FF920F931F93DF93CF9325
:100FC0000F920F92CDB7DEB76C01DC018C9190E0EF
:100FD00029E031E0F9018E9F90018F9F300D9E9F97
:100FE000300D11242E5832463A83298300D000D088
:100FF000EDB7FEB7319693EF892E98E1992EADB7F4
:10100000BEB712969C928E9211978CE99EE09383C4
:101010008283358324830E9451F1E981FA81E15072
:10102000FF4F1082F6018481958188559A4FFC010B
:1010300084E1DF011D928A95E9F7EDB7FEB7369698
:101040000FB6F894FEBF0FBEEDBFD60114968D917A
:101050009C91159788559A4F68E372E00E94B4EF0F
:10106000F6016481758168557A4F89819A818E0174
:101070000F5F1F4FA8010E94A0F05C01009719F4B8
:10108000FF24F39426C085E59DE00E94C6EFAC01E5
:10109000C50165E57DE00E94CFEF892B19F082E064
:1010A000F82E17C0D6011496ED91FC911597E855CE
:1010B000FA4FC80162E37DE047E025E00AE51DE064
:1010C0007F010E941F38182F882309F0BEC003E05B
:1010D000F02E00D000D0EDB7FEB7319603EF18E147
:1010E000ADB7BEB712961C930E93119780E89EE0A1
:1010F00093838283F48215820E9451F10F920F92A2
:10110000EDB7FEB73196ADB7BEB712961C930E93EE
:10111000119781E79EE09383828389819A819583E9
:101120008483B782A6820E9451F1EDB7FEB738964C
:101130000FB6F894FEBF0FBEEDBFF2E0FF1679F0D8
:1011400043E0F416A9F0D6011496ED91FC911597A1
:10115000B1E0FB16B1F4EF55FA4F8DE015C0D601A2
:101160001496ED91FC911597EF55FA4F8EE00CC057
:10117000D6011496ED91FC911597EF55FA4F8AE040
:1011800003C0EF55FA4F8FE08083C6010E9429808B
:10119000F601808190E029E031E0AC01429FC0017E
:1011A000439F900D529F900D11248E589246FC0142
:1011B00080E091E0DF01AC011D9241505040E1F729
:1011C000D6018C9190E0829FF001839FF00D929F59
:1011D000F00D1124E759F246118210828C9190E0B3
:1011E000829FF001839FF00D929FF00D1124E7592B
:1011F000F24612828C9190E0829FF001839FF00D65
:10120000929FF00D1124E759F246148213828C91BB
:1012100090E0829FF001839FF00D929FF00D1124CA
:10122000E759F24615821682178210860F900F90AA
:10123000CF91DF911F910F91FF90EF90DF90CF90B2
:10124000BF90AF909F908F90089500D00F92EDB710
:10125000FEB7928281828FE89EE0948383830E940E
:1012600051F10F900F900F900F9049815A81C60154
:10127000612F0E942C85F82EFFEF8F1709F485CF80
:101280005CCF4F925F926F927F928F929F92BF92AC
:10129000CF92DF92EF92FF920F931F93DF93CF9342
:1012A000CDB7DEB7A4970FB6F894DEBF0FBECDBFA3
:1012B0007C0184E5898393E59A8384E48B839C8312
:1012C000D70114960D911C911597DE011996E7E848
:1012D000F4E086E001900D928150E1F718861F82BC
:1012E000F7018481958180509F4FFC0180E094E05C
:1012F000DF019C011D9221503040E1F7C701BE0182
:101300006F5F7F4F42E050E00E944282D701149607
:101310006D917C91159760507F4F97E0C92ED12C2D
:10132000CC0EDD1EC701A6010E94E5818F81988544
:101330000B9709F024C1412C81E0582E400E511E1C
:10134000F70144815581BA0160507F4F425D5A4F89
:10135000DA01BC904E5255408B2D90E0880F991FBA
:10136000FC01A3E0EE0FFF1FAA95E1F7E81BF90BC4
:10137000E40FF51FE15DFA4FDB010D911D912D91F9
:101380003C91139700831183228333838B2D90E04C
:10139000880F991F9C0163E0220F331F6A95E1F7C4
:1013A000281B390B420F531F4D5C5A4F14968D91D9
:1013B0009D910D90BC91A02DFA0180839183A28311
:1013C000B38380E060E040E024E630E00E942A2E13
:1013D00018861F82C701BE016D5F7F4F42E050E05B
:1013E0000E944282D70114966D917C9115976050AE
:1013F0007F4FC701A6010E94E5819FE0C92ED12C35
:10140000CC0EDD1E00E089E0682E712C6C0E7D1E76
:1014100015E0812E912C8C0E9D1EC201B301A401FA
:101420000E94A0F0009709F497C0F6018193919370
:101430006F010F5F442455240B3079F78D899E8905
:101440006FE774E00E9437F0009709F085C0D7017C
:1014500014960D911C911597898D9A8D0E9459EFC4
:101460002B2D30E0220F331FF901A3E0EE0FFF1FF9
:10147000AA95E1F7E21BF30BE00FF11FE95CFA4FCD
:1014800080838B8D9C8D0E94967F2B2D30E0220FC8
:10149000331FF90173E0EE0FFF1F7A95E1F7E21BAE
:1014A000F30BE00FF11FE85CFA4F80838D8D9E8D6A
:1014B0000E9459EF2B2D30E0220F331FF90153E02A
:1014C000EE0FFF1F5A95E1F7E21BF30BE00FF11F40
:1014D000E75CFA4F805D80838F8D98A10E9459EF61
:1014E0002B2D30E0220F331FF90193E0EE0FFF1F89
:1014F0009A95E1F7E21BF30BE00FF11FE65CFA4F60
:10150000808389A19AA10E9459EF2B2D30E0220FF0
:10151000331FF901A3E0EE0FFF1FAA95E1F7E21BCD
:10152000F30BE00FF11FE55CFA4F80838BA19CA1C8
:101530000E9459EF2B2D30E0220F331FA90163E0E9
:10154000440F551F6A95E1F7421B530B040F151FFB
:10155000045C1A4FF8018083D7011496ED91FC9139
:101560001597DF01A25DBA4F8C918F5F8C93E75E78
:10157000FA4F9081891718F0C7010E946A81A496DA
:101580000FB6F894DEBF0FBECDBFCF91DF911F9194
:101590000F91FF90EF90DF90CF90BF909F908F9032
:1015A0007F906F905F904F900895AF92BF92CF92CF
:1015B000DF92EF920F931F93DF93CF9300D000D071
:1015C000CDB7DEB75C011A821982DC0111968C91CD
:1015D000813021F4C12C53E0D52E0EC0823021F48D
:1015E000C12C45E0D42E08C0833021F4C12C37E053
:1015F000D32E02C0CC24DD24D5011496ED91FC91AC
:101600001597309741F08CEB96E0DF019C011D921D
:1016100021503040E1F7D50111968C9140E855E218
:1016200060E070E026E000E0EE240E943833F5012F
:1016300081816FEF40E00E94A238C114D104B9F15A
:101640008601005C1F4F23E0C22ED12CCC0EDD1E84
:10165000C801B60144E050E00E9467378B819C814D
:10166000AD81BE810197A109B1098E5F9F4FAF4F38
:10167000BF4F70F08CE390E0A0E0B0E08B839C83E0
:10168000AD83BE83C801B60144E050E00E94F73745
:10169000D5011496ED91FC911597E050FB4F8B818D
:1016A0009C81AD81BE8180839183A283B38380E0DE
:1016B00060E041E020E030E00E942A2EF5018181C7
:1016C0006DE04AE050E00E94F331D50114966D912F
:1016D0007C91159760507F4FC501AE014F5F5F4F02
:1016E0000E94E581C5010E947484F5018481958181
:1016F000DC01A25EBA4FFC01EC5FFA4F80E1019081
:101700000D928150E1F760E040E024E630E00E9475
:101710002A2ED5011496ED91FC911597E75EFA4FAC
:1017200088E0808335971192108211821282138291
:101730008FEF26960FB6F894DEBF0FBECDBFCF91C8
:10174000DF911F910F91EF90DF90CF90BF90AF90FE
:1017500008958FEF80939EA181E060E040E020E05B
:1017600030E00E942A2EF8CF0F931F93CF93DF9380
:10177000EC018C819D818F58994FFC0184E6DF013B
:101780001D928A95E9F78C819D818B52994FFC01BE
:1017900080E091E0DF019C011D9221503040E1F793
:1017A0008C819D816F3F29F48F58994F6EEE7FE0B9
:1017B00004C08F58994F67EF7FE00E94B4EF8C818F
:1017C0009D818F58994F6FEF7FE00E94B4EFEC81BD
:1017D000FD81E95AFA4F8081E65EFE4F8F3F21F48A
:1017E000CF0167EE7FE003C0CF016AEE7FE00E9489
:1017F000B4EF8C819D818F58994F65E070E10E9414
:10180000B4EFEC81FD81EA5AFA4F8081E55EFE4F2C
:101810008F3F21F4CF0167EE7FE003C0CF016AEE76
:101820007FE00E94B4EFEC81FD81EC5FFA4F808194
:101830009181E359FE4F8F3F910529F020F0CF01B0
:101840006DE070E103C0CF016FE470E10E94B4EF7E
:10185000AC81BD81A050BB4F6D917D914D915C914C
:101860001197AE50BD4F2D913C91119716968C91CA
:10187000AA5FB740882319F486E994E002C08AE998
:1018800094E0EDB7FEB73E970FB6F894FEBF0FBEDB
:10189000EDBF0DB71EB70F5F1F4FAB52B94FB283ED
:1018A000A183A456B040F801B383A28375836483F7
:1018B000578346833187208793878287AD56B1400F
:1018C0008D919C91958784870E942DF1EC81FD81FB
:1018D000EA5AF94F81E08083AC81BD81CD018B5202
:1018E000994FFC0101900020E9F73197E81BF90BB3
:1018F000A85AB94FEC932DB73EB7225F3F4F0FB6B2
:10190000F8943EBF0FBE2DBF8FEFDF91CF911F9197
:101910000F910895CF93DF93EC018C819D818B52C1
:10192000994FFC0180E091E0DF019C011D92215064
:101930003040E1F78C819D81FC01EA5EFA4F208105
:101940008B52994F222321F0BF010E942CF004C03A
:1019500062E471E10E94B4EFEC81FD81CF018B5212
:10196000994FDC010D900020E9F71197A81BB90BE6
:10197000E85AF94FA0838FEFDF91CF9108950F932D
:101980001F93CF93DF938C01EB016115710511F467
:10199000C2E0D0E0CE0101978F5F9E4F10F080E053
:1019A00014C0D80112968D919C9113978C5B9F4F18
:1019B000BE010E94D637D8011496ED91FC9115977F
:1019C000EE5FFA4FD183C0838FEFDF91CF911F91EC
:1019D0000F9108951F93CF93DF93EC01162F862F5D
:1019E00081508A3010F080E00EC08A819B818E5B2E
:1019F0009F4F70E00E94D637EC81FD81EE5FFA4F79
:101A0000108311828FEFDF91CF911F910895EF9294
:101A1000FF920F931F93DF93CF930F92CDB7DEB753
:101A20007C011982809151199091521960E070E007
:101A3000AE014F5F5F4F0E94C2288091950790E0F2
:101A400026E331E0829F8001839F100D929F100D4D
:101A50001124035F1C4480E290E0D80113969C930C
:101A60008E93129782E01C968C93D7011496ED9179
:101A7000FC911597EC5AF94F81919191D8011E96DE
:101A80009C938E931D97D7018C9190E02091E40355
:101A90003091E503822B932BD80150969C938E9323
:101AA0001F972081E655F6402A3020F5E85AF94F75
:101AB000408150E0425E5F4F11965C934E934E51D1
:101AC00050408DE351968C9351975B965C934E9367
:101AD0005A9759962C935997829158968C939801BE
:101AE000245E3F4FE258FF4FC901BF0150E00E9402
:101AF0001CF00CC08DE190E0F8019183808386E2B8
:101B0000818B81E090E0918F808F228FD701149696
:101B1000ED91FC911597E75AF94F80819181A2814F
:101B2000B381F801828B938BA48BB58B80819181DB
:101B30004A97978B868B80919507833020F48F5F2F
:101B40008093950702C01092950790919507809118
:101B50009607981741F4933020F49F5F909396076F
:101B600002C01092960780915119909152190E94CB
:101B700036270F90CF91DF911F910F91FF90EF903B
:101B800008950F931F93DF93CF930F92CDB7DEB7D6
:101B90008C011982809151199091521960E070E086
:101BA000AE014F5F5F4F0E94C2288091930790E083
:101BB00026E331E0829FF001839FF00D929FF00DAC
:101BC0001124E35AF645DF01C9011D920197E9F797
:101BD000D80114964D915C9115974D595A4FDA01E1
:101BE0002C9188E1289F90011124275E3F4F31837B
:101BF000208382E090E09383828381E9848721516E
:101C00003040368725873F961797CF01BD01A90140
